:100000000C94150D0C94360D0C94360D0C94360D85
:100010000C94360D0C94360D0C94360D0C94360D54
:100020000C94360D0C94360D0C9420580C943D58BD
:100030000C94360D0C94360D0C94FE580C942B59E0
:100040000C9458590C9485590C94B2590C94DF595E
:100050000C940C5A0C94395A0C94665A0C94935A7A
:100060000C94360D0C94A8F90C94DFF90C94360D11
:100070000C94360D0C94360D0C94360D0C94360DF4
:100080000C94360D0C94360D0C94360D0C94360DE4
:100090000C94360D0C94360D0C94360D0D9488246A
:1000A0000D94BA240D94EC240D941E250C9458E064
:1000B0000C94360D0C94360D0C94360D0C94825C19
:1000C0000C94AF5C0C94DC5C0C94095D0C94365D74
:1000D0000C94635D0C94905D0C94BD5D0C94EA5D92
:1000E0000C94175E0C94360D0C94CCF80C9403F918
:1000F0000C94360D0C94360D0C94360D0C94360D74
:100100000C94360D0C94360D0C9469E30C94360D5A
:100110000C94360D0C94360D0C94360D0D94C023B2
:100120000D94F2230D9424240D9456240C94360D32
:100130000C94360D0C94C05A0C94ED5A0C941A5B26
:100140000C94475B0C94745B0C94A15B0C94CE5B99
:100150000C94FB5B0C94285C0C94555C0C94360D51
:100160000C943AF90C9471F90C94360D0C94360DEC
:100170000C94360D0C94360D0C94360D0C94360DF3
:100180000C94360D0C94360D0C94360D0C94360DE3
:100190000C94360D0C94360D0C94360D0C94360DD3
:1001A0000C9425E00C94360D0C94360D0C94360D01
:1001B0000C94445E0C94715E0C949E5E0C94CB5E29
:1001C0000C94F85E0C94255F0C94360D0C94360D4F
:1001D0000C94360D0C94360D0C94360D0C9416FAC6
:1001E0000C944DFA0C94360D0C94360D0C94360D7F
:1001F0000C94360D0C94BD6A0C94786BEF0D720E56
:10020000010E720E130E720E250E3F0E250E590EA4
:100210002010341048106E1094100F11FC100F11A4
:10022000D610301630166816A516E9162616D217FF
:10023000EE172B1889172C1F361F401F4A1F541FFB
:100240005E1F681F6D1F721F7C1FEA23EA23F123C4
:10025000F12304242724EA232724F12360246024A3
:10026000682468247D24A4246024A4246824882588
:100270009325A225BD25D325F5253B2644265F26BB
:100280001B265E51D551D551EE50D551D551D55182
:10029000D551D551D551D551D551D551D551D5512E
:1002A000D551D551D5510351D551D551D551D551F0
:1002B000D551D551D5515851B651D551D551C351BC
:1002C000D551D551D551D551D551D5517151D55162
:1002D000D551CF51D551D251D551D551D551D551F7
:1002E000CC51D551D551D551D551D551D551D551E7
:1002F000D551D551D551D551D551D551D551D551CE
:10030000D551D551D551D551D551D551D551D551BD
:10031000D551D551D551D551D551D551D551D551AD
:10032000D551D551D551D551D551D551D551D5519D
:10033000D551D551D5515B519165946597659A65B5
:100340009D65A065A365106D236D366D496D5C6D6F
:100350006F6D826D40724072047204720472BD71DE
:10036000BD71047204720472047204720472047225
:1003700004720472047204720472047204720472CD
:10038000BD71047204720472047204724E81987F0B
:10039000D17F11806780B280C780F9801B813C814A
:1003A00001838E819681B381F28105824F827182B1
:1003B00088829D82FC82FC82FC82FC82FC82FC8220
:1003C000FC82FC82FC82FC82B482BC82C782DC821A
:1003D000E28256A359A3AAA3AAA3AAA3AAA3AAA343
:1003E000AAA3AAA3AAA3AAA3AAA3AAA3AAA3AAA3A5
:1003F000AAA3AAA3AAA3AAA3AAA3AAA390A3AAA3AF
:10040000AAA3AAA3AAA3AAA3AAA376A3AAA3AAA3B8
:10041000AAA3AAA3AAA35CA3AAA3AAA3AAA3AAA3C2
:10042000AAA3AAA3AAA3AAA3AAA3AAA3AAA3AAA364
:10043000AAA3AAA3AAA3AAA3AAA3AAA390A3AAA36E
:10044000AAA3AAA3AAA3AAA3AAA376A3AAA3AAA378
:10045000AAA3AAA3AAA35CA353A650A665A665A6B1
:1004600065A665A665A665A665A665A665A665A634
:1004700065A665A665A665A665A69CA56FA58DA5BE
:1004800065A665A613A656A565A665A665A665A676
:1004900065A67EA556A665A665A6A6A565A665A6BB
:1004A00065A665A665A665A665A665A665A665A6F4
:1004B00065A665A665A665A665A69CA56FA58DA57E
:1004C00065A665A613A656A565A665A665A665A636
:1004D00065A67EA556A665A665A6A6A5DFA722A841
:1004E0002CA82CA82CA82CA82CA82CA82CA82CA86C
:1004F0002CA82CA82CA82CA82CA816A72CA8CDA7D3
:10050000C7A72FA7D9A72CA82CA83FA716A72CA808
:100510002CA8EEA723A7D3A727A82CA835A7E4A724
:10052000C1A73AA72CA8E9A712A72CA82CA82CA8E9
:1005300029A72CA82CA82CA82CA82CA82CA8CDA77F
:10054000C7A72FA7D9A72CA82CA83FA716A72CA8C8
:100550002CA8EEA723A7D3A727A82CA835A7E4A7E4
:10056000C1A73AA72CA8E9A712A72CA82CA82CA8A9
:1005700029A7F2A603AEF3ADF5ADF7ADF9ADFBAD2E
:10058000FDADFFAD20AE10AE12AE14AE16AE18AE7D
:100590001AAE1CAE4DAE6FAE55AE6FAE55AE6FAE71
:1005A00055AE6FAE55AE6FAE55AE6FAE6FAE6FAEB1
:1005B0006FAE6FAE6FAE6FAE5CAE63AEC9C1F8BF6B
:1005C00004C04FC080C164C0A6C0CAC0F3C04EC141
:1005D0008CC48CC4CEC4A9C53AC62AC72CC8E3C8EB
:1005E0002CC8F7C9DBCBDBCBF7CB38CC58CC87CCCE
:1005F000BCCCDCCCBCCC0BCD45CF78CFABCF2CD09A
:10060000A0D067D15ED2E8D25ED2BCD34E414E4973
:100610004E495459494E46CDCCCC3D0AD7233C17C0
:10062000B7D13877CC2B329595E6241FB14F0A000D
:100630000020410000C84200401C4620BCBE4CCAFD
:100640001B0E5AAEC59D743235304D4F686D003269
:10065000354D4F686D003630487A003530487A00A5
:100660004E6F6E2D496E740048692D4C4F004750F7
:10067000530054696D650044697374616E6365006D
:100680005075736820427574746F6E00496D7065A3
:100690007269616C004D657472696300494E430074
:1006A000444543004F4E004F46460026072107179A
:1006B0000710070407FD06F106E006D206BF063262
:1006C00078496D702E204349505326327844435662
:1006D0004700506172616C6C656C20434950530057
:1006E0003278496D702E2043495053264443564773
:1006F000003278496D702E204349505300347844BD
:1007000043564700434950532632784443564700E6
:100710003278444356470043495053264443564792
:100720000044435647004349505300600F9E0EDC7F
:100730000D1A0D580C960BD40A120A50098E08C1D6
:100740000FFF0E3D0E7B0DB90CF70B350B730AB185
:1007500009EF0853616D706C652F7365633A00454E
:1007600052524F5220202020202000432D43495038
:10077000532C20522D434950532C200000000000E0
:100780000000000000000000000000000000000069
:100790000000000000000000000000000000000059
:1007A0000000000000000000000000000000000049
:1007B0000000000000000000000000000000000039
:1007C0000000000000000000000000004C6F2D43FE
:1007D0004950532C2048692D434950532C20000088
:1007E0000000000000000000000000000000000009
:1007F00000000000000000000000000000000000F9
:1008000000000000000000000000000000000000E8
:1008100000000000000000000000000000000000D8
:1008200000000000000000000000000000434950EC
:10083000532C200000000000000000000000000019
:1008400000000000000000000000000000000000A8
:100850000000000000000000000000000000000098
:100860000000000000000000000000000000000088
:100870000000000000000000000000000000000078
:100880000000000000000000000000000000522DE9
:1008900044435647204F6E2C204C2D44435647204E
:1008A0004F6E2C204C6F2D43495053204F6E2C20FF
:1008B00048692D43495053204F6E2C20522D4443FC
:1008C0005647204F66662C204C2D44435647204FF8
:1008D00066662C204C6F2D43495053204F66662C82
:1008E0002048692D43495053204F66662C20005202
:1008F0002D44435647204F66662C204C2D444356CA
:1009000047204F66662C204C6F2D43495053204F93
:1009100066662C2048692D43495053204F66662C4B
:1009200020522D44435647204F6E2C204C2D4443DB
:100930005647204F6E2C204C6F2D43495053204F6B
:100940006E2C2048692D43495053204F6E2C2000B7
:10095000432D43495053204F6E2C20522D43495074
:1009600053204F6E2C20432D43495053204F666631
:100970002C20522D43495053204F66662C200000F6
:100980000000000000000000000000000000000067
:100990000000000000000000000000000000000057
:1009A0000000000000000000000000000000000047
:1009B00000432D43495053204F66662C20522D434F
:1009C000495053204F66662C20432D4349505320F5
:1009D0004F6E2C20522D43495053204F6E2C200037
:1009E0000000000000000000000000000000000007
:1009F00000000000000000000000000000000000F7
:100A000000000000000000000000000000000000E6
:100A10000000522D44435647204F6E2C204C6F2D22
:100A200043495053204F6E2C2048692D4349505361
:100A3000204F6E2C20522D44435647204F66662C83
:100A4000204C6F2D43495053204F66662C20486937
:100A50002D43495053204F66662C200000000000B3
:100A60000000000000000000000000000000000086
:100A7000000000522D44435647204F66662C204C00
:100A80006F2D43495053204F66662C2048692D43F3
:100A9000495053204F66662C20522D444356472020
:100AA0004F6E2C204C6F2D43495053204F6E2C20FD
:100AB00048692D43495053204F6E2C200000000000
:100AC0000000000000000000000000000000000026
:100AD000000000004C6F2D43495053204F6E2C20D6
:100AE00048692D43495053204F6E2C204C6F2D43A5
:100AF000495053204F66662C2048692D4349505376
:100B0000204F66662C20000000000000000000005E
:100B100000000000000000000000000000000000D5
:100B200000000000000000000000000000000000C5
:100B300000000000004C6F2D43495053204F666663
:100B40002C2048692D43495053204F66662C204C79
:100B50006F2D43495053204F6E2C2048692D434937
:100B60005053204F6E2C20000000000000000000B9
:100B70000000000000000000000000000000000075
:100B80000000000000000000000000000000000065
:100B9000000000000000522D44435647204F6E2CA9
:100BA000204C2D44435647204F6E2C20462D444365
:100BB0005647204F6E2C20422D44435647204F6EFF
:100BC0002C20522D44435647204F66662C204C2D36
:100BD00044435647204F66662C20462D44435647D3
:100BE000204F66662C20422D44435647204F6666B0
:100BF0002C200000000000522D44435647204F6631
:100C0000662C204C2D44435647204F66662C2046C8
:100C10002D44435647204F66662C20422D444356B0
:100C200047204F66662C20522D44435647204F6E76
:100C30002C204C2D44435647204F6E2C20462D44EB
:100C4000435647204F6E2C20422D44435647204F99
:100C50006E2C200000000000522D44435647204FC8
:100C60006E2C204C2D44435647204F6E2C20434978
:100C70005053204F6E2C20522D44435647204F6630
:100C8000662C204C2D44435647204F66662C20434B
:100C9000495053204F66662C2000000000000000E1
:100CA0000000000000000000000000000000000044
:100CB000000000000000000000522D444356472071
:100CC0004F66662C204C2D44435647204F66662CB9
:100CD0002043495053204F66662C20522D444356E2
:100CE00047204F6E2C204C2D44435647204F6E2CEE
:100CF0002043495053204F6E2C200000000000007C
:100D000000000000000000000000000000000000E3
:100D100000000000000000000000522D4443564730
:100D2000204F6E2C204C2D44435647204F6E2C20D4
:100D3000522D44435647204F66662C204C2D444389
:100D40005647204F66662C2000000000000000007F
:100D50000000000000000000000000000000000093
:100D60000000000000000000000000000000000083
:100D70000000000000000000000000522D44435617
:100D800047204F66662C204C2D44435647204F6623
:100D9000662C20522D44435647204F6E2C204C2D5C
:100DA00044435647204F6E2C2000000000000000F6
:100DB0000000000000000000000000000000000033
:100DC0000000000000000000000000000000000023
:100DD000000000000000000000000000522D44430D
:100DE0005647204F6E2C2043495053204F6E2C20E5
:100DF000522D44435647204F66662C20434950539A
:100E0000204F66662C20000000000000000000005B
:100E100000000000000000000000000000000000D2
:100E200000000000000000000000000000000000C2
:100E300000000000000000000000000000522D44EF
:100E4000435647204F66662C2043495053204F6637
:100E5000662C20522D44435647204F6E2C20434988
:100E60005053204F6E2C20000000000000000000B6
:100E70000000000000000000000000000000000072
:100E80000000000000000000000000000000000062
:100E90000000000000000000000000000000522DD3
:100EA00044435647204F6E2C20522D444356472032
:100EB0004F66662C200000000000000000000000CB
:100EC0000000000000000000000000000000000022
:100ED0000000000000000000000000000000000012
:100EE0000000000000000000000000000000000002
:100EF00000000000000000000000000000000052A0
:100F00002D44435647204F66662C20522D444356AD
:100F100047204F6E2C200000000000000000000061
:100F200000000000000000000000000000000000C1
:100F300000000000000000000000000000000000B1
:100F400000000000000000000000000000000000A1
:100F50000000000000000000000000000000000091
:100F600043495053204F6E2C2043495053204F6625
:100F7000662C2000000000000000000000000000BF
:100F80000000000000000000000000000000000061
:100F90000000000000000000000000000000000051
:100FA0000000000000000000000000000000000041
:100FB0000000000000000000000000000000000031
:100FC0000043495053204F66662C2043495053201C
:100FD0004F6E2C2000000000000000000000000008
:100FE0000000000000000000000000000000000001
:100FF00000000000000000000000000000000000F1
:1010000000000000000000000000000000000000E0
:1010100000000000000000000000000000000000D0
:10102000000044656C61792054696D653B00466938
:101030006C65204E616D653A2000436861696E61A0
:1010400067652C2000004C6F63616C54696D652CE2
:10105000204C6F63616C444D592C204C61742D44BD
:1010600065672C204C61742D4D696E2C204C617489
:101070002D5365632C204E532C204C6F6E2D4465F0
:10108000672C204C6F6E2D4D696E2C204C6F6E2D91
:101090005365632C2045572C20466978537461743E
:1010A0002C204E756D5361742C2050444F502C20D1
:1010B000416C745F4D2C2043686B2C20436F6D6D29
:1010C000000000484558434F524445522043414C8C
:1010D0004942482E5458540000007777772E6361B8
:1010E00074682D746563682E636F6D0000000000E6
:1010F000004C494D49544544203930352D38353759
:101100002D31303530000000434154484F444943AD
:1011100020544543484E4F4C4F47590000007B70C8
:101120002C30302C662C007B702C30302C657D00F0
:101130007B702C30302C6F7D00456E7465722053AF
:10114000434F504520766F6C7461676520696E204F
:101150006D5620284E4E4E4E4E2900456E746572D7
:10116000204349505320766F6C7461676520696E27
:10117000206D562A313020284E4E4E4E4E290045C5
:101180006E746572204443564720766F6C746167B5
:101190006520696E206D562A313020284E4E4E4E05
:1011A0004E2900D911D211CE11CA11C611C211B3E4
:1011B00011B311432D53474E44205B352D34305627
:1011C0005D00432D4200432D4600432D5200432D28
:1011D0004C00522D53474E4400432D53474E44007C
:1011E00020616E6420656E74657220766F6C746128
:1011F000676520696E206D562A313020284E4E4E8C
:101200004E4E2900506C6561736520636F6E6E658C
:10121000637420004572726F722C206D697373695C
:101220006E6720414443206E756D2028302D37298C
:10123000000A0D5363616C696E6743616C696220DB
:101240004F66667365743A20004572726F722C2087
:10125000656E74657220766F6C7461676520696E67
:10126000206D562A313020284E4E4E4E4E29001DFC
:1012700013FE12E812DC12B812A5127D1243535B62
:10128000302F312F322F332F345D5B7676767676A2
:101290005D202D204443205363616C696E672043B9
:1012A000616C6962004342202D2042617474657252
:1012B000792043616C696200435A5B302F312F32D1
:1012C0002F332F345D202D204443205A65726F4FF9
:1012D00066667365742043616C69620056202D2038
:1012E000566E756D626572004C5B696E785D5B4F22
:1012F0004E2F4F46465D202D204C65647300416E95
:101300006E202D2052656164204144433120666F78
:1013100072206E6E207365636F6E64730041202DC2
:1013200020526561642041444331004552524F527E
:10133000004F4B0043415448205445434820484502
:1013400058434F52444552205630302E3734000116
:1013500000020003000400050006000A000C000F54
:101360000014001E003C007800B400F0002C01685E
:1013700001000000000A0002000100B80B0F270165
:101380000064006801100E010010271027102710BC
:1013900027102710270100010001000100F80101BA
:1013A00000010002000100F4010000000001000043
:1013B0000000000A00F1D8000001000100C8000090
:1013C00000640064006400640064006400000000C5
:1013D000000000000050FE000000000000000001BE
:1013E00000000000000100000000000A00000001F1
:1013F000000100020058020000FA00FA00FA00FAA8
:1014000000780078000000000000000100000001EA
:101410000001000000000001000100008000190030
:101420008000190080001900800019008000190058
:10143000800019008000190080001900000100FFE1
:1014400003771469145B145414244A42494E2C390E
:10145000342C3100244A5341564500244A41534319
:101460002C47504753412C3100244A4153432C47C9
:1014700050524D432C3100244A4153432C4750478E
:1014800047412C310024504D544B3636372A3335E2
:101490000024504D544B3331342C302C312C302C13
:1014A000312C312C302C302C302C302C302C302C5A
:1014B000302C302C302C302C302C302C302C302A4E
:1014C000323900756E6C6F67206C62616E64747285
:1014D00061636B7374617461006C6F67206C62612F
:1014E0006E64747261636B7374617461206F6E7487
:1014F000696D6520313000756E6C6F672070737296
:10150000706F7361006C6F6720707372706F7361BE
:10151000206F6E74696D6520313000646174756D83
:1015200020757365720020302E3020302E30203030
:101530002E3020302E300075736572646174756DC5
:101540002000646174756D20776773383400756EA0
:101550006C6F67206770616C6D006C6F67206770DF
:10156000616C6D206F6E74696D6520313000D71528
:10157000C815B915AA15A21589157C15245047520E
:101580004D432C2C2C39362C00245047524D432CE3
:10159000412C2C3130302C2C2C2C2C2C2C2C2C2C69
:1015A0002C00245047524D434500245047524D4F84
:1015B0002C5047524D542C3000245047524D4F2C44
:1015C0005047524D462C3100245047524D4F2C4726
:1015D000504753562C3000245047524D4F2C2C343A
:1015E00000381629161A160B16FC15ED15445A204C
:1015F0003D20000000000000000000004459203D94
:1016000020000000000000000000004458203D20A1
:1016100000000000000000000000466C6174203DE6
:101620002000000000000000004D616A6F72412040
:101630003D2000000000000053545052204441540B
:10164000554D2E54585400661759174C173F1732F2
:1016500017251718170B17FE16F116E416D716CA1A
:1016600016BD16B016A316961689167C166F16426E
:10167000415454202043616C203D200041432020F0
:10168000205343616C203D200041432020205A43D9
:10169000616C203D200041444337205653636C2049
:1016A0003D200041444337205A43616C203D2000D7
:1016B00041444336205653636C203D20004144434F
:1016C00036205A43616C203D20004144433520566A
:1016D00053636C203D200041444335205A43616CE4
:1016E000203D200041444334205653636C203D206C
:1016F0000041444334205A43616C203D2000414462
:101700004333205653636C203D2000414443332033
:101710005A43616C203D20004144433220565363BC
:101720006C203D200041444332205A43616C203DEF
:10173000200041444331205653636C203D2000413A
:10174000444331205A43616C203D200041444330E2
:10175000205653636C203D200041444330205A43BF
:10176000616C203D200046696C6520496E64657897
:10177000203D2000141AFE19E819D219BC19A61927
:1017800090197A1964194E19381922190C19F6187A
:10179000E018CA18B4189E18881872185C184618F1
:1017A00030181A180418EE17D817C217454E4400FF
:1017B0000000000000000000000000000000000029
:1017C00000004443564720446566656374205661B3
:1017D0006C203D20000000004443564720446566CD
:1017E00065637420456E203D2000000000005379A1
:1017F0006E632054797065203D20000000000000D9
:101800000000000053686F7720476F6F676C65209A
:101810004D6170203D200000000053686F77204725
:10182000505320436F6F7264203D20000000000081
:101830004C6F63616C47505354696D654F666673B6
:101840006574203D20004143204672657175656EC8
:101850006379203D200000000000000042726F6BA1
:10186000656E5769726520416C61726D203D200084
:1018700000004C6F7720506F7420416C61726D20B6
:101880003D20000000000000496E70757420496D15
:10189000706564616E6365203D2000000000444374
:1018A00056474D44656C4F4E203D2000000000001F
:1018B00000000000444356474D44656C4F464620A7
:1018C0003D20000000000000000043495053324D0D
:1018D00044656C4F4E203D200000000000000000D9
:1018E00043495053324D44656C4F4646203D2000DD
:1018F00000000000000043495053314D44656C4FD7
:101900004E203D20000000000000000043495053DD
:10191000314D44656C4F4646203D200000000000DC
:101920000000537461727457697468203D20000090
:1019300000000000000000004F666654696D6520DD
:101940005B6D7365635D203D200000000000546FF7
:1019500074616C4379636C65205B7365635D203DE6
:101960002000000054696D652056616C7565203D4E
:1019700020000000000000000000436861696E6103
:10198000676520446972656374696F6E203D20004D
:10199000537461727420436861696E616765203DAC
:1019A00020000000000044697374616E6365205676
:1019B000616C7565203D2000000000004D6561737D
:1019C0007572656D656E7420556E697473203D2067
:1019D000000053746F7261676520416374696F6EB4
:1019E000203D200000000000537572766579205478
:1019F000797065203D2000000000000000004F705D
:101A0000657261746F72204E616D65203D2000002B
:101A100000000000537572766579204E616D652077
:101A20003D20000000000000000011241FBECFEF89
:101A3000CDBFDFE5DEBF00E00CBF1DE2A0E0B0E2FD
:101A4000EAE5FBE502E00BBF02C007900D92AA3168
:101A5000B107D9F727E4AAE1BDE201C01D92A73F73
:101A6000B207E1F70E9483330D94AB2D0C94000074
:101A7000CF93DF93CDB7DEB72B97CDBFDEBFBE01CF
:101A80006F5F7F4F80E092E00F94A025AE01485F2A
:101A90005F4F68E080E092E00F94FC258A819B8193
:101AA0009F789B8395E09D83817E8A831C82BE0103
:101AB0006F5F7F4F80E092E00F94502581E0888730
:101AC00088E18987AE01485F5F4F68E080E092E07F
:101AD0000F94C32580E092E00F94B1232B96CDBFE5
:101AE000DEBFDF91CF9108959FB7F894E0E0F2E078
:101AF0008081806280839FBF0895009781F020914C
:101B0000060223FF0EC020913C0230913D02FC01F1
:101B10002083318388E08093060281E0089580E08D
:101B2000089580E00895CF92DF92EF92FF92CF93D5
:101B3000DF930097D1F061157105C9F0EB01FC014D
:101B4000A081B18128EE33E00F94E8286B017C017D
:101B500083E10E9417A99B01AC01C701B6010F9454
:101B600093282883398381E003C080E001C080E0AE
:101B7000DF91CF91FF90EF90DF90CF900895EEE747
:101B8000F2E310821182148215821282138216826D
:101B900017828BE00E943BA9672B682B692B19F4F5
:101BA0001092863203C081E080938632EEE7F2E342
:101BB000118612860895CF93DF93EC01892B09F4E7
:101BC00091C0862F90E0FC013197EA30F10508F0D2
:101BD00089C08827E250FF4F8F4F0D94D128809104
:101BE0008632811107C088819981809382329093D7
:101BF000833278C08A819B81809382329093833232
:101C000071C080918632811107C08A819B81809347
:101C100082329093833266C08E819F81809382321C
:101C2000909383325FC080918632811107C08C818E
:101C30009D81809382329093833254C08A859B85A4
:101C400080938232909383324DC08091863281118D
:101C50000BC088819981EEE7F2E3848395838A81C2
:101C60009B81868397833EC08C819D81EEE7F2E362
:101C7000848395838E819F818683978333C08091EF
:101C8000863281110BC08A819B81EEE7F2E3848367
:101C900095838C819D818683978324C0EEE7F2E350
:101CA00088859985848395838A859B858683978398
:101CB00019C08091863281110BC08C819D81EEE725
:101CC000F2E3848395838E819F81868397830AC004
:101CD000EEE7F2E38C859D85848395838E859F85D1
:101CE00086839783DF91CF910895EEE7F2E38481B5
:101CF00095818083918386819781828393830895E0
:101D0000EEE7F2E381E0818712860895EEE7F2E3E1
:101D100011861286089580918832089583E10E9489
:101D20003BA9672B682B692B19F0809187320895A6
:101D300080E00895CF92DF92EF92FF926B01072E21
:101D4000000CEE08FF08C216D306E406F5067CF484
:101D500086179707E4F0092E000CAA0BBB0BE1E0F5
:101D6000281739074A075B07ACF4E0E013C06C01A1
:101D7000092E000CEE08FF08C216D306E406F5068D
:101D800044F0E1E0681779072CF4E0E003C0E0E0FC
:101D900001C0E0E08E2FFF90EF90DF90CF9008958C
:101DA000FF920F931F93CF93DF93CEE7D2E302E826
:101DB00012E3F12CE991F991309719F1AF010F2E4F
:101DC000000C660B770BDB01CA0177231CF401962C
:101DD000A11DB11DB595A795979587959A01AB0162
:101DE000280F391F4A1F5B1FBF01FF2314F46F5FC9
:101DF0007F4F759567958A819B819CDF813009F0C3
:101E0000F394C017D107B1F6FF2011F079DF01C0BC
:101E10007DDF6BDFDF91CF911F910F91FF900895D0
:101E2000EEE7F2E381E090E0A0E0B0E08787908BFE
:101E3000A18BB28B838B948BA58BB68B178A138661
:101E4000148615861686108E0895EEE7F2E381E07B
:101E5000878B108E0895EEE7F2E3178A108E0895AF
:101E600080919632089584E10E943BA9672B682BEC
:101E7000692B19F080919532089580E00895EEE77E
:101E8000F2E387859089A189B289838B948BA58B96
:101E9000B68B83859485A585B6858787908BA18B26
:101EA000B28B08956093893270938A3280938B321B
:101EB00090938C3208958F929F92AF92BF92CF925F
:101EC000DF92EF92FF92EEE7F2E3C388D488E588D1
:101ED000F68887859089A189B289C816D906EA064D
:101EE000FB0691F48090893290908A32A0908B32D8
:101EF000B0908C32C4DFC814D904EA04FB0411F496
:101F0000A4DF04C0A8DF02C0BADFFCCFFF90EF90CF
:101F1000DF90CF90BF90AF909F908F9008958BE10E
:101F20000E943BA9609397327093983280939932C4
:101F300090939A32ABE9B2E3EEE7F2E386E892E3FC
:101F40001D9211A212A232968E179F07C9F7EEE7D3
:101F5000F2E311A612A6089581E09091A7329111A3
:101F600001C080E008958AE10E943BA9672B682B9D
:101F7000692B39F081E09091A732911103C080E084
:101F8000089580E008950F931F938B019C01809129
:101F9000973290919832A0919932B0919A320097ED
:101FA000A105B10529F1880F991FAA1FBB1FAC011C
:101FB000BD01440F551F661F771F440F551F661F35
:101FC000771F840F951FA61FB71FB901A8013323E0
:101FD0003CF444275527BA01401B510B620B730B8D
:101FE00021E084179507A607B7071CF020E001C081
:101FF00020E0822F1F910F9108950F931F93CF938D
:10200000DF93009709F40BC1AEE7B2E35D961C9233
:102010005D975E961C925E975F961C925F97909676
:102020001C92462F50E0FA013297E930F10508F092
:10203000F6C0EC018827E85FFE4F8F4F0D94D12842
:1020400080918632811108C06C817D818E819F8153
:102050009ADF80939B32E3C0688179818A819B817A
:1020600092DF80939B32DBC080918632811108C061
:10207000688579858A859B8586DF80939B32CFC072
:10208000688179818A819B817EDF80939B32C7C082
:1020900080918632811111C0688579858A859B85FA
:1020A00072DF0EE712E3F801858F6C857D858E85E2
:1020B0009F8569DFF801868FB2C0688179818A8146
:1020C0009B8161DF0EE712E3F801858F6C817D81D2
:1020D0008E819F8158DFF801868FA1C08091863262
:1020E000811111C06C857D858E859F854CDF0EE743
:1020F00012E3F801858F688979898A899B8943DF92
:10210000F801868F8CC0688179818A819B813BDF51
:102110000EE712E3F801858F6C817D818E819F81AE
:1021200032DFF801868F7BC08091863281111FC01B
:10213000688979898A899B8926DF0EE712E3F8018D
:10214000858F6C897D898E899F891DDFF801868F37
:10215000688D798D8A8D9B8D16DFF801878F6C8D48
:102160007D8D8E8D9F8D0FDFF80180A358C0688113
:1021700079818A819B8107DF0EE712E3F801858F61
:102180006C817D818E819F81FEDEF801868F68855E
:1021900079858A859B85F7DEF801878F6C857D853B
:1021A0008E859F85F0DEF80180A339C0809186324C
:1021B000811111C0688979898A899B89E4DE0EE7DB
:1021C00012E3F801858F6C897D898E899F89DBDE1A
:1021D000F801868F24C0688179818A819B81D3DE52
:1021E0000EE712E3F801858F6C817D818E819F81DE
:1021F000CADEF801868F13C080918632811108C033
:102200006C857D858E859F85BEDE80939B3207C061
:10221000688179818A819B81B6DE80939B32DF91D0
:10222000CF911F910F910895843040F5EEE7F2E3CE
:1022300041A552A5242F30E0082E02C035952795E0
:102240000A94E2F720FF0AC0252F30E0082E02C0D2
:10225000359527950A94E2F720FD10C021E030E083
:10226000B90102C0660F771F8A95E2F7CB01EEE74E
:10227000F2E3462B41A78095852382A708958430F9
:1022800090F421E030E0A90102C0440F551F8A9567
:10229000E2F7CA018095EEE7F2E391A5982391A7B2
:1022A00092A5892382A70895BF92CF92DF92EF92E1
:1022B000FF920F931F93CF93DF930BE912E3CEE7C7
:1022C000D2E36E017801B12CF70181917F01F60113
:1022D00021A190E0820F911D22A1820F911D0397F1
:1022E00019F48B2DA1DF02C08B2DC9DFB394F2E06E
:1022F000CF0ED11C84E0B812E7CF26E832E389A1E3
:102300008AA3F80181918F0189A32296C217D3076E
:10231000B1F7DF91CF911F910F91FF90EF90DF9078
:10232000CF90BF900895843060F42091A73230E0C0
:10233000A90102C0559547958A95E2F7CA018170B7
:10234000089580E00895843060F42091A83230E050
:10235000A90102C0559547958A95E2F7CA01817097
:10236000089581E00895843000F5662379F0EEE762
:10237000F2E321E030E0A90102C0440F551F8A9525
:10238000E2F7CA0192A5892B82A70895EEE7F2E34E
:1023900021E030E0A90102C0440F551F8A95E2F701
:1023A000CA01809592A5892382A70895CF9383308F
:1023B00009F128F4813031F0823061F02CC088308E
:1023C00008F129C080919532882329F181E080931A
:1023D000963221C0C1DD8823F1F061E080E0C3DFE7
:1023E00061E081E0C0DF61E082E0BDDF61E083E0C9
:1023F000BADF11C080918732882369F081E0809331
:10240000883209C0CCEFC80F8C2F8DDF882319F0DC
:1024100061E08C2FA8DFCF910895009781F0FC0137
:10242000DC01AF5BBD4F80818C936083643021F40D
:1024300081E00C9426E4089580E00C9426E408954D
:10244000009719F0FC018081089580E00895CF93F2
:10245000DF93009709F48FC0EC0181E08883198233
:102460001A821B821C821D82DE01169682E1EEE634
:10247000F3E201900D928A95E1F7CE0148960E9411
:102480002DAF888D8F83898D88878A8D89878B8DE5
:102490008A8780E00E9417A9673E23E072078105C2
:1024A0009105CCF49F938F937F936F9383EE90E28B
:1024B0009F938F93CE01C4969F938F930F94D92AA5
:1024C0008CA9888B8DA9898B8EA98A8B8DB79EB795
:1024D00008968DBF9EBF1C8E1D8E18AA19AAFE01DC
:1024E000EC5CFD4F1082319610823196108231964D
:1024F00081E0808331961082118212821382349699
:1025000081E090E0A0E0B0E080839183A283B38378
:1025100034961082319688818083E751F24086E0BC
:10252000DF011D928A95E9F7E85EFD4F1082118266
:102530003296108211823296108211823296108267
:102540001182329610823196108232961082319624
:102550001082319610823196108231961082319617
:102560001082319610821182128213823496108268
:10257000C85ADD4F1882DF91CF910895009741F03E
:10258000613021F421E0FC0120AB0895FC0110AA88
:102590000895009741F0613021F421E0FC0121AB66
:1025A0000895FC0111AA08958F929F92AF92BF9255
:1025B000DF92EF92FF920F931F93CF93DF9341151A
:1025C000510509F46BC08A017B01C82F0E94E8AD58
:1025D000D82F8C2F0E9405AED82EDD2309F460C0C1
:1025E000882309F45FC08D2F0E9417A94B015C015D
:1025F0008D2D0E9417A9672B682B692B39F4F801E0
:10260000108211821282138280E04DC09701280D42
:10261000391D032E000C440B550BC63050F4A0E1BD
:10262000B7E20F94EE28F80160837183828393836D
:1026300009C0A8EEB3E00F94EE28F801608371831F
:10264000828393838D2D0E9417A99B01AC01F80111
:1026500060817181828193810F94B52888279927A1
:10266000DC01821B930BA40BB50BF80180839183D3
:10267000A283B3838C2F0E94A3B0F8018080918045
:10268000A280B380DC01CB01880D991DAA1DBB1D62
:1026900080839183A283B38381E005C080E003C07F
:1026A00080E001C080E0DF91CF911F910F91FF90FA
:1026B000EF90DF90BF90AF909F908F900895CF9351
:1026C000DF93009709F460C0EC010E945CEF813059
:1026D00091F58C830E9417E18823F9F0809190385E
:1026E000811119C089E0E9EEF0E2A1EDBDE30190AE
:1026F0000D928A95E1F7E1EDFDE301900020E9F705
:102700003197AF01415D5D4321E061ED7DE38BE0F9
:1027100093E30E94D0F60E9450E10E941AE18823C0
:1027200099F18FEB91E40E942BB60E9414E18A8309
:102730000E9461E129C01C820E9488EF8823F9F081
:1027400080919038811119C089E0E2EFF0E2A1EDAB
:10275000BDE301900D928A95E1F7E1EDFDE3019073
:102760000020E9F73197AF01415D5D4321E061ED64
:102770007DE38BE093E30E94D0F60E948BEF0E94F2
:1027800074EF81110E9477EFDF91CF9108950F933D
:102790001F93CF93DF93009709F463C0EC010E946D
:1027A000D3F1882381F18B8181115BC080919038B6
:1027B000811126C00E949CEF182F0E9414E11F92E5
:1027C0001F931F928F9384E091E29F938F9301ED6B
:1027D0001DE31F930F930F94D92AF8010190002055
:1027E000E9F73197AF01415D5D4320E0B8018BE02F
:1027F00093E30E94D0F68DB79EB708968DBF9EBF1B
:1028000081E08B832EC08B81813059F51B828091B2
:102810009038811126C00E949CEFC82F0E9414E1BD
:102820001F92CF931F928F938BEF90E29F938F9382
:10283000C1EDDDE3DF93CF930F94D92A09900020F7
:10284000E9F72197AE01415D5D4320E061ED7DE355
:102850008BE093E30E94D0F68DB79EB708968DBFAC
:102860009EBFDF91CF911F910F910895CF92DF927C
:10287000EF92FF920F931F93CF93DF93009709F48A
:10288000AAC06115710509F4A6C08B01EC010E9474
:10289000C9B5882309F49FC00E941BF06B017C011D
:1028A0000E94C0F186E10E943BA9AB01BC018AE60F
:1028B00096E30E945FB6D701C6010197A109B1094D
:1028C000883E9340A105B10508F03FC00E94CEA20A
:1028D000823088F18091903881112DC00E9414E1DE
:1028E0001F928F9380917F471F928F93FF92EF9259
:1028F000DF92CF9287E191E29F938F930F2EF1EDBC
:10290000EF2EFDE3FF2EF02DFF92EF920F94D92AC8
:10291000F70101900020E9F73197AF01415D5D4378
:1029200021E0B7018BE093E30E94D0F68DB79EB70C
:102930000C968DBF9EBF26ED3EE340EF50E46AE269
:1029400070E4C8010E94A8B843C0D701C601895EDF
:102950009340A109B10984369105A105B105C0F5DF
:1029600080EF9EE30E94C1B5811132C08091903802
:10297000811125C0FF92EF92DF92CF9283E291E224
:102980009F938F930F2EF1EDEF2EFDE3FF2EF02D91
:10299000FF92EF920F94D92AF70101900020E9F7F6
:1029A0003197AF01415D5D4321E0B7018BE093E3D7
:1029B0000E94D0F68DB79EB708968DBF9EBF26EDBC
:1029C0003EE340EF50E46AE270E4C8010E94A8B818
:1029D000CE010E94E2B5DF91CF911F910F91FF9040
:1029E000EF90DF90CF900895FC01892B39F011868C
:1029F00089E0DF011D928A95E9F7128608950F9309
:102A00001F93CF93DF93CCEAD2E304E013E3CE012C
:102A1000EBDF2B96C017D107D1F7DF91CF911F9134
:102A20000F910895FC01892B31F081E0928591305E
:102A300019F080E0089580E008951F93CF93DF930D
:102A4000CDB7DEB76097CDBFDEBF9C01FE013196EA
:102A5000AE014F5E5F4F21933193255F3F4FE417E7
:102A6000F507C9F7892BC1F010E010C0E12FF0E0A5
:102A7000EE0FFF1F81E090E08C0F9D1FE80FF91F04
:102A800080819181CFDF882341F01F5F0E94C0F2D7
:102A9000181760F381E001C080E06096CDBFDEBF13
:102AA000DF91CF911F910895CF92DF92EF92FF9225
:102AB0000F931F93CF93DF93CDB7DEB72597CDBF8D
:102AC000DEBF19821A821B821C824115510559F101
:102AD0006A017B01182FCA0187DFAE014F5F5F4F8C
:102AE000B701812F61DD8823C9F009811A812B810B
:102AF0003C814BE0BE016B5F7F4FC6010E94F0FD41
:102B0000F60101900020E9F73197EC19FD09D60193
:102B10001996EC93199781E01A968C9369817A81C2
:102B20008B819C8103C060E070E0CB012596CDBF16
:102B3000DEBFDF91CF911F910F91FF90EF90DF905B
:102B4000CF9008958F929F92AF92BF92EF92FF9293
:102B50000F931F93CF93DF930097A1F06115710539
:102B600089F0142F7B01EC010E9459E44B015C01B8
:102B7000113009F497D9950184014BE0B701CE01DA
:102B80000E9442FCDF91CF911F910F91FF90EF9037
:102B9000BF90AF909F908F900895AF92BF92CF92C9
:102BA000DF92EF92FF920F931F93CF93DF93CDB7F6
:102BB000DEB76097CDBFDEBF8C01CE0101967C01F0
:102BC0004096F70161937193655F7F4FE817F907AE
:102BD000C9F70115110509F46BC282E00E943BA9F7
:102BE000D62E96E0D91206C0C8010E943BEE811194
:102BF00065C239C38FEF8D0D823030F4C8010E9459
:102C00003BEE811107C02FC3C8010E943BEE882311
:102C100009F429C380E2E0EAF9E3DF011D928A9515
:102C2000E9F780E1E9E1F5E3DF011D928A95E9F733
:102C30008D2D90E0FC013197EA30F10508F03AC2A1
:102C40008827EF5EFE4F8F4F0D94D12858010F2E2D
:102C5000F0EACF2EF9E3DF2EF02D01E010E00EC1F7
:102C60000E9438EEC82E49815A81F8016081718135
:102C70001BDF0F2EF0EAEF2EF9E3FF2EF02DD70128
:102C80006D937D938D939C9313974B815C81F80199
:102C9000628173818C2D08DFD70114966D937D932B
:102CA0008D939C931797B2E0DB1206C28091A039F6
:102CB0009091A139A091A239B091A339809319358F
:102CC00090931A35A0931B35B0931C3581E0CBC28D
:102CD00058010F2EF0EACF2EF9E3DF2EF02D01E0A0
:102CE00010E00BC01F5F0F5FE2E0EE0EF11CF2E0A0
:102CF000AF0EB11C84E0C80ED11C112309F4FBC136
:102D0000123009F4EAC1D7014D915C91F50160815F
:102D1000718180E0C9DED6016D937D938D939C9384
:102D200013970430F8F28091A0399091A139A091C5
:102D3000A239B091A3398093193590931A35A09395
:102D40001B35B0931C3581E08EC258010F2EF0EA7E
:102D5000CF2EF9E3DF2EF02D01E010E00BC01F5F56
:102D60000F5FB2E0EB0EF11CE2E0AE0EB11CF4E03E
:102D7000CF0ED11C112309F4DBC1123009F4CAC1F2
:102D8000D7014D915C91F5016081718182E08CDE0B
:102D9000D6016D937D938D939C9313970430F8F235
:102DA000E9E1F5E3A0EAB9E34D915D916D917C9184
:102DB0001397408351836283738314968D919D9101
:102DC0000D90BC91A02D84839583A683B78381E069
:102DD0004AC258010F2EF0EACF2EF9E3DF2EF02D74
:102DE00001E010E00BC01F5F0F5FB2E0EB0EF11CC3
:102DF000E2E0AE0EB11CF4E0CF0ED11C112309F4B9
:102E0000B8C1133009F4A3C1113009F4A2C11430C0
:102E100009F4A1C1D7014D915C91F50160817181E7
:102E200080E042DED6016D937D938D939C93139742
:102E30000630C8F2E9E1F5E3A0EAB9E34D915D910E
:102E40006D917C91139740835183628373831496B1
:102E50008D919D910D90BC91A02D84839583A68327
:102E6000B78381E000C21F5F0F5FB2E0EB0EF11C81
:102E7000E2E0AE0EB11CF4E0CF0ED11C112309F438
:102E800099C1143009F484C1812F8B7F813009F4FA
:102E900081C1823009F480C1D7014D915C91F50167
:102EA0006081718185E000DED6016D937D938D9305
:102EB0009C9313970830B8F2E9E1F5E3A0EAB9E38F
:102EC0004D915D916D917C91139740835183628305
:102ED000738314964D915D916D917C911797448306
:102EE00055836683778318964D915D916D917C91A2
:102EF0001B9740875187628773871C968D919D91A0
:102F00000D90BC91A02D84879587A687B78781E017
:102F1000AAC158010F2EF0EACF2EF9E3DF2EF02DD3
:102F200001E010E00BC01F5F0F5FB2E0EB0EF11C81
:102F3000E2E0AE0EB11CF4E0CF0ED11C112309F477
:102F400058C1143009F445C1812F8B7F813009F4B9
:102F500042C1D7014D915C91F5016081718180E0A2
:102F6000A3DDD6016D937D938D939C9313970830C9
:102F7000D0F2E9E1F5E3A0EAB9E34D915D916D91FD
:102F80007C911397408351836283738314968D9150
:102F90009D910D90BC91A02D84839583A683B783CA
:102FA00081E061C1680100EA19E35E01B9E0AB0E9E
:102FB000B11CF701419151917F01D6016D917D9135
:102FC0006D0180E071DDF8016193719381939193BC
:102FD0008F01EA14FB0469F781E045C158010F2E07
:102FE000F0EACF2EF9E3DF2EF02D01E010E00BC068
:102FF0001F5F0F5FF2E0EF0EF11C82E0A80EB11C24
:1030000094E0C90ED11C112309F402C1133009F454
:103010000DC1D7014D915C91F5016081718180E016
:1030200043DDD6016D937D938D939C93139706306A
:10303000F8F28091A0399091A139A091A239B09174
:10304000A3398093193590931A35A0931B35B0930B
:103050001C3581E008C158010F2EF0EACF2EF9E3AC
:10306000DF2EF02D01E010E00BC01F5F0F5FB2E01C
:10307000EB0EF11CE2E0AE0EB11CF4E0CF0ED11C61
:10308000112309F4E2C0D7014D915C91F5016081F3
:10309000718181E0123009F480E006DDD6016D9384
:1030A0007D938D939C9313970430F8F281E0DBC0FD
:1030B00080E0D9C080E0D7C081E0D5C080E2E0EAFE
:1030C000F9E3DF011D928A95E9F780E1E9E1F5E393
:1030D000DF011D928A95E9F7B9CDF7014081518151
:1030E000D5016D917C9183E0DFDCF6016083718313
:1030F00082839383F7CDD7014D915C91F501608177
:10310000718183E0D1DCD6016D937D938D939C9387
:103110001397E8CDF70140815181D5016D917C91E4
:1031200083E0C2DCF601608371838283938317CED0
:10313000D7014D915C91F5016081718183E0B4DC30
:10314000D6016D937D938D939C93139708CE83E066
:1031500003C082E001C082E0F70140815181D501C6
:103160006D917C91A1DCF6016083718382839383EE
:103170003ACED7014D915C91F5016081718183E078
:1031800093DCD6016D937D938D939C9313972BCEF7
:1031900083E003C082E001C084E0F70140815181F7
:1031A000D5016D917C9180DCF6016083718382830F
:1031B000938359CED7014D915C91F5016081718166
:1031C00083E072DCD6016D937D938D939C9313976E
:1031D0004ACE83E001C082E0F70140815181D501F0
:1031E0006D917C9161DCF6016083718382839383AE
:1031F0009ACED7014D915C91F5016081718183E098
:1032000053DCD6016D937D938D939C9313978BCE56
:10321000F70140815181D5016D917C9183E044DCBF
:10322000F6016083718382839383E2CED7014D914F
:103230005C91F5016081718183E036DCD6016D938C
:103240007D938D939C931397D3CEF7014081518149
:10325000D5016D917C9180E027DCF601608371835C
:103260008283938302CF6096CDBFDEBFDF91CF9183
:103270001F910F91FF90EF90DF90CF90BF90AF9094
:1032800008950E9452EC882329F00E9463EC84E0A8
:10329000809327060895CF93DF93009799F1EC016F
:1032A00088818130A8F0833018F0863019F010C082
:1032B000E8DF25C08091280682FD03C084E080936A
:1032C00025060E94ECEB8823D1F00E94FDEB17C08D
:1032D0000E94ECEB882399F00E94FDEB84E0809340
:1032E00027060DC08D8181110DC00E9430EC88230E
:1032F00049F00E9441EC84E08093270603C0888156
:10330000863081F7DF91CF9108950E940FBC0E9413
:10331000A0F020E137E240E050E00F949328672BC3
:10332000682B692BE1F40E940FBC813019F40C94D6
:1033300023BB08950E940FBC823021F481E00C94DD
:1033400012BC08950E940FBC833019F40C9418BE6F
:1033500008950E940FBC843011F40C946CBE089543
:103360000F931F93CF93DF931F921F92CDB7DEB7BA
:1033700019821A820097B9F08C010E94524790E09E
:1033800006969E012F5F3F4F43E060E0800F911F44
:103390000E94A1FA882339F049815A8160E070E0E7
:1033A00080E00E9426A90F900F90DF91CF911F918E
:1033B0000F910895CF92DF92EF92FF920F931F9398
:1033C000CF93DF931F92CDB7DEB70097C9F18C0181
:1033D0007C0186E2E80EF11CBE016F5F7F4FC701E2
:1033E0000E9400C4882399F0F801C6A0D7A0E0A4E9
:1033F000F1A489E00E943BA9AB01BC0103E612E401
:1034000023E532E489810E94BBF081E01AC0BE014D
:103410006F5F7F4FC7010E9471CBF801C6A0D7A094
:10342000E0A4F1A489E00E9449A9AB01BC0103E634
:1034300012E423E532E489810E94BBF081E001C0FF
:1034400080E00F90DF91CF911F910F91FF90EF904F
:10345000DF90CF900895CF92DF92EF92FF920F937B
:103460001F93CF93DF931F92CDB7DEB7009779F10B
:103470008C01BE016F5F7F4F86960E948BCD8823A3
:1034800099F0F801C6A0D7A0E0A4F1A489E00E94B9
:103490003BA9AB01BC0103E612E423E532E48981D8
:1034A0000E94BBF081E014C0F801C6A0D7A0E0A440
:1034B000F1A489E00E9449A9AB01BC0103E612E432
:1034C00023E532E489810E94BBF081E001C080E005
:1034D0000F90DF91CF911F910F91FF90EF90DF90B0
:1034E000CF90089589E10E943BA9623059F482E0AF
:1034F0000E943BA9673041F0693031F0613021F022
:1035000081E0089580E0089580E0089589E10E94B7
:1035100049E5623059F482E00E9449E5673041F0A4
:10352000693031F0613021F081E0089580E0089544
:1035300080E008952F923F924F925F926F927F9218
:103540008F929F92AF92BF92CF92DF92EF92FF92B3
:103550000F931F93CF93DF93CDB7DEB76197CDBFA6
:10356000DEBFB82E8B017A0189E10E943BA9A62E0D
:103570000115110509F4D2C180919038882339F0E2
:103580000F2EFBE0CF2EF3E3DF2EF02D06C00F2E23
:10359000F2E1CF2EF4E3DF2EF02D82E08A1508F45D
:1035A000A12C8BE7F801808383E781838CE28283FF
:1035B000F2E3BF1207C082E38A0DF80183838CE235
:1035C00084830BC0F801B3828CE28483F0E3BF16DE
:1035D00009F455C182E3B8127CC18CEA92E3FE0182
:1035E00032969E012E5E3F4F819391930B962E173C
:1035F0003F07D1F788E08983E114F10469F086E0A0
:10360000F701D801159601900D928A95E1F70F2EDA
:10361000FBE0FF2EF02D04C00F2EF5E0FF2EF02D65
:10362000F801EF0DF11D8CE2808382E00E943BA93E
:10363000862F062E000C990B9F936F9380E291E2E8
:103640009F938F93F394C8018F0D911D9F938F9338
:103650000F94D92AF80101900020E9F73197E01B77
:10366000F10B7F01FF24F801EE0DFF1D118221E017
:10367000A701B801C6010E94D0F60F900F900F90DD
:103680000F900F900F9080919038811107C020E02B
:10369000A701B8018BE093E30E94D0F691E09A1560
:1036A00008F472C01982712C0F2EFCE26F2EF02DDF
:1036B0001801EFEF2E1A3E0A0F2EF0E9AF2EF8E3B5
:1036C000BF2EF02D5AC00E94C0F25980851509F412
:1036D000A7C0F8016082E52CF12CF701EE0FFF1F67
:1036E00081E090E08C0F9D1FE80FF91F8180928090
:1036F000F401418550E0B401C1010F94B32AF401F3
:1037000081856894442441F8480E8F5FF801E80FE2
:10371000F11D6082F7013196EE0FFF1F81E090E00E
:103720008C0F9D1FE80FF91F81809280F401418565
:1037300050E0B401C801840D911D0F94B32AF40127
:10374000E1844E0C539453945982E42CF12CF801EB
:10375000EE0DFF1D118221E0A701B801C6010E94F4
:10376000D0F6F5018081811107C020E0A701B801E2
:103770008BE093E30E94D0F673940E94C0F286958A
:10378000781608F4A0CF4CC01982612C0F2EFCE2F1
:103790005F2EF02D4801FFEF8F1A9F0A0F2EF0E9E0
:1037A000AF2EF8E3BF2EF02D36C00E94C0F2798014
:1037B0008715B1F1F8015082E72DF0E0EE0FFF1F01
:1037C00081E090E08C0F9D1FE80FF91FE180F280EF
:1037D000F701418550E0B701C4010F94B32AF70106
:1037E000E184E39473947982F12CF801EE0DFF1DCE
:1037F000118221E0A701B801C6010E94D0F6F501AF
:103800008081811107C020E0A701B8018BE093E31C
:103810000E94D0F663940E94C0F28695681628F242
:103820000F2EFCE2FF2EF02DF801F08284E00E94C2
:103830003BA9605DF8016183F28240E0BE016F5FE9
:103840007F4FC80103967ED9898193E0980FF801D4
:10385000E90FF11D9DE790838C5FE82EF12CF801B4
:10386000EE0DFF1D118221E0A701B801C6010E94E3
:10387000D0F680919038882309F445C04FC00F2EB0
:10388000F9E2EF2EF0E4FF2EF02DF701408150E039
:1038900062EF7FE3C80105960F94B32AF701808198
:1038A00095E0980FF801E90FF11D9DE790838A5F7D
:1038B000E82EF12CF801EE0DFF1D118221E0A70189
:1038C000B801C6010E94D0F680919038811126C0BF
:1038D00011C021E045E050E0B801C6010E94D0F6D9
:1038E0008091903881111AC0F0E3BF120FC045E0FB
:1038F00050E002C04E2D5F2D20E0B8018BE093E335
:103900000E94D0F60BC04E2D5F2D02C045E050E066
:1039100021E0B8018BE093E30E94D0F66196CDBF21
:10392000DEBFDF91CF911F910F91FF90EF90DF905D
:10393000CF90BF90AF909F908F907F906F905F904F
:103940004F903F902F900895CF93892B81F00E9444
:103950006046CAE00E9423470E945D46882321F00A
:103960000E947346811105C0C150A1F703C0C0E099
:1039700001C0C1E08C2FCF91089589E10E943BA93D
:10398000611104C00E942BE1882371F081E0409115
:103990008447509185476091864770918747452BB2
:1039A000462B472B09F080E008958F929F92AF92AB
:1039B000BF92CF92DF92EF92FF920F931F93CF931C
:1039C000DF930097A9F1EC0186E00E943BA94B012F
:1039D0005C0184E00E943BA9162F87E00E943BA96E
:1039E000062F812F0E943DE40E9459E46B017C0167
:1039F00086169706A806B906D9F0AB01BC0186E089
:103A00000E9493AA8823A1F00E94E6E3B701A601D1
:103A100086E00E9431A9B701A60186E00E945CE51C
:103A2000602F812F0E943DE468E0CE010E940D12BC
:103A3000DF91CF911F910F91FF90EF90DF90CF908A
:103A4000BF90AF909F908F90089582E10E943BA914
:103A500028E0E6EBF7E4DF01322F1D923A95E9F713
:103A6000EEEBF7E4DF011D922A95E9F721E030E063
:103A7000672B682B692B11F420E030E0F901E1534A
:103A8000FF4D80818560ECE7F7E482AF83AF81E092
:103A90000895009761F0613031F4FC01EC5CFD4F5A
:103AA00021E020830895FC01EC5CFD4F1082089515
:103AB0000097B1F0FC0180818430A1F40E94F3EF03
:103AC000823039F089E10E943BA9672B682B692B72
:103AD00059F00E94D0EF91E0811107C090E005C03D
:103AE00090E003C090E001C090E0892F08950F930B
:103AF0001F93CF93DF938C01EB01209709F442C011
:103B00001882892B19F189E10E943BA9F801808173
:103B10008130C0F0833018F08530D0F013C06111CF
:103B200006C02097B9F087E4888380E02EC06150FA
:103B3000623090F0209791F087E4888380E025C080
:103B4000209771F082E4888380E01FC080E01DC070
:103B500081E01BC080E019C081E017C080E015C083
:103B600080E013C081E011C080E00FC089E10E94B5
:103B70003BA9F8018081813018F3833080F28530D1
:103B800088F3DECF892B91F7EFCFDF91CF911F9193
:103B90000F910895009739F0FC01808181508430A5
:103BA00020F481E0089580E0089580E00895009772
:103BB00051F0FC018081813040F0843010F085307C
:103BC00021F481E0089580E0089580E00895CF9287
:103BD000DF92EF92FF92CF93DF93009709F45FC0DB
:103BE000EC0183E00E943BA96B017C01AB01BC01AD
:103BF00055276627772783E00E9493AA882309F434
:103C00004BC08C2DFE01EB5CFD4FC082813021F159
:103C1000823009F044C088E00E943BA9FE01E95CC3
:103C2000FD4F6083AB01BC0155276627772788E0ED
:103C30000E9493AA811105C081E0FE01E95CFD4F5D
:103C40008083FE01EA5CFD4F1082C85CDD4F188264
:103C500019821A821B8223C087E00E943BA9F62E9C
:103C600084E00E943BA9862F6F2D0E943DE485E0F1
:103C70000E943BA90E94EEE4FE01E45CFD4F6083DC
:103C80007183828393830E9406E4C85CDD4F1882AF
:103C900019821A821B8203C0CB5CDD4F1882DF9130
:103CA000CF91FF90EF90DF90CF900895009761F152
:103CB000FC01EA5CFD4F208131963081321710F013
:103CC00021111BC0FC01EA5CFD4F3150308332965C
:103CD0004081518162817381403821E5520721E0A2
:103CE0006207710598F44F5F5F4F6F4F7F4F4083BE
:103CF00051836283738381E00895FC01EA5CFD4F88
:103D00002150208380E0089580E0089580E00895A8
:103D10000F931F93CF93DF93009741F1EC010E9423
:103D20001DE4FE01E45CFD4F00811181228133819D
:103D30006017710782079307D8F00E9406E4FE011E
:103D4000E85CFD4F80819181A281B381803821E5BB
:103D5000920721E0A207B10568F40196A11DB11DEB
:103D600080839183A283B38381E005C080E003C098
:103D700080E001C080E0DF91CF911F910F91089505
:103D8000CF93DF93009709F43DC0FC01EC5CFD4F3D
:103D900020812223B9F1EC018BDE813021F4CC5C4F
:103DA000DD4F18822FC089E10E943BA961111AC022
:103DB0000E94F3EF813031F1823089F4DEDD882317
:103DC00009F10E94ADEFCC5CDD4F188280EF9EE3DD
:103DD0000E94BBB58FEB91E40E94E2B513C00E9434
:103DE000E1EF10C0CADD882369F00E94ADEFCC5C22
:103DF000DD4F188280EF9EE30E94BBB58FEB91E40C
:103E00000E94E2B5DF91CF910895FF920F931F9327
:103E1000CF93DF936115710509F47CC041155105FD
:103E200009F478C08A01EB01F82E82E10E9449E58D
:103E300021E0672B682B692B09F420E08F2D90E09F
:103E4000FC013197EA30F10508F05BC08827E55E98
:103E5000FE4F8F4F0D94D1281882E22FF0E0E153EE
:103E6000FF4D80818560F801808354C083E08883A2
:103E7000E22FF0E0E153FF4D8081F80180834AC0DA
:103E80001882E22FF0E0E153FF4D80818160F8015C
:103E9000808340C083E08883E22FF0E0E153FF4D50
:103EA0008081F801808336C01882E22FF0E0E15370
:103EB000FF4D80818160F80180832CC083E088837E
:103EC000E22FF0E0E153FF4D8081F801808322C0B2
:103ED000188285E0F80180831DC0188281E0F80116
:103EE000808318C01882E22FF0E0E153FF4D8081FB
:103EF0008160F80180830EC0188281E0F801808320
:103F000009C01882E22FF0E0E153FF4D8081856007
:103F1000F8018083DF91CF911F910F91FF90089559
:103F20008F929F92AF92BF92CF92DF92EF92FF92C9
:103F30000F931F93CF93DF93892B09F486C089E0F9
:103F40000E943BA99B01AC01A8EEB3E00F94EE28C0
:103F50006B017C010E9404F0C616D706E806F9063C
:103F600009F475C0C701B60128EE33E040E050E027
:103F70000F949328F22ED22F2E3108F06AC02130F0
:103F800009F469C00E9404F028EE33E040E050E0FC
:103F90000F949328822FF21638F46F2D0F94602817
:103FA000C92F992309F45CC00E949CEFE82E6D2F65
:103FB0000F946028D92F892F90E08E0D911DCA97FC
:103FC0000CF04BC08D2E912CA12CB12C0E941BF01B
:103FD000162F072FD82EC92EA8EEB3E0A501940105
:103FE0000F94EE284F2D0E9449F0C0919038C111D6
:103FF00036C00E941BF09F938F937F936F93CF9255
:10400000DF920F931F931F92DF931F92EF9285E32E
:1040100091E29F938F9301ED1DE31F930F930F94F4
:10402000D92AF80101900020E9F73197AF01415DED
:104030005D4321E0B8018BE093E30E94D0F68DB799
:104040009EB740968DBF9EBF0BC0C0E009C0C0E0C8
:1040500007C0C1E005C0C0E003C0C1E001C0C0E0CE
:104060008C2FDF91CF911F910F91FF90EF90DF90F8
:10407000CF90BF90AF909F908F900895EF92FF9256
:104080000F931F93CF93DF9320919038222339F021
:104090000F2EFBE0EF2EF3E3FF2EF02D06C00F2EC8
:1040A000F2E1EF2EF4E3FF2EF02D0097D1F1EC01B9
:1040B0008BE7888388E689838CE28A8392E69B83F8
:1040C0008C837F936F938DE691E29F938F93CE01C4
:1040D00005969F938F930F94D92AFE01019000209B
:1040E000E9F73197EC1BFD0B8F01112721E0A801A7
:1040F000BE01C7010E94D0F60E94CEA20F900F9081
:104100000F900F900F900F90873059F48091903856
:10411000811107C021E0A801BE018BE093E30E945A
:10412000D0F6DF91CF911F910F91FF90EF900895FE
:104130009F92AF92BF92CF92DF92EF92FF920F9336
:104140001F93CF93DF93009709F46CC020919038B0
:10415000222339F00F2EFBE0EF2EF3E3FF2EF02D9C
:1041600006C00F2EF2E1EF2EF4E3FF2EF02DEC014E
:104170008BE7888388E689838CE28A8393E79B8335
:104180008C830E947C8F982E00E416E3A0908F38D9
:10419000B0908C38F801C280D0800E942BE11F9231
:1041A0009F921F92AF921F92BF921F92CF921F9227
:1041B000DF921F928F93F80185811F928F938481E4
:1041C0001F928F9383811F928F9385E591E29F9336
:1041D0008F93CE0105969F938F930F94D92AFE015A
:1041E00001900020E9F73197EC1BFD0B8F0111279F
:1041F00021E0A801BE01C7010E94D0F68DB79EB78D
:1042000046968DBF9EBF8091903881110BC0A8014A
:1042100042505109BE016F5F7F4F21E08BE093E375
:104220000E94D0F6DF91CF911F910F91FF90EF90F8
:10423000DF90CF90BF90AF909F900895FF920F9323
:104240001F93CF93DF9300D01F92CDB7DEB70E94AC
:1042500074EC882349F00E9485EC0E94740D86E777
:104260009CE366DF80E057C0CE0101960E947D0D81
:10427000882309F450C01091A80600916806F090B8
:104280002806BE016D5F7F4FCE0101960E94930DFF
:10429000882309F43FC00E94DAA28823A1F180910B
:1042A0009038811130C0F0FAFF24F0F81F92FF928D
:1042B000029501701F920F9316FB112710F91F92A0
:1042C0001F938A818F9389818F938C818F938B81A8
:1042D0008F9381E791E29F938F9301ED1DE31F93ED
:1042E0000F930F94D92AF80101900020E9F7319734
:1042F000AF01415D5D4321E0B8018BE093E30E9493
:10430000D0F6CDBFDEBF6B817C8186E79CE3B6DE55
:1043100081E001C081E02496CDBFDEBFDF91CF9167
:104320001F910F91FF900895882321F081E08093E1
:104330008F38089510928F3808950F931F93CF935D
:10434000DF936115710571F0009761F0EB018C014D
:104350000E9496EC882331F00E94A7ECBE01C801B0
:104360000E944E7FDF91CF911F910F910895CF93BF
:10437000DF93009751F0EC010E94E2EC882329F0D2
:10438000CE010E9476810E94F3ECDF91CF910895D7
:10439000009791F0FC01EE5BFD4F2FEF3FE720838C
:1043A0003183329620E030E82083318332961082C8
:1043B000118232961082118208950F93CF93DF936A
:1043C0000097A1F0662371F0EA01FC01E65BFD4F66
:1043D00081E08083C9010E9412F2602FCE010E9409
:1043E0007F8F04C0FC01E65BFD4F1082DF91CF910F
:1043F0000F910895EF92FF920F931F93CF93DF9346
:104400001F921F92CDB7DEB7009709F458C061150F
:10441000710509F454C0FC0120A9211104C021A98F
:10442000222309F44CC08B017C01FC0110AA11AAC3
:104430000E94D00E0E945B0F0E945411F70142A906
:1044400053A9B7016C5C7F4F9E012F5F3F4FC8019E
:104450000F945D1FC8010F940B21F701E95AFD4F1E
:10446000D701AF5ABD4F8C918083319611968C91B4
:104470008083F70122A933A989819A8128173907F6
:1044800019F00E942C9002C00E94BC8FE2EBFCE36A
:10449000808190E0DC01AE54B34C25853685880FD1
:1044A000991FFC01EE54F34C418152811F960C91EF
:1044B00061E0C70182DF0E94C8830E9478F20F90FA
:1044C0000F90DF91CF911F910F91FF90EF90089582
:1044D0000F931F93CF93DF93009709F448C06115A2
:1044E000710509F444C08B01EC01FC01E65BFD4F52
:1044F00080818823C1F1DB018C91882341F10E94E6
:104500002EF28823A1F1F80160816150608361116E
:1045100008C00E94F18F0E94DE8FC65BDD4F1882BB
:1045200026C070E0F801E60FF71FD8011D962D9107
:104530003C911E97660F771FA60FB71F11964D91DE
:104540005C911297078561E0CE0137DF10C00E94B1
:104550002EF2882361F00E94F18F0E94DE8FC65BED
:10456000DD4F188204C00E94F18F0E94DE8FDF9120
:10457000CF911F910F9108958F929F92BF92CF92EA
:10458000DF92FF920F931F93CF93DF93009709F46D
:10459000DAC06115710509F4D6C020919038222344
:1045A00009F4C0C0CBE0D3E3BFC08B014C010E9433
:1045B000330FB82E0E94B30FD82E0E948E0EC82E35
:1045C0008D2D90E08B0D911D8C0D911D892B71F41B
:1045D000F401E55BFD4F8081813009F4B4C081E0D6
:1045E000808380E090E00E9445F2ADC0F401E55B7D
:1045F000FD4F8081823009F43EC0BB2051F00E9403
:10460000300F811108C061E0CE010E94A08301E05B
:1046100003C000E001C000E0CC2009F48AC00E9481
:104620008B0E811186C063E0CE010E94A08301E061
:1046300080C0DD2081F0812F0E949311882359F0E2
:10464000812F0E94A311811106C064E0610FCE0189
:104650000E94A08301E01F5F143059F7002309F482
:1046600072C0E401C55BDD4F82E0888384EF91E096
:104670000E9445F268C00E9461F2882309F463C079
:10468000BB2009F45DC00E94300F811159C00E9407
:104690004390CC2009F44FC0FF24F39401C0F12CC7
:1046A0000E948B0E811149C00E94439016C0D0E039
:1046B000C0E0DD2069F08D2F0E949311882341F026
:1046C0008D2F0E94A311811103C00E944190C1E06F
:1046D000DF5FD43071F7CC23E1F084EF91E00E94EA
:1046E00045F2D8018C9190E0F801E80FF91F1D9672
:1046F0002D913C911E97880F991FA80FB91F1196F5
:104700004D915C911297078561E080E496E355DE58
:104710001AC0F401E55BFD4F80818230A1F481E095
:10472000808311C0C2E1D4E3FC012081243059F41C
:104730003CCF10E07ECFFF24F394F110CECFB7CF63
:10474000C110ADCFB4CFDF91CF911F910F91FF90EA
:10475000DF90CF90BF909F908F900895009721F0A9
:10476000FC01E55BFD4F60830895CF93DF930097D5
:10477000C1F0EC01198218820E94861A813031F44E
:1047800082E0888389E1898391E006C0CE010E949E
:10479000BECE91E0811190E081E0992319F080E094
:1047A00001C080E0DF91CF910895CF93892B09F468
:1047B0004CC082E00E943BA9862F90E0FC0132971A
:1047C000E930F10508F043C08827EB5DFE4F8F4FBD
:1047D0000D94D12840E050E0BA0180E00E9475B00D
:1047E00037C040E050E0BA0180E00E9475B0C82FA9
:1047F00040E050E0BA0181E00E9475B0C80F81E04E
:10480000C23031F180E024C040E050E0BA0180E0E5
:104810000E9475B0C82F40E050E0BA0181E00E94CC
:1048200075B0C80F40E050E0BA0182E00E9475B058
:10483000C80F40E050E0BA0183E00E9475B0C80F95
:1048400081E0C43029F080E003C080E001C080E056
:10485000CF910895CF92DF92EF92FF92843098F437
:10486000E82FF0E0EE0FFF1FEE0FFF1FE75EFA4CA0
:10487000C080D180E280F3800E9445B06C197D0930
:104880008E099F0903C060E070E0CB01FF90EF90BC
:10489000DF90CF900895CF93892B09F453C082E025
:1048A0000E943BA9862F90E0FC013297E930F10588
:1048B00008F04AC08827E25DFE4F8F4F0D94D12843
:1048C00080E0C8DFAB01BC0180E00E9475B03DC054
:1048D00080E0C0DFAB01BC0180E00E9475B0C82F52
:1048E00081E0B8DFAB01BC0181E00E9475B0C80F68
:1048F00081E0C23051F180E028C080E0ABDFAB0145
:10490000BC0180E00E9475B0C82F81E0A3DFAB013D
:10491000BC0181E00E9475B0C80F82E09BDFAB0153
:10492000BC0182E00E9475B0C80F83E093DFAB0149
:10493000BC0183E00E9475B0C80F81E0C43029F04B
:1049400080E003C080E001C080E0CF910895853011
:10495000A1F118F4833041F0A8C0883009F47EC07A
:104960008A3009F453C0A1C0ECE7F7E4868D978D37
:10497000A0A1B1A1428D538D648D758D841B950BC3
:10498000A60BB70B86399105A105B10508F48FC0B8
:1049900046A157A160A571A582A193A1A4A1B5A12B
:1049A000481B590B6A0B7B0B81E0463951056105A9
:1049B000710508F483C080E00895ECE7F7E482A174
:1049C00093A1A4A1B5A1468D578D60A171A1841BAF
:1049D000950BA60BB70B86399105A105B10508F417
:1049E00068C046A557A560A971A982A593A5A4A5ED
:1049F000B5A5481B590B6A0B7B0B81E04639510565
:104A00006105710508F45AC080E00895ECE7F7E409
:104A100082A193A1A4A1B5A1468D578D60A171A1DA
:104A2000841B950BA60BB70B86399105A105B10523
:104A300008F441C042A953A964A975A986A597A500
:104A4000A0A9B1A9481B590B6A0B7B0B81E0463921
:104A500051056105710590F180E00895ECE7F7E4F8
:104A6000868D978DA0A1B1A1428D538D648D758DDA
:104A7000841B950BA60BB70B86399105A105B105D3
:104A8000E0F042A553A564A575A586A197A1A0A5B0
:104A9000B1A5481B590B6A0B7B0B81E046395105C8
:104AA0006105710558F080E0089580E0089581E087
:104AB000089581E0089581E0089581E00895CF93FD
:104AC00082E10E943BA9C1E0672B682B692B09F4A6
:104AD000C0E082E00E943BA988E0A6EBB7E4FD01BC
:104AE000982F11929A95E9F7AEEBB7E4FD01119278
:104AF0008A95E9F7862F90E0FC013197EA30F105BD
:104B000008F0EFC08827E95CFE4F8F4F0D94D12845
:104B1000EC2FF0E0E153FF4D80818560ECE7F7E496
:104B200082AF83AFE8C0EC2FF0E0E153FF4D80810E
:104B3000ECE7F7E482AF83AF83E08093BE478093D6
:104B4000BF47D9C083E003DFEC2FF0E0E153FF4D16
:104B5000908121E0811101C020E0822F892BECE7B8
:104B6000F7E482AF84AF83E08093BE478093C04771
:104B7000892F816083AF85AFBEC0EC2FF0E0E15399
:104B8000FF4D8081ECE7F7E482AF84AF93E0909330
:104B9000BE479093C04783AF85AF82E08093BF4705
:104BA0008093C147A8C085E0D2DEEC2FF0E0E1534E
:104BB000FF4D208191E0811101C090E0892F822B6F
:104BC000ECE7F7E482AF85AF93E09093BE47909314
:104BD000C14783AF86AF82E08093BF478093C247CF
:104BE000822F816084AF87AF86C0EC2FF0E0E15365
:104BF000FF4D8081ECE7F7E482AF86AF93E09093BE
:104C0000BE479093C24783AF87AF92E09093BF4770
:104C10009093C34784AF8093BC4794E09093C04780
:104C20009093C44785AF8093BD4785E08093C1478B
:104C30008093C54760C08AE08ADE91E0811101C09F
:104C400090E0892F8F70ECE7F7E482AF86AF93E0B6
:104C50009093BE479093C24783AF87AF82E0809323
:104C6000BF478093C34781E084AF8093BC4795AF33
:104C70009093BD4740C0ECE7F7E485E082AF84AF96
:104C800087E083AF85AF37C088E061DE91E08111B6
:104C900001C090E0EC2FF0E0E153FF4D8081892BC3
:104CA000ECE7F7E482AF85AF83E08093BE47809363
:104CB000C14791E093AF96AF84AF87AF1CC0EC2F94
:104CC000F0E0E153FF4D80818160ECE7F7E482AFD3
:104CD00084AF83AF85AF81E08093BF478093C147A6
:104CE0000AC0EC2FF0E0E153FF4D80818560ECE7D6
:104CF000F7E482AF83AF81E0CF9108951F93CF9304
:104D0000DF930097D9F1EC0118AA19AA0E94FF14A9
:104D100087E00E943BA9162F84E00E943BA9862FC2
:104D2000612F0E943DE489E10E943BA96130710539
:104D30008105910521F481E00E9432F003C080E0FA
:104D40000E9432F00E94721A813031F4CE010E942A
:104D50002B1A0E94251D04C0CE010E94DA19AFDE75
:104D60000E94C3F2CE010E94E71D0E944EF10E94F4
:104D7000BF0D0E94100F0E948F0F1982DF91CF91FB
:104D80001F910895CF93DF93009791F0FC0120814C
:104D9000243071F4EC010E94D51CCE01AFDF0E94DB
:104DA000BFEF10928B3863E0CE010E940D12198282
:104DB000DF91CF910895882321F081E0809390388E
:104DC0000895109290380895809190380895AF9288
:104DD000BF92CF92DF92EF92FF920F931F93CF93E8
:104DE000DF93DC01009709F45AC04115510509F41D
:104DF00058C02115310509F456C0FA01C081D0E030
:104E0000F901008110E06115710561F0FC017C0180
:104E1000E60EF71E9191C90FD11D0C0F1D1FEE1646
:104E2000FF06C1F7F9017B016D01DA01CC93008324
:104E3000F601E60FF71F8CE280838BE181835B0133
:104E4000A2E0AA0EB11CAC0CBD1C8C2F82958F70F9
:104E50000E9484FAF50180835701F3E0AF0EB11C84
:104E6000AC0CBD1C8C2F8F700E9484FAD5018C93E2
:104E7000E7012496CC0DDD1D802F82958F700E9456
:104E800084FA8883D7011596E601CA0FDB1F802FAD
:104E90008F700E9484FA8883C701069605C0CB01F3
:104EA00003C0CB0101C0CB01DF91CF911F910F91C6
:104EB000FF90EF90DF90CF90BF90AF9008957F92DA
:104EC0008F929F92AF92BF92CF92DF92EF92FF921A
:104ED0000F931F93CF93DF93CDB7DEB76197CDBF0D
:104EE000DEBF8C017B015A01722E89E10E943BA931
:104EF000962E0115110509F4D3C0E114F10409F44B
:104F0000D1C0A114B10409F4CFC0B701FE0132969B
:104F1000CE01429661937193655F7F4FE817F90761
:104F2000C9F78DE0D801D4968C93D49782E090E0B5
:104F3000D2968D939C93D3978AE0D5968C936801F3
:104F4000B6E3CB0ED11C41E0BE016F5F7F4FC601BF
:104F50000E94A2152981F80182A993A9820F911DAF
:104F60009C012F5F3F4F22AB33ABE80FF91F2CE2C0
:104F700024ABF1E0F91590F5F12C0F2EFCE2EF2EA9
:104F8000F02D61C0EF2DF0E0EE0FFF1F81E090E00B
:104F90008C0F9D1FE80FF91F81809280D801D29657
:104FA0008D919C91D397C496F401418550E0B40152
:104FB000800F911F0F94B32AD40119962C91F801F8
:104FC00082A993A9820F911D9C012F5F3F4F22ABB5
:104FD00033ABE80FF91FE4AAF39405C0F12C0F2EB0
:104FE000FCE2EF2EF02D0E94C0F2F81658F230C00D
:104FF000EF2DF0E0EE0FFF1F81E090E08C0F9D1F82
:10500000E80FF91F81809280D801D2968D919C91F2
:10501000D397C496F401418550E0B401800F911FED
:105020000F94B32AD40119962C91F80182A993A95F
:10503000820F911D9C012F5F3F4F22AB33ABE80FD6
:10504000F91FE4AAF3940E94C0F28695F81680F244
:10505000F1E07F121CC0D801D2968D919C91D3971C
:10506000C4967501BFEFEB0EF11CF701408150E0D3
:10507000B501800F911F0F94B32AD7012C91F8012D
:1050800082A993A9820F911D82AB93AB0FC0D80167
:10509000D296ED91FC91D397E00FF11F14AA06C0B0
:1050A00080E024C080E022C080E020C0A8014F5AE8
:1050B0005D4FF801E95AFD4F8081FA018083980124
:1050C0002E5A3D4F37968081D9018C93F80162A901
:1050D00073A962507109C6017ADE0296D801D29690
:1050E0008D939C93D39781E0D0968C936196CDBF9E
:1050F000DEBFDF91CF911F910F91FF90EF90DF9076
:10510000CF90BF90AF909F908F907F9008954F92D7
:105110005F926F927F928F929F92AF92BF92CF9247
:10512000DF92EF92FF921F93CF93DF93CDB7DEB75D
:105130006097CDBFDEBF009709F46DC061157105A2
:1051400009F469C09B01FE013196AE014F5E5F4FCD
:1051500021933193255F3F4FE417F507C9F77B0192
:105160006C0110E012C0E12FF0E0EE0FFF1F81E0B4
:1051700090E08C0F9D1FE80FF91F808191810E94A4
:105180001215882309F447C01F5F0E94C0F2181748
:1051900050F30E941BF04B015C010E9404F02B01B4
:1051A0003C0180EF9EE30E94C1B5182F81110BC016
:1051B0009EE1890E911CA11CB11C84149504A604C7
:1051C000B70448F115C040E050E066E77CE380E3B7
:1051D0000E949A1A212F40EF5EE3B701C6016FDEED
:1051E00042EF5FE366E77CE382E30E949A1A0DC018
:1051F00020E040EF5EE3B701C60161DE40E050E031
:1052000066E77CE382E30E949A1A80EF9EE30E94A5
:10521000BBB50E94FF146096CDBFDEBFDF91CF917A
:105220001F91FF90EF90DF90CF90BF90AF909F9035
:105230008F907F906F905F904F9008951F93CF93C2
:10524000DF93009709F4A0C0EC0198819230D1F06F
:1052500018F4913031F098C0943019F19830F1F091
:1052600093C08B81813009F08FC08C81813009F02F
:105270008BC00E94E1EFCE0141DD62E0CE010E94D1
:105280000D1282C080914B42813029F463E0CE013F
:105290000E940D1279C00E94851976C00E94C443F5
:1052A00073C0CE010E94C01E6CEA72E380E396E3F5
:1052B0000E94CD15813009F054C082E00E943BA9C4
:1052C000162F80E396E30E94DB0D612F80EA99E3BD
:1052D0000E94FD0F6CEA72E3CE0119DF48C00E9404
:1052E0002EE5882309F44DC00E945FF160EE79E35A
:1052F000CE0180D80E941DE544C08981811144C03F
:10530000CE010E94881E882339F00E945FF160EE72
:1053100079E3CE016FD838C018AA81E089AB34C0D8
:1053200088A9882389F1898181112EC0CE010E942C
:10533000561E882339F00E945FF160EE79E3CE01BA
:1053400059D822C018AA20C00E942EE58823E1F077
:105350000E945FF160EE79E3CE014CD80E941DE51A
:1053600013C08CEA92E30E941D158111B3CFFE0198
:10537000EB5CFD4F8081813009F4B1CF823021F7A1
:10538000CFCF88A98111B9CFDF91CF911F91089517
:10539000009789F06115710571F04115510559F0BB
:1053A0002115310541F0FC011082FB011082FA0148
:1053B0001082F901108208952F923F924F925F92CE
:1053C0006F927F928F929F92AF92BF92CF92DF9215
:1053D000EF92FF920F931F93CF93DF93CDB7DEB77A
:1053E0002597CDBFDEBF009709F461C04115510577
:1053F00009F45FC02115310509F45DC0613BE4E0AB
:105400007E0708F45AC02B01E0EB4E1AE4E05E0A76
:10541000612C712CE2E04E165104610471040CF40D
:1054200054C02C833D831A018C01C12CD12C7601F0
:10543000C3944B01A12CB12CB501A4014C195D09F9
:105440006E097F09C8010F945D219E012F5F3F4FB8
:1054500041E050E0BE016D5F7F4FC8010F94111E07
:1054600081112DC08B818B3191F18FEFC81AD80A31
:10547000E80AF80AC414D504E604F704ECF225C0DF
:1054800089819A810497E8F0B10181ED9DE30E9442
:1054900076FE982F882341F16C817D8183ED9DE319
:1054A0000E9476FE91E081111FC090E01DC090E047
:1054B0001BC090E019C090E017C090E015C090E0CC
:1054C00013C090E011C090E00FC090E00DC09E01AD
:1054D0002F5F3F4F44E050E061ED7DE3C8010F9442
:1054E000111E882369F2EFCF892F2596CDBFDEBF2D
:1054F000DF91CF911F910F91FF90EF90DF90CF90B0
:10550000BF90AF909F908F907F906F905F904F90E3
:105510003F902F9008950097A9F061157105B1F0A3
:10552000FC019C01260F371F60E070E0CB01419128
:105530004D3021F46F5F7F4F8F4F9F4F2E173F07E6
:10554000B1F7089560E070E0CB01089560E070E08D
:10555000CB0108952F923F924F925F926F927F926C
:105560008F929F92AF92BF92CF92DF92EF92FF9273
:105570000F931F93CF93DF9300D01F92CDB7DEB769
:10558000009709F455C00115110509F453C0613B9A
:105590007440C0F4F801108211821282138280E0FC
:1055A0004CC009811A81B801C101B5DF460E571EF2
:1055B000681E791E0815190500F1C00ED11EE11CE8
:1055C000F11C0BC00B831C8349011A015C01C12C27
:1055D000D12C7601412C512C3201B701A601C50115
:1055E0000F945D219E012F5F3F4FA401B101C501C2
:1055F0000F94111E8823A9F21FC0F6E24F16510422
:105600006104710440F4EB81FC81108211821282EA
:10561000138281E012C0F5E24F1A51086108710847
:10562000EB81FC81408251826282738281E005C0FD
:1056300080E003C080E001C080E02496CDBFDEBFE3
:10564000DF91CF911F910F91FF90EF90DF90CF905E
:10565000BF90AF909F908F907F906F905F904F9092
:105660003F902F900895009741F0FC01ED5AFD4FB7
:105670006081718182819381089560E070E0CB0147
:105680000895009739F0FC01ED5AFD4F1082118208
:10569000128213820895CF93DF93009781F12091B6
:1056A000903821112CC0EC010E9470ED882339F153
:1056B000CE010E9404880E9455ED0E9414E11F92C1
:1056C0008F9380E991E29F938F93C1EDDDE3DF93A8
:1056D000CF930F94D92A09900020E9F72197AE01C2
:1056E000415D5D4320E061ED7DE38BE093E30E944B
:1056F000D0F60F900F900F900F900F900F90DF91BA
:10570000CF910895EF92FF920F931F93CF93DF9362
:10571000CDB7DEB72797CDBFDEBF7C01FB0184810B
:105720008D8385818E8386818F8380819181A28103
:10573000B38189839A83AB83BC83870180EAE816AF
:1057400088E0F80629F460E183E00F94830814C030
:1057500080EBE81688E0F80629F460E283E00F9415
:10576000830813C080EAE81689E0F80629F460E1AE
:1057700084E00F94830812C0003B89E0180729F4E5
:1057800060E284E00F94830812C0003A8AE01807B0
:1057900029F460E185E00F94830810C0003B8AE0A3
:1057A000180729F460E285E00F94830807C0003AE7
:1057B0001B4021F460E186E00F948308BE016F5F17
:1057C0007F4FC7010E9473612796CDBFDEBFDF9177
:1057D000CF911F910F91FF90EF900895DC01892BDD
:1057E000E1F0E62FE695E695E69580E2E89FF00188
:1057F0001124FA5F8085677021E030E002C0220F3B
:10580000331F6A95E2F7282381E009F480E08C9346
:1058100011968C93119712961C920895CF93DF9353
:10582000009709F4A1C06D3209F0A0C03091A8061C
:1058300021E0432F407235FF20E0FC0120833181BD
:10584000231709F495C0EC01442309F468C0311111
:1058500066C00E9404ED0097F1F4B6DA811119C018
:1058600086E0EBEAF1E2A1EDBDE301900D928A95AD
:10587000E1F7E1EDFDE301900020E9F73197AF0199
:10588000415D5D4321E061ED7DE38BE093E30E94A8
:10589000D0F61A8265C0803D974000F595DA8111F7
:1058A00019C086E0E1EBF1E2A1EDBDE301900D92BC
:1058B0008A95E1F7E1EDFDE301900020E9F73197EA
:1058C000AF01415D5D4321E061ED7DE38BE093E35A
:1058D0000E94D0F60E9418ED1A8242C081E08A83AD
:1058E0000E9418ED71DA81113BC086E0E7EBF1E22E
:1058F000A1EDBDE301900D928A95E1F7E1EDFDE3A5
:1059000001900020E9F73197AF01415D5D4321E04F
:1059100061ED7DE38BE093E30E94D0F621C01A8213
:1059200081E090E00E942BED4FDA811119C086E0F2
:10593000EDEBF1E2A1EDBDE301900D928A95E1F767
:10594000E1EDFDE301900020E9F73197AF01415D02
:105950005D4321E061ED7DE38BE093E30E94D0F6AF
:10596000888189838A8105C080E003C080E001C00E
:1059700080E0DF91CF9108958FEB91E40C949ABF72
:10598000089522DA811117C063E57EE38BE093E38B
:105990000E947CF68091D53E813029F543E55EE397
:1059A00065E57EE38BE093E30E94C6A683E59EE374
:1059B0000C946DF6089563E57EE38BE093E30E941B
:1059C000F38C8091D53E813071F420E436E343E5D9
:1059D0005EE365E57EE38BE093E30E94E48C83E580
:1059E0009EE30C946DF608950E940983882329F0A4
:1059F00081E59BE30C94B7210895E6D981112DC070
:105A00006FE67BE382E194E30E94F38C8091F13BAB
:105A1000813019F5D9D9811112C062E480910B331C
:105A200090910C330E94586040916F3B5091703BB5
:105A300021E061E77BE38BE093E30E94D0F620E472
:105A400036E34FE65BE361E77BE382E194E30E94A8
:105A5000E48C8FE69BE30C946DF60895EF92FF9231
:105A60000F931F93CF93DF93AFD9882319F0CBE027
:105A7000D3E302C0C2E1D4E380E69BE30E94FA8E46
:105A8000882331F060E67BE3CE010E949D210EC2A7
:105A900080916E3B813009F02EC10E947C8F88235B
:105AA00009F404C26BE17AE389E998E30E94818EEC
:105AB00080914C3B813009F0F9C18091203A8F7D73
:105AC0008C3409F0C0C0E0901B3AF0901C3A7CD9AD
:105AD000811157C087E0E3ECF1E2A1EDBDE3019055
:105AE0000D928A95E1F7E1EDFDE301900020E9F7E1
:105AF0003197AF01415D5D4320E061ED7DE38BE0D7
:105B000093E30E94D0F610921D3A10921E3AE114CF
:105B1000F104A9F080E090E00BE11AE3FC01E55EFE
:105B2000F54C65818BE093E30E945CF7F80182817C
:105B300093810196828393838E159F0578F30E944B
:105B400071F11F928F938AEC91E29F938F9301EDF5
:105B50001DE31F930F930F94D92AF80101900020A1
:105B6000E9F73197AF01415D5D4321E0B8018BE07A
:105B700093E30E94D0F60F900F900F900F900F902C
:105B80000F900E9471F1882371F181E00E94917E53
:105B9000813069F48BE19AE30E94C78E8BE19AE32E
:105BA0000E94D98E0E944EF10E94CB8F02C00E94AB
:105BB0002C90E2EBFCE3808190E0DC01AE54B34C2E
:105BC00025853685880F991FFC01EE54F34C4181E1
:105BD00052811F960C9161E080E496E30E94DD21E2
:105BE0000E9478F281C0E0924F3BF092503B0E94BD
:105BF00071F1682FCE010E945581E6D8811174C0E1
:105C00000E9471F11F928F9380ED91E29F938F9389
:105C1000C1EDDDE3DF93CF930F94D92A09900020E3
:105C2000E9F72197AE01415D5D4321E061ED7DE340
:105C30008BE093E30E94D0F60F900F900F900F909F
:105C40000F900F9051C0C0D881114AC08AE0E4EE95
:105C5000F1E2A1EDBDE301900D928A95E1F7E1ED4E
:105C6000FDE301900020E9F73197AF01415D5D430D
:105C700020E061ED7DE38BE093E30E94D0F6EBE161
:105C8000FAE31282138280819181892BA9F080E04E
:105C900090E0EF01FC01E55EF54C65818BE093E35C
:105CA0000E945CF78A819B8101968A839B8328816D
:105CB00039818217930770F3E1EDFDE380E290E014
:105CC0008083918301900020E9F73197AF01415D16
:105CD0005D4321E061ED7DE38BE093E30E94D0F62C
:105CE0008BE19AE30E94D98E8BE19AE30E94C78EE2
:105CF0000E944EF1DBC06BE17AE389E998E30E94F0
:105D00001A8E80914C3B813009F0D0C08BE19AE330
:105D10000E944A8F882321F0E0904E3BF12C04C072
:105D2000E0901B3AF0901C3A4FD8811157C087E0A1
:105D3000E3ECF1E2A1EDBDE301900D928A95E1F76C
:105D4000E1EDFDE301900020E9F73197AF01415DFE
:105D50005D4320E061ED7DE38BE093E30E94D0F6AC
:105D600010921D3A10921E3AE114F104A9F080E05D
:105D700090E00BE11AE3FC01E55EF54C65818BE0F8
:105D800093E30E945CF7F8018281938101968283FC
:105D900093838E159F0578F30E9471F11F928F9364
:105DA0008AEC91E29F938F9301ED1DE31F930F9374
:105DB0000F94D92AF80101900020E9F73197AF013B
:105DC000415D5D4321E0B8018BE093E30E94D0F692
:105DD0000F900F900F900F900F900F900E9471F105
:105DE000882371F181E00E94917E813069F48BE11A
:105DF0009AE30E94C78E8BE19AE30E94D98E0E949B
:105E00004EF10E94CB8F02C00E942C90E2EBFCE38B
:105E1000808190E0DC01AE54B34C25853685880F37
:105E2000991FFC01EE54F34C418152811F960C9155
:105E300061E080E496E30E94DD210E9478F230C0A8
:105E4000E0924F3BF092503B0E9471F1682FCE01DF
:105E50000E9455810E94E426811122C00E9471F1A6
:105E60001F928F9380ED91E29F938F93C1EDDDE3BD
:105E7000DF93CF930F94D92A09900020E9F7219757
:105E8000AE01415D5D4321E061ED7DE38BE093E395
:105E90000E94D0F60F900F900F900F900F900F90E0
:105EA0008BE19AE30E94C78E0E944EF1DF91CF9161
:105EB0001F910F91FF90EF9008958F929F92AF9254
:105EC000BF92CF92DF92EF920F931F93CF93DF9306
:105ED000EC0180E00E9417A94B015C01209709F4B6
:105EE00056C11D8EFE01E25BFD4F1082CE010E9465
:105EF000A41C882309F44BC16E0184E3C80ED11C95
:105F0000BE01635E7F4FC6010E9457DA8C8F8111FC
:105F10001FC00E94E426811119C08BE1EEEEF1E270
:105F2000A1EDBDE301900D928A95E1F7E1EDFDE36E
:105F300001900020E9F73197AF01415D5D4321E019
:105F400061ED7DE38BE093E30E94D0F681E08D8FDD
:105F50006DE770E4C6010E9420DFFE01E35BFD4FA8
:105F600080838DE790E40E94B1AF8823A1F181E0A6
:105F7000FE01E25BFD4F80838DE790E40E944EAF0F
:105F80000E94E426811127C0FE01E25BFD4F808163
:105F90001F928F93319780811F928F9389E092E2B5
:105FA0009F938F9301ED1DE31F930F930F94D92AB5
:105FB000F80101900020E9F73197AF01415D5D43A1
:105FC00021E0B8018BE093E30E94D0F6ADB7BEB7F5
:105FD0001896ADBFBEBF8D8D813039F0FE01E25BFA
:105FE000FD4F8081813009F05AC00E94E426811162
:105FF00019C08CE1ECE1F2E2A1EDBDE301900D925C
:106000008A95E1F7E1EDFDE301900020E9F7319792
:10601000AF01415D5D4321E061ED7DE38BE093E302
:106020000E94D0F66894EE24E2F808E312E2A5019B
:106030009401BE01685E7F4FCE0106960E943C4AE5
:106040008D8340E050E0BA01CE011BDB8D818823B7
:1060500009F49DC082E00E943BA9062F8BE00E94BC
:106060003BA921E0611120E0BE016E5C7F4F40EE54
:1060700059E3C6010E944F45CE010E94B0199E010E
:10608000285A3D4FAE01495A5D4FBE016E5A7D4FB1
:10609000CE018F5A9D4F7CD90E9406E678C08E01B2
:1060A0000A5F1F4FB80180EE99E30E9414498D8367
:1060B000811137C0A5019401BE01685E7F4FC80100
:1060C0000E9476468D8340E050E0BA01CE01D9DAD5
:1060D0008D81882309F45BC082E00E943BA9062FD2
:1060E0008BE00E943BA921E0611120E0BE016E5CC3
:1060F0007F4F40EE59E3C6010E944F45CE010E94FA
:10610000B0199E01285A3D4FAE01495A5D4FBE015C
:106110006E5A7D4FCE018F5A9D4F3AD90E9406E6A6
:1061200036C08E010D5A1D4F0F2EF0EEAF2EF9E343
:10613000BF2EF02DF5016285738520E032E0A601C7
:10614000C50108DA015011096E01FFEACF1AFDEF0F
:10615000DF0AD5011A966D917C911B979801A601D3
:10616000C5012AD9FE01E95AFD4FD6018C918083E1
:10617000C85ADD4FF80180818883D5011A964D9168
:106180005D916D917C911D97C5010F945D21DF910B
:10619000CF911F910F91EF90DF90CF90BF90AF9074
:1061A0009F908F9008956DE289EA92E337DB882310
:1061B00009F467C080911A2D882309F446C00E9413
:1061C000EA5384E0809326060E9441EC8DE790E438
:1061D0000E944BBE80E496E370DE80918E38882367
:1061E000F1F00E940FBC813019F0823069F017C0C5
:1061F00080918D38882329F08DE790E40E94ADBB13
:106200000EC00E9480BB0BC080918D38882329F07E
:106210008DE790E40E942FBD02C00E94FABC10924C
:106220001A2D0E9478F280E496E30E94901F81115B
:106230000E94E1EF80E496E30E947E26609181381F
:1062400080E496E30E940D121CC00E9478F20E9426
:10625000BFEF66E080E496E30E940D1261E086E401
:1062600096E30E94E2480E9461460E9445FF0E9418
:10627000C05381E080931A2D84E0809325060E940C
:1062800041EC80911A2D882331F00E943E528111F9
:10629000FCCF80911A2D08954F925F926F927F925A
:1062A0008F929F92AF92BF92CF92DF92EF92FF9226
:1062B0001F93CF93DF93CDB7DEB72797CDBFDEBF58
:1062C0007C0110924C4210E00F2E812CFBE49F2E9B
:1062D000A12CB12CF02D0F2EF1EDCF2EFDE3DF2EF2
:1062E000F02D0F2EF0E84F2EF5E25F2E612C712C71
:1062F000F02D111120C080E096E9A0E0B0E0F70198
:1063000080839183A283B3838AE0EDE3F2E2D60136
:1063100001900D928A95E1F7F60101900020E9F7CE
:106320003197AF01415D5D4321E0B6018BE093E31E
:106330000E94D0F65CC0113001F580EC92E1A0E043
:10634000B0E0F70180839183A283B38389E0E7E41F
:10635000F2E2D60101900D928A95E1F7F6010190E3
:106360000020E9F73197AF01415D5D4321E0B601BF
:106370008BE093E30E94D0F63AC01230E9F4D701E3
:106380004D925D926D927C92139789E0E0E5F2E286
:10639000D60101900D928A95E1F7F6010190002057
:1063A000E9F73197AF01415D5D4321E0B6018BE034
:1063B00093E30E94D0F61BC0F70180829182A282F3
:1063C000B38289E0E9E5F2E2D60101900D928A9567
:1063D000E1F7F60101900020E9F73197AF01415D47
:1063E0005D4321E0B6018BE093E30E94D0F6D70134
:1063F00014968C9114978D8315968C9115978E8396
:1064000016968C9116978F838D919D910D90BC91CE
:10641000A02D89839A83AB83BC8360E185E00F94D0
:106420008308BE016F5F7F4F80EA9AE00E9473612C
:106430000E94EBF108C08FEB91E40E949ABF81307B
:1064400041F00E9441190E94FEF1803A9F4098F36A
:106450007AC011111DC08CE0E2E6F2E2A1EDBDE3CD
:1064600001900D928A95E1F7E1EDFDE301900020A6
:10647000E9F73197AF01415D5D4321E061ED7DE3D7
:106480008BE093E30E94D0F682E080934C4278C088
:106490001130E9F48BE0EEE6F2E2A1EDBDE301900C
:1064A0000D928A95E1F7E1EDFDE301900020E9F717
:1064B0003197AF01415D5D4321E061ED7DE38BE00C
:1064C00093E30E94D0F681E080934C4259C0123091
:1064D000E9F48BE0E9E7F2E2A1EDBDE301900D9272
:1064E0008A95E1F7E1EDFDE301900020E9F73197AE
:1064F000AF01415D5D4321E061ED7DE38BE093E31E
:106500000E94D0F683E080934C423AC08BE0E4E8EE
:10651000F2E2A1EDBDE301900D928A95E1F7E1ED84
:10652000FDE301900020E9F73197AF01415D5D4344
:1065300021E061ED7DE38BE093E30E94D0F684E0FF
:1065400080934C421DC01F5F143009F0D2CE89E009
:10655000EFE8F2E2A1EDBDE301900D928A95E1F73B
:10656000E1EDFDE301900020E9F73197AF01415DD6
:106570005D4321E061ED7DE38BE093E30E94D0F683
:106580002796CDBFDEBFDF91CF911F91FF90EF9097
:10659000DF90CF90BF90AF909F908F907F906F9043
:1065A0005F904F900895CF92DF92EF92FF920F93FA
:1065B0001F93CF930E94C6B0882309F49CC080E447
:1065C00096E30E942012883009F495C080E496E397
:1065D0000E942012863009F48EC00E94AFF28823F8
:1065E00019F10E94B9F281111FC00E94BCF20E94F1
:1065F000E426811119C088E1E8E9F2E2A1EDBDE3EA
:1066000001900D928A95E1F7E1EDFDE30190002004
:10661000E9F73197AF01415D5D4321E061ED7DE335
:106620008BE093E30E94D0F60E94A5F2882309F440
:1066300062C00E94BFEF0E9461460E94E426811161
:1066400019C08EE0E0EBF2E2A1EDBDE301900D9206
:106650008A95E1F7E1EDFDE301900020E9F731973C
:10666000AF01415D5D4321E061ED7DE38BE093E3AC
:106670000E94D0F60E941FEC01E010E0C0E00F2E57
:10668000F2E1CF2EF1E2DF2EF02D0F2EF1EDEF2E05
:10669000FDE3FF2EF02D0E940EEC882341F10E94B5
:1066A0001FECCF5F0E94E42681111CC01F930F9343
:1066B000DF92CF92FF92EF920F94D92AF7010190C7
:1066C0000020E9F73197AF01415D5D4321E0B7015B
:1066D0008BE093E30E94D0F60F900F900F900F90F5
:1066E0000F900F900F5F1F4FC33019F0D4CFC330FE
:1066F00090F20E9454E0CF911F910F91FF90EF9084
:10670000DF90CF900895F8940E94F2560F942E08CF
:106710000E9445FF0E94AD8D0E94F0E20E9474C26B
:1067200041E060EA78E082E194E30E9432F765E1BB
:1067300070E280EA98E00E94822BE0EAF8E0838130
:106740008F7C806183838FE69BE30E946DF661E01E
:1067500081E59BE30E94EA8E41E060EA7BE089E903
:1067600098E30E9432F76EE070E280EA9BE00E94BC
:10677000822BE0EAFBE083818F7C806183838BE165
:106780009AE30E94C78E8BE19AE30E94D98E61E062
:1067900080E69BE30E94EA8E10926E3B1092753C5D
:1067A00082EF9BE30E946DF641E060EA7AE089E2C5
:1067B00095E30E9432F767E070E280EA9AE00E9477
:1067C000822BE0EAFAE083818F7C8061838341E061
:1067D00060EA79E08BE093E30E9432F760E070E2D8
:1067E00080EA99E00E94822BE0EAF9E083818F7CC5
:1067F0008061838383E59EE30E946DF60E94B1EB86
:106800000E947AED0E940BEF0E9487F10E949EED9C
:106810000E9403E10E94ADE40E94380DC0E08C2F7D
:106820000E9414E3CF5FC830D1F787E08093A200C5
:106830007894E0E2F6E082E0868384E086830E943A
:10684000D3A8811110C00E94D9A90E9403AA0E9456
:106850001EAF0E94A2AF0E9497B00E94DEB081E0FE
:1068600080938C3827C00E9491AE882309F181E083
:1068700080938C380E94E42681111CC08DE1EEEBE0
:10688000F2E2A1EDBDE301900D928A95E1F7E1ED11
:10689000FDE301900020E9F73197AF01415D5D43D1
:1068A00021E061ED7DE38BE093E30E94D0F602C02E
:1068B00010928C380E9422AE0E9406E60E9471AEB1
:1068C00081E00E94BDEE6DE289EA92E30E94EE2B28
:1068D0000E94DE8F60EF7EE38FEB91E40E9402B6B0
:1068E0008FEB91E40E94E4B080E496E30E942712CB
:1068F00080E00E9426E48DE790E40E944BBE80E495
:1069000096E3DBDA81E00E94D1A280E00E94CBA274
:1069100080E00E94D4A280E00E94D7A20E94FF14CF
:106920000E94B18D8FEB91E40E94E4B087E090E289
:10693000B3DC0E940FBC813029F480918D380E9415
:10694000DDC125C00E940FBC823091F481E00E941D
:1069500012BC80918D38882329F08DE790E40E9445
:106960002FBD02C00E94FABC81E00E94C4BC0FC0CF
:106970000E940FBC833029F481ED9DE30E94F4BD99
:1069800006C00E940FBC843011F40E941BC284E038
:10699000809326060E9480C280E496E30E947E26B1
:1069A0008BE093E30E947A960E94740D0BED12E245
:1069B000C1EDDDE30E94BC2C60EF7EE38FEB91E440
:1069C0000E94361480E496E30E94C71380E496E3A5
:1069D0000E945F1380E496E30E944B2B80E496E3D1
:1069E0000E941E290E94C12CDEDB0E94F42C36D8A6
:1069F00080E496E30E944B190E94ADC20E94CEA291
:106A0000833031F50E94BD1C882311F10E94E426D9
:106A100081111EC00E949CEF1F928F931F930F93B2
:106A2000DF93CF930F94D92AFE0101900020E9F75C
:106A30003197AF01415D5D4321E0BE018BE093E3FF
:106A40000E94D0F60F900F900F900F900F900F9024
:106A50000E941E2162EB7CE380E496E30E946822A0
:106A600062EB7CE380E496E30E94BC220E9431E565
:106A70009ADD0FB607FC9ECF80E00E946F6C0E94EB
:106A8000836CFFCFEF92FF920F931F93CF93DF930F
:106A9000009749F16115710541F14115510539F131
:106AA0008A017B01EC010F94682AF80180839183AD
:106AB000892B89F0D70120E030E0FE01E20FF31FBF
:106AC000E491ED932F5F3F4FF8018081918128176A
:106AD000390798F302C020E030E0F701E20FF31F1E
:106AE000108281E005C080E003C080E001C080E04A
:106AF000DF91CF911F910F91FF90EF9008950F9329
:106B00001F93CF93DF930097C9F061157105C1F012
:106B100041155105B9F0EA018B01FC0165917491B1
:106B2000C8010F94612AF80101900020E9F731971C
:106B3000E01BF10BE883F98381E005C080E003C02E
:106B400080E001C080E0DF91CF911F910F91089507
:106B50007F928F929F92AF92BF92CF92DF92EF92ED
:106B6000FF920F931F93CF93DF931F921F92CDB786
:106B7000DEB7009709F49BC06115710509F497C051
:106B8000D42E7B018C01AE014F5F5F4FBC0188E0CA
:106B900091E178DF882309F48AC089819A815C01B8
:106BA0002FEFA21AB20AF801E80FF91F20E22083A2
:106BB000B8016A0D7B1DAE014F5F5F4F81EF90E121
:106BC00061DF882309F473C089819A81A80EB91EF8
:106BD000F801EA0DFB1D8DE0808382E0A80EB11C58
:106BE0008AE08183B8016A0D7B1DAE014F5F5F4F64
:106BF0008AED90E147DF882309F459C0A981BA8161
:106C0000AA0EBB1E48018A0C9B1C0F2EFDE07F2E96
:106C1000F02DF40170820F2EFAE0CF2EF02DC182FC
:106C2000C5010296800F911F0E94F9A8F401748E8D
:106C3000D5015E96C58EDD2059F1A00FB11F8AE007
:106C4000E3EEF2E201900D928A95E1F7F7E2AF0EE2
:106C5000B11C0E94F1AEBC01C8018A0D9B1D0F94AE
:106C6000C32A0E94F1AEFC0101900020E9F73197A0
:106C7000E81BF90BE131F10518F4E983FA8304C04C
:106C800080E190E089839A83A981BA81AA0DBB1D16
:106C9000F801EA0FFB1F8DE0808312968AE0818362
:106CA000F801EA0FFB1F1082F701A083B1830F9058
:106CB0000F90DF91CF911F910F91FF90EF90DF9098
:106CC000CF90BF90AF909F908F907F900895CF927C
:106CD000DF92EF92FF920F931F93CF93DF931F9258
:106CE0001F92CDB7DEB76115710591F141155105C0
:106CF00079F1009769F17A016B018C0119821A828E
:106D0000AE014F5F5F4F8EE290E1BCDE882301F160
:106D1000C80106969F938F938DEE92E29F938F9377
:106D200089819A818C0D9D1D9F938F930F94D92AF1
:106D3000F60101900020E9F73197EC19FD09D70120
:106D4000ED93FC930F900F900F900F900F900F907A
:106D50000F900F90DF91CF911F910F91FF90EF90C7
:106D6000DF90CF900895BF92CF92DF92EF92FF9283
:106D70000F931F93CF93DF931F921F92CDB7DEB770
:106D8000009709F482C06115710509F47EC06B019A
:106D90008C0119821A82DB011D921C92AE014F5F99
:106DA0005F4FBC0182E290E16DDE882309F46DC083
:106DB000ECE7F7E487858F9386858F9385858F939E
:106DC00084858F938AE399E29F938F9389819A8137
:106DD000800F911F9F938F930F94D92AF8010190F0
:106DE0000020E9F73197E01BF10BE983FA83CDBF6F
:106DF000DEBFB12C0F2EF2EFEF2EF2E2FF2EF02DC0
:106E00002DC0EB2DF0E0EE0FFF1FEE0FFF1FE4583B
:106E1000F84BDF015A9613968C9113978F93129625
:106E20008C9112978F9311968C918F93828D8F9363
:106E3000FF92EF9289819A81800F911F9F938F9388
:106E40000F94D92AF80101900020E9F73197E01B4F
:106E5000F10BE983FA83B394CDBFDEBF0E94C0F289
:106E6000B81678F2E981FA81E00FF11F8DE09AE01F
:106E7000808391831282F80101900020E9F7319715
:106E8000E01BF10BD601ED93FC930F900F90DF9177
:106E9000CF911F910F91FF90EF90DF90CF90BF9017
:106EA0000895CF92DF92EF92FF920F931F93CF93AB
:106EB000DF9300D01F92CDB7DEB719821A821B82F2
:106EC0001C82009709F445C06115710509F441C0A1
:106ED000CC24CA94C20E29E02C1508F4C12CD42E5F
:106EE0007B018C01AE014F5F5F4FBC018AE390E1F3
:106EF000C9DD882371F1DD2091F069817A81600F0D
:106F0000711F2C2D30E0C901880F991FAE014D5F14
:106F10005F4F815C984FF3DD811112C01AC0698107
:106F20007A81600F711F2C2D30E0C901880F991FE5
:106F3000AE014D5F5F4F855D984FE1DD882349F0DD
:106F400029813A818B819C81820F931FF701808375
:106F500091832496CDBFDEBFDF91CF911F910F911A
:106F6000FF90EF90DF90CF90089589E10E943BA9B8
:106F700081E0623009F080E00895CF92DF92EF92D5
:106F8000FF921F93CF93DF9300D01F92CDB7DEB750
:106F900019821A821B821C82009709F453C0611562
:106FA000710509F44FC0142F6B017C01AE014F5FD6
:106FB0005F4FBC018AE390E165DD882309F442C09C
:106FC000173089F01930E1F0113039F569817A8193
:106FD0006E0D7F1DAE014D5F5F4F8DE298E052DD7B
:106FE000811127C02FC069817A816E0D7F1DAE018E
:106FF0004D5F5F4F8CEC97E045DD81111AC022C0D8
:1070000069817A816E0D7F1DAE014D5F5F4F8BE60A
:1070100097E038DD81110DC015C069817A816E0D50
:107020007F1DAE014D5F5F4F8DE298E02BDD882321
:1070300049F029813A818B819C81820F931FF6014F
:10704000808391832496CDBFDEBFDF91CF911F91C6
:10705000FF90EF90DF90CF900895EF92FF920F9303
:107060001F93CF93DF931F921F92CDB7DEB7198284
:107070001A820097D9F061157105C1F07B018C016E
:10708000AE014F5F5F4FBC0186E490E1FBDC8823DB
:1070900069F089819A81F801E80FF91F2DE02083BA
:1070A0002AE021830296F701808391830F900F904D
:1070B000DF91CF911F910F91FF90EF900895EF9284
:1070C000FF920F931F93CF93DF931F921F92CDB721
:1070D000DEB7009709F47EC04115510509F47CC064
:1070E000F22E8A01E62EAE014F5F5F4FB80107DD39
:1070F000811102C019821A8283E0E81629F18E15E7
:1071000038F091E0E91659F082E0E81699F03AC0BB
:1071100094E0E91619F185E0E81651F133C0EDE786
:10712000F0E401900020E9F73197ED57F0446DE766
:1071300070E42BC0E4E9F0E401900020E9F7E559A0
:10714000F04464E970E421C0EBEAF0E4019000202F
:10715000E9F7EC5AF0446BEA70E417C0E2ECF0E4B3
:1071600001900020E9F7E35CF04462EC70E40DC0AC
:10717000E9EDF0E401900020E9F7EA5DF04469ED03
:1071800070E403C06DE770E4E0E0EF3008F0EEE09B
:10719000CB018E0F911DFC01108289819A81800F95
:1071A000911F0F94C32AF80101900020E9F731974D
:1071B000E01BF10BFF2091F0C8018E0F911DFC0127
:1071C0008CE29DE0808391838AE090E082839383C8
:1071D00081E005C080E003C080E001C081E00F9045
:1071E0000F90DF91CF911F910F91FF90EF90089535
:1071F0008F929F92AF92BF92CF92DF92EF92FF92C7
:107200000F931F93CF93DF931F921F92CDB7DEB7DB
:1072100030918D38311104C0FB011082118236C0CB
:107220000097A1F1672B91F14115510579F1022FDA
:107230004A016C010F2EF3EEEF2EF5E1FF2EF02D3B
:1072400011E0202FA601612FC70139DF8823A9F0A3
:10725000F60101900020E9F731975F01AC18BD08F5
:107260009E012F5F3F4FA501B601C4010F945D1F22
:1072700089819A81A816B90631F41F5FF2E0EF0EFA
:10728000F11C1630F1F6C4010F940B210F900F90F2
:10729000DF91CF911F910F91FF90EF90DF90CF90F2
:1072A000BF90AF909F908F9008958F929F92AF92D2
:1072B000BF92DF92EF92FF920F931F93CF93DF93D2
:1072C000CDB7DEB72597CDBFDEBF009709F493C4D5
:1072D0004115510509F491C4D22E7A01162FAE0141
:1072E0004F5F5F4FB7010BDC811102C019821A8218
:1072F000163109F06DC00E940FD64B015C01672B5F
:10730000682B692BE1F486E10E943BA920E13EE075
:1073100040E050E00F94B5285F934F933F932F9335
:107320008DEF92E29F938F9389819A818E0D9F1D9D
:107330009F938F930F94D92ACDBFDEBF45C486E1BA
:107340000E943BA9992324F586E10E943BA920E1F4
:107350003EE040E050E00F94B528CA01B9010E9418
:10736000E9FBBF92AF929F928F929F938F937F93EF
:107370006F9388EF92E29F938F9389819A818E0D0C
:107380009F1D9F938F930F94D92ACDBFDEBF1CC43E
:1073900086E10E943BA9BF92AF929F928F9220E11B
:1073A0003EE040E050E00F94B5285F934F933F9349
:1073B0002F9389EF92E29F938F9389819A818E0D0B
:1073C0009F1D9F938F930F94D92ACDBFDEBFFCC31F
:1073D000123060F4812F0E94A0A929813A81BC015A
:1073E000C701820F931F0F94C32AEEC3163081F496
:1073F00086E00E943BA98B019C0189819A814BE028
:10740000BE016B5F7F4F8E0D9F1D0E9442FCDCC34F
:10741000153081F485E00E943BA98B019C01898194
:107420009A814BE0BE016B5F7F4F8E0D9F1D0E94C6
:107430008EFDCAC3123009F06EC082E00E943BA9E3
:107440006B3071058105910524F061E070E080E00A
:1074500090E0013009F049C029813A812E0D3F1D8D
:10746000DC01CB010197A109B109880F991FAE0179
:107470004D5F5F4FB9018555994F41DB8130F9F47C
:10748000F70101900020E9F73197EE19FF09E98330
:10749000FA8382E00E943BA99F938F937F936F931F
:1074A00082E093E29F938F9389819A818E0D9F1D35
:1074B0009F938F930F94D92ACDBFDEBF85C382E0FF
:1074C0000E943BA99F938F937F936F9383E093E2F6
:1074D0009F938F9389819A818E0D9F1D9F938F9388
:1074E0000F94D92ACDBFDEBF6FC382E00E943BA9B3
:1074F0009F938F937F936F938BE399E29F938F93E7
:1075000089819A818E0D9F1D9F938F930F94D92A05
:10751000CDBFDEBF59C31B3059F08DEE810F8230D5
:1075200038F089EE810F823018F01A3109F05CC012
:10753000812F0E943BA94B015C01011113C0BF9236
:10754000AF929F926F938BE399E29F938F93898180
:107550009A818E0D9F1D9F938F930F94D92ACDBF33
:10756000DEBF32C3672B682B692BF9F469817A81FE
:107570006E0D7F1DAE014D5F5F4F87EA96E082DAA8
:10758000811122C31F921F921F921F928BE399E2D7
:107590009F938F9389819A818E0D9F1D9F938F93C7
:1075A0000F94D92ACDBFDEBF0FC369817A816E0DDA
:1075B0007F1DAE014D5F5F4F84EA96E063DA811173
:1075C00003C3BF92AF929F928F928BE399E29F93F6
:1075D0008F9389819A818E0D9F1D9F938F930F9416
:1075E000D92ACDBFDEBFF0C2173009F05CC087E0FA
:1075F0000E943BA94B015C01011113C0BF92AF92E5
:107600009F926F938BE399E29F938F9389819A81E5
:107610008E0D9F1D9F938F930F94D92ACDBFDEBFF0
:10762000D3C2672B682B692BF9F469817A816E0DBF
:107630007F1DAE014D5F5F4F80EA96E023DA811136
:10764000C3C21F921F921F921F928BE399E29F93D6
:107650008F9389819A818E0D9F1D9F938F930F9495
:10766000D92ACDBFDEBFB0C269817A816E0D7F1D80
:10767000AE014D5F5F4F8CE996E004DA8111A4C240
:10768000BF92AF929F928F928BE399E29F938F93D9
:1076900089819A818E0D9F1D9F938F930F94D92A74
:1076A000CDBFDEBF91C2143009F05CC084E00E94FF
:1076B0003BA94B015C01011113C0BF92AF929F9295
:1076C0006F938BE399E29F938F9389819A818E0DBB
:1076D0009F1D9F938F930F94D92ACDBFDEBF74C295
:1076E000672B682B692BF9F469817A816E0D7F1DF8
:1076F000AE014D5F5F4F85E996E0C4D9811164C248
:107700001F921F921F921F928BE399E29F938F9378
:1077100089819A818E0D9F1D9F938F930F94D92AF3
:10772000CDBFDEBF51C269817A816E0D7F1DAE0172
:107730004D5F5F4F8CE896E0A5D9811145C2BF929D
:10774000AF929F928F928BE399E29F938F9389815F
:107750009A818E0D9F1D9F938F930F94D92ACDBF31
:10776000DEBF32C2133009F0ABC083E00E943BA9F8
:107770004B015C01011113C0BF92AF929F926F93B6
:107780008BE399E29F938F9389819A818E0D9F1D40
:107790009F938F930F94D92ACDBFDEBF15C291E07E
:1077A00089169104A104B10461F182E08816910464
:1077B000A104B10409F445C081149104A104B104E9
:1077C00009F05FC069817A816E0D7F1DAE014D5F4A
:1077D0005F4F80E896E056D98111F6C11F921F9243
:1077E0001F921F928BE399E29F938F9389819A81D5
:1077F0008E0D9F1D9F938F930F94D92ACDBFDEBF0F
:10780000E3C169817A816E0D7F1DAE014D5F5F4FCF
:1078100087E796E037D98111D7C11F921F921F9237
:1078200081E08F938BE399E29F938F9389819A8173
:107830008E0D9F1D9F938F930F94D92ACDBFDEBFCE
:10784000C3C169817A816E0D7F1DAE014D5F5F4FAF
:1078500082E796E017D98111B7C11F921F921F923C
:1078600082E08F938BE399E29F938F9389819A8132
:107870008E0D9F1D9F938F930F94D92ACDBFDEBF8E
:10788000A3C169817A816E0D7F1DAE014D5F5F4F8F
:1078900080E896E0F7D8811197C1BF92AF929F928E
:1078A0008F928BE399E29F938F9389819A818E0DBA
:1078B0009F1D9F938F930F94D92ACDBFDEBF84C1A4
:1078C000193109F0ABC089E10E943BA94B015C0171
:1078D000011113C0BF92AF929F926F938BE399E215
:1078E0009F938F9389819A818E0D9F1D9F938F9374
:1078F0000F94D92ACDBFDEBF67C191E089169104EC
:10790000A104B10461F182E088169104A104B104DC
:1079100009F445C081149104A104B10409F05FC0C9
:1079200069817A816E0D7F1DAE014D5F5F4F8EE6DE
:1079300096E0A8D8811148C11F921F921F921F92F2
:107940008BE399E29F938F9389819A818E0D9F1D7E
:107950009F938F930F94D92ACDBFDEBF35C1698124
:107960007A816E0D7F1DAE014D5F5F4F88E696E018
:1079700089D8811129C11F921F921F9281E08F9394
:107980008BE399E29F938F9389819A818E0D9F1D3E
:107990009F938F930F94D92ACDBFDEBF15C1698104
:1079A0007A816E0D7F1DAE014D5F5F4F80E696E0E0
:1079B00069D8811109C11F921F921F9282E08F9393
:1079C0008BE399E29F938F9389819A818E0D9F1DFE
:1079D0009F938F930F94D92ACDBFDEBFF5C06981E5
:1079E0007A816E0D7F1DAE014D5F5F4F8EE696E092
:1079F00049D88111E9C0BF92AF929F928F928BE3D9
:107A000099E29F938F9389819A818E0D9F1D9F93F9
:107A10008F930F94D92ACDBFDEBFD6C0123109F0A3
:107A20005DC082E10E943BA94B015C01011113C0C2
:107A3000BF92AF929F926F938BE399E29F938F9344
:107A400089819A818E0D9F1D9F938F930F94D92AC0
:107A5000CDBFDEBFB9C0672B682B692BF9F46981F4
:107A60007A816E0D7F1DAE014D5F5F4F8FE496E012
:107A700009D88111A9C01F921F921F921F928BE3F8
:107A800099E29F938F9389819A818E0D9F1D9F9379
:107A90008F930F94D92ACDBFDEBF96C069817A81BA
:107AA0006E0D7F1DAE014D5F5F4F87E496E00E9433
:107AB0004235811189C0BF92AF929F928F928BE322
:107AC00099E29F938F9389819A818E0D9F1D9F9339
:107AD0008F930F94D92ACDBFDEBF76C0153109F040
:107AE0005EC085E10E943BA94B015C01011113C0FE
:107AF000BF92AF929F926F938BE399E29F938F9384
:107B000089819A818E0D9F1D9F938F930F94D92AFF
:107B1000CDBFDEBF59C0672B682B692B01F569818A
:107B20007A816E0D7F1DAE014D5F5F4F8BE596E054
:107B30000E944235811148C01F921F921F921F92CE
:107B40008BE399E29F938F9389819A818E0D9F1D7C
:107B50009F938F930F94D92ACDBFDEBF35C0698123
:107B60007A816E0D7F1DAE014D5F5F4F86E596E019
:107B70000E944235811128C0BF92AF929F928F928E
:107B80008BE399E29F938F9389819A818E0D9F1D3C
:107B90009F938F930F94D92ACDBFDEBF15C0812F3D
:107BA0000E943BA99F938F937F936F938BE399E2FE
:107BB0009F938F9389819A818E0D9F1D9F938F93A1
:107BC0000F94D92ACDBFDEBFF70101900020E9F75D
:107BD0003197EE19FF09DD2091F0C7018E0F911D3D
:107BE000FC018CE29DE0808391838AE090E08283B7
:107BF000938381E005C080E003C080E001C081E0A4
:107C00002596CDBFDEBFDF91CF911F910F91FF90E1
:107C1000EF90DF90BF90AF909F908F9008956F92FC
:107C20007F928F929F92AF92BF92CF92DF92EF920C
:107C3000FF920F931F93CF93DF931F921F92CDB7A5
:107C4000DEB70097B1F1672BA1F14115510589F11C
:107C5000802E922E3A016C010F2EF4E7EF2EF7E101
:107C6000FF2EF02D10E0082D292DA601612FC70150
:107C70001CDB8823A9F0F60101900020E9F7319779
:107C80005F01AC18BD089E012F5F3F4FA501B601F3
:107C9000C3010F945D1F89819A81A816B90631F43A
:107CA0001F5F82E0E80EF11C1C31E9F6C3010F945E
:107CB0000B210F900F90DF91CF911F910F91FF90AB
:107CC000EF90DF90CF90BF90AF909F908F907F907C
:107CD0006F9008958F929F92AF92BF92DF92EF9232
:107CE000FF920F931F93CF93DF931F921F92CDB7F5
:107CF000DEB7009709F45EC06115710509F45AC03A
:107D00004B017C010E94F1AE9F938F9389E093E237
:107D10009F938F93FF92EF920F94D92AF7010190CE
:107D20000020E9F73197AF014E195F094231510543
:107D300010F041E150E09E012F5F3F4FB701C401B9
:107D40000F945D1F0F900F900F900F900F900F905A
:107D5000D12C0F2EF8E1AF2EF9E2BF2EF02D8D2D94
:107D60000E9417A99F938F937F936F93BF92AF92B7
:107D7000FF92EF920F94D92AF70101900020E9F7C2
:107D800031978F010E191F099E012F5F3F4FA801E8
:107D9000B701C4010F945D1FCDBFDEBF89819A81F9
:107DA0000817190721F4D39494E1D912D8CFC4014C
:107DB0000F940B210F900F90DF91CF911F910F9196
:107DC000FF90EF90DF90BF90AF909F908F900895BD
:107DD0002F923F924F925F926F927F928F929F92DB
:107DE000AF92BF92CF92DF92EF92FF920F931F93C9
:107DF000CF93DF93CDB7DEB7E197CDBFDEBF91E084
:107E00009BA76115710509F4B6C34115510509F425
:107E1000B4C38A017B0189AB0E9478F229A9213081
:107E200089F4A8016BE17DE2CE010B960E948747A1
:107E3000182F86E08BA70E94B4E66DA77EA78FA7B8
:107E400098AB1AC0A8016BE17DE2CE010B960E94AF
:107E5000FC47182F0E94B4E66DA77EA78FA798ABAA
:107E600082E00E9449E5862FAE01445D5F4FBE016E
:107E7000655D7F4F0E94051F112309F480C341E017
:107E8000BE01675F7F4FC7010E94A83549855A85AB
:107E9000CA01A0E0B0E089839A83AB83BC839E01D2
:107EA000275F3F4FB701CE010B960F945D1FCE01A8
:107EB0000B960F940B21BE01655F7F4FC7010ADF50
:107EC0000DE0D7010C931AE011961C939E01275FD9
:107ED0003F4F42E050E0B701CE010B960F945D1F7B
:107EE000CE010B960F940B21EBE1FDE2018B128B7F
:107EF0009E01275F3F4F43E150E0BF01CE010B964B
:107F00000F945D1FCE010B960F940B21B9A9B111EF
:107F10003CC30E9409E70E94F2E637C301E021E07A
:107F2000A701612FC601C1D9882381F0F701019013
:107F30000020E9F73197AF014E195F099E01275FD5
:107F40003F4FB701CE010B960F945D1FE2E0CE0EBE
:107F5000D11C1F5F133011F70F2EF6E8CF2EF7E17B
:107F6000DF2EF02D19E001E021E0A701612FC6010D
:107F70009CD9882381F0F70101900020E9F731971F
:107F8000AF014E195F099E01275F3F4FB701CE0138
:107F90000B960F945D1FF2E0CF0ED11C1F5F1B30BC
:107FA00011F70F2EF2E18F2E912CA12CB12CF02D78
:107FB00028E182169104A104B10451F401E021E00A
:107FC000A70169E186EA97E170D981110EC030C03E
:107FD00001E021E0A701682DC401880F991F8C588A
:107FE000984E63D98823C1F007C00F2EF9E18F2E78
:107FF000912CA12CB12CF02DF70101900020E9F774
:108000003197AF014E195F099E01275F3F4FB701BE
:10801000CE010B960F945D1F33E0830E911CA11CC3
:10802000B11C4AE184169104A104B10408F4C0CF44
:10803000CE010B960F940B2189E00E943BA96F3172
:10804000710581059105C0F4DC01CB01072E7CE0B0
:10805000880F991FAA1FBB1F7A95D1F7702D8983AE
:108060009A83AB83BC8380E090E1A0E0B0E08D8395
:108070009E83AF83B88717C0DC01CB01072E79E060
:10808000880F991FAA1FBB1F7A95D1F7702D89837E
:108090009A83AB83BC8380E092E0A0E0B0E08D8364
:1080A0009E83AF83B88789819A81AB81BC812DA5DE
:1080B0003EA54FA558A9281739074A075B07A1F124
:1080C000AE01475F5F4FB7018FE597E00E944235F1
:1080D000813081F4F70101900020E9F73197AF0179
:1080E0004E195F099E01275F3F4FB701CE010B96E6
:1080F0000F945D1FCE010B960F940B21CE010B96B2
:108100000F94522139A931113CC20E9480E780E4CA
:1081100096E30E94901F81110E94E1EF80E496E3B4
:108120000E947E2680E039C2AE01475F5F4FB701F3
:1081300083E597E00E944235813081F4F701019098
:108140000020E9F73197AF014E195F099E01275FC3
:108150003F4FB701CE010B960F945D1F48A94F9377
:108160005FA55F938EA58F939DA59F9388858F9321
:108170008F818F938E818F938D818F938DE093E28A
:108180009F938F93FF92EF920F94D92AF70101905A
:108190000020E9F73197AF014E195F099E01275F73
:1081A0003F4FB701CE010B960F945D1F88E290E020
:1081B00089879A8768E2C7010E94B495482F50E0EA
:1081C00060E070E049835A836B837C83682F70E0A2
:1081D000C7010E94D2FDCDBFDEBF8823C9F049810F
:1081E0005A819E01275F3F4FB701CE010B960F9436
:1081F0005D1F8DE0F70180838AE081839E01275F08
:108200003F4F42E050E0B701CE010B960F945D1F47
:10821000BE016F5F7F4FC7010E942D3849815A818F
:108220009E01275F3F4FB701CE010B960F945D1F54
:108230006BE370E0C7010E940795A0E0B0E089837E
:108240009A83AB83BC830E94E42681110EC0F701A0
:1082500001900020E9F73197AF014E195F0920E046
:10826000B7018BE093E30E94D0F649815A816B817C
:108270007C814115510561057105C1F09E01275FA3
:108280003F4FB701CE010B960F945D1F8DE0D701D4
:108290008C938AE011968C939E01275F3F4F42E0BA
:1082A00050E0B701CE010B960F945D1FCE010B96E7
:1082B0000F940B210E94A64B19821A821B821C82EA
:1082C0002DA53EA54FA558A9232B242B252B09F41A
:1082D00033C180E090E0DC010F2EF6E42F2EF3E2B4
:1082E0003F2EF02D0F2EF8E18F2EF3E29F2EF02D72
:1082F000880F991FAA1FBB1FBC01CD017E5F8F4F46
:108300009F4F0E94AE4B0E94394E8111FCCF80E0FE
:1083100091E0E7ECFCE3DF019C011D92215030402D
:10832000E1F76F010F2EF7ECAF2EFDE3BF2EF02D1E
:108330008F010E94C894D8018D939D938D01AA1638
:10834000BB06B9F70E94794C0E9445FFCE010B96FF
:108350000F940B21412C512C3201F6016191719146
:108360006F01AE014B5F5F4F8BA50E94D412882333
:1083700009F496C088858F938F818F938E818F9318
:108380008D818F9389819A81AB81BC81840D951DEC
:10839000A61DB71DBF93AF939F938F939F928F920C
:1083A000FF92EF920F94D92AF70101900020E9F78C
:1083B0003197AF014E195F099E01275F3F4FB7010B
:1083C000CE010B960F945D1F182FCDBFDEBF882303
:1083D00009F48CC00E94E426811126C089819A810B
:1083E000AB81BC81840D951DA61DB71DBF93AF93B6
:1083F0009F938F931F921F9342E253E25F934F9399
:10840000FF92EF920F94D92AF70101900020E9F72B
:108410003197AF014E195F0920E0B7018BE093E37C
:108420000E94D0F6CDBFDEBFF70101900020E9F732
:108430003197AF014E195F099E01275F3F4FB7018A
:10844000CE010B960F945D1F182F0E94E426811118
:108450004DC089819A81AB81BC81840D951DA61D7B
:10846000B71DBF93AF939F938F931F921F93E3E327
:10847000F3E2FF93EF93FF92EF920F94D92AF70163
:1084800001900020E9F73197AF014E195F0920E014
:10849000B7018BE093E30E94D0F6CDBFDEBF26C0CC
:1084A0000E94E426811122C089819A81AB81BC811E
:1084B000840D951DA61DB71DBF93AF939F938F93FA
:1084C0003F922F92FF92EF920F94D92AF7010190D9
:1084D0000020E9F73197AF014E195F0920E0B7019D
:1084E0008BE093E30E94D0F6CDBFDEBF9FEF491A29
:1084F000590A690A790AA0E84A165104610471040C
:1085000009F02BCFCE010B960F940B2189819A8114
:10851000AB81BC8180589F4FAF4FBF4F89839A83F7
:10852000AB83BC832DA53EA54FA558A98217930701
:10853000A407B50708F4DCCECE010B960F940B21EF
:10854000CE010B960F94522110922C2D8BE19DE2BF
:1085500032D639A9311117C00E9480E780E496E332
:108560000E94901F81110E94E1EF80E496E30E9437
:108570007E2681E012C080E010C080E00EC080E066
:108580000CC080E00AC081E008C00F2EF4E7CF2EB7
:10859000F7E1DF2EF02D10E0C1CCE196CDBFDEBFBC
:1085A000DF91CF911F910F91FF90EF90DF90CF90CF
:1085B000BF90AF909F908F907F906F905F904F9003
:1085C0003F902F900895CF92DF92EF92FF920F93FA
:1085D0001F93CF93DF931F921F92CDB7DEB7009703
:1085E00009F457C06115710509F453C07B018C0172
:1085F000AE014F5F5F4FBC0188E091E10E944235C0
:10860000882309F446C089819A816C012FEFC21A30
:10861000D20AF801E80FF91F20E22083B8016C0D9F
:108620007D1DAE014F5F5F4F81EF90E10E944235AB
:10863000882379F189819A81C80ED91EF801EC0D41
:10864000FD1D8DE0808382E0C80ED11C8AE081830D
:10865000B8016C0D7D1DAE014F5F5F4F83EC90E163
:108660000E9442358823A9F089819A81C80ED91EBB
:10867000F801EC0DFD1D8DE0808322E0C20ED11CBF
:108680008AE08183F801EC0DFD1D1082F701C082A4
:10869000D1820F900F90DF91CF911F910F91FF909A
:1086A000EF90DF90CF900895EF92FF920F931F937A
:1086B000CF93DF93CDB7DEB7A297CDBFDEBF0097D4
:1086C00009F451C06115710509F44FC07B018C019B
:1086D00060E0CE01039605D5882309F44BC0B701AD
:1086E000C80171DFF701408151819E012F5F3F4F2B
:1086F000B801CE0103960F945D1FCE0103960F942F
:108700000B21F7012081318189819A81281739074E
:1087100071F5BE016D5F7F4FC801DCDAA701B801BA
:108720008CEA97E10E944235813099F4F70140814B
:1087300051819E012F5F3F4FB801CE0103960F94E8
:108740005D1FF7012081318189819A8128173907BE
:1087500081F4CE0103960F94522181E002D50E944C
:1087600078F281E007C080E005C080E003C080E0CF
:1087700001C080E0A296CDBFDEBFDF91CF911F91F7
:108780000F91FF90EF9008950F931F93CF93DF9376
:108790001F921F92CDB7DEB70E9478F28091803889
:1087A000823009F462C028F4882359F0813081F1C5
:1087B000D6C0843009F485C008F464C08A30E1F082
:1087C000CEC060E080EC99E36FD3811107C0609167
:1087D000813880E496E30E940D12C9C00E942BE10B
:1087E000811104C081E080938038C1C08AE0809309
:1087F00080380E9489F0BBC00E94A0F06C3D75409B
:108800008105910508F4B3C081E080938038AFC042
:1088100040E062E776E384E796E30E94A83500E44F
:1088200016E3F80142A953A99E012F5F3F4F64E769
:1088300076E380EC99E30F945D1F80EC99E30F944D
:108840000B21F80122A933A989819A8128173907B8
:1088500041F01092803860918138C8010E940D1259
:1088600086C082E08093803882C000E021E040EC46
:1088700059E362E776E384E796E3D1D983E0809316
:10888000803875C042E756E364E776E38CEA97E107
:108890000E944235813069F44091723650917336AE
:1088A0009E012F5F3F4F64E776E380EC99E30F94DE
:1088B0005D1F80EC99E30F94522184E0809380380F
:1088C00056C00E940FBC882381F10E94D3F18823F7
:1088D000C9F00E94BD1C882309F449C080E496E3D6
:1088E0000E94901F81110E94E1EF80E496E30E94B4
:1088F0007E26109280386091813880E496E30E9451
:108900000D1235C080E496E30E94901F81110E94F1
:10891000E1EF80E496E30E947E261092803861E0C9
:1089200080E496E30E940D1222C00E941BF0672B88
:10893000682B692BE1F480E496E30E94901F81117B
:108940000E94E1EF80E496E30E947E261092803838
:108950006091813880E496E30E940D1208C0109265
:1089600080386091813880E496E30E940D120F9068
:108970000F90DF91CF911F910F9108959F92AF9229
:10898000BF92CF92DF92EF92FF920F931F93CF93FC
:10899000DF9300D0CDB7DEB7009709F471C0611541
:1089A000710509F46DC0A42E6B017C018EE0E1E538
:1089B000F3E2D70101900D928A95E1F7F70101905A
:1089C0000020E9F73197EE19FF09E983AF01552738
:1089D0009E012E5F3F4FB701C6010F945D1FB12C62
:1089E0000F2EFCE29F2EF02D8B2D0E9445B08B01A7
:1089F0009C0148E0BE016F5F7F4FC7010E94F0FD00
:108A000082E08B1550F08981F701E80FF11D90820B
:108A10008F5FF701E80FF11D1082F7010190002030
:108A2000E9F73197EE19FF09E983AF0155279E0158
:108A30002E5F3F4FB701C6010F945D1F898190E003
:108A40002A813B818217930721F4B394E4E0BE129C
:108A5000CBCFAA2081F08DE0F70180838AE081836B
:108A600082E089839E012E5F3F4F42E050E0B701D4
:108A7000C6010F945D1FC6010F940B210E9478F26E
:108A80002396CDBFDEBFDF91CF911F910F91FF9055
:108A9000EF90DF90CF90BF90AF909F9008959F92FE
:108AA000AF92BF92CF92DF92EF92FF920F931F93FC
:108AB000CF93DF931F921F92CDB7DEB7009709F4D3
:108AC000E0C06115710509F4DEC04115510509F4D6
:108AD000DCC0902E122F5A016B017C010E9478F2AB
:108AE00041E0B601C7010E94A835F60140815181DD
:108AF0009E012F5F3F4FB701C5010F945D1FC50158
:108B00000F940B21F6012081318189819A812817E8
:108B1000390709F0BCC08DE0EFE5F3E2D701019021
:108B20000D928A95E1F7F70101900020E9F731975E
:108B3000AF014E195F0955279E012F5F3F4FB701C7
:108B4000C5010F945D1FC5010F940B21B501C7012D
:108B5000C1D88DE0F70180838AE081839E012F5F79
:108B60003F4F42E050E0B701C5010F945D1FC501C2
:108B70000F940B2141E0B501C70100DFA601B70149
:108B800080E496E30E946736F601408151819E01A0
:108B90002F5F3F4FB701C5010F945D1FC5010F94B3
:108BA0000B21F6012081318189819A8128173907AB
:108BB00009F06FC0B601C7010E94B336F6014081CB
:108BC00051819E012F5F3F4FB701C5010F945D1F7B
:108BD000C5010F940B21F6012081318189819A8191
:108BE0002817390709F057C001E021E0A501B601B7
:108BF000C70115D821E0A501B601C7010E94F838C8
:108C00000E94B537882331F0492DB601C7010E9473
:108C1000BD3706C0292D412FB601C7010E9451372B
:108C2000F601408151819E012F5F3F4FB701C50181
:108C30000F945D1FC5010F940B21F6012081318136
:108C400089819A812817390741F5B601C7010E9429
:108C50002D38F601408151819E012F5F3F4FB701B2
:108C6000C5010F945D1FC5010F940B2181E0F60132
:108C70004081518129813A814217530779F080E080
:108C80000DC080E00BC080E009C080E007C080E03C
:108C900005C080E003C080E001C080E00F900F902D
:108CA000DF91CF911F910F91FF90EF90DF90CF90C8
:108CB000BF90AF909F90089508958091302D0895B2
:108CC00008951092302D80912F2D882331F010922D
:108CD0002F2D80EE99E30D945221089580EE99E3B3
:108CE0000D945221089580912F2D0895CF92DF92F7
:108CF000EF92FF921F93CF93DF93CDB7DEB76897C4
:108D0000CDBFDEBF6C017B0184E1ECE6F3E2DE0166
:108D1000159601900D928A95E1F7DA01C901019645
:108D2000A11DB11D883E23E09207A105B1050CF4F9
:108D300060C01F921F921F9281E08F9383EE90E29A
:108D40009F938F93CE0101969F938F930F94D92A6F
:108D50008981898B8A818A8B8B818B8B80E38D8340
:108D60008AE38E83CDBFDEBFE114F10459F0D70151
:108D7000FE0138969E01245F3F4F8D918193E2174B
:108D8000F307D9F710E346E0BE016B5F7F4F80EE3B
:108D900099E30F94BF1C99EF980F9230C8F48B8918
:108DA000893399F48A89893361F48989893321F473
:108DB00010922F2D80E03CC08F5F898B1A8B1B8B0C
:108DC000E2CF1B8B8F5F8A8BDECF8F5F8B8BDBCFEE
:108DD000882321F010922F2D80E02AC081E080931B
:108DE0002F2DBE01695F7F4FC6010F94C32A81E01A
:108DF0001FC0BF93AF939F938F9383EE90E29F9397
:108E00008F93CE0101969F938F930F94D92A8981D6
:108E1000898B8A818A8B8B818B8B80E38D838AE31C
:108E20008E83CDBFDEBFE114F10409F0A0CFAACF3D
:108E30006896CDBFDEBFDF91CF911F91FF90EF907D
:108E4000DF90CF90089580E00E9472E1882361F066
:108E50008250823030F58091302D882311F11092AC
:108E6000302D10922F2D08958091302D811119C031
:108E700081E08093302D8EE292E0E1E3FDE2DF01BC
:108E80009C011D9221503040E1F7BF0180E00F941A
:108E9000A11C8B3019F410922F2D089581E080933E
:108EA0002F2D08958AE00895CF93DF93CDB7DEB7D5
:108EB0006097CDBFDEBF009719F120E329832AE335
:108EC0002A832BE0E0E8F3E2DE01139601900D9295
:108ED0002A95E1F7613041F441E0BE016F5F7F4FB9
:108EE0000F94BF1C982F07C04AE0BE016F5F7F4FF1
:108EF0000F94BF1C982F81E0992319F080E001C0E6
:108F000080E06096CDBFDEBFDF91CF910895DF9204
:108F1000EF92FF920F931F93CF93DF93CDB7DEB7FE
:108F20006497CDBFDEBF8C0184E1EBE8F3E2DE01A4
:108F3000119601900D928A95E1F70115110509F43A
:108F400049C06115710509F447C080E389838AE34C
:108F50008A834115510559F0DA01FE0134969E01CC
:108F6000285F3F4F9D919193E217F307D9F77B015B
:108F70000F2EF0E3DF2EF02D46E0BE016F5F7F4F36
:108F8000C8010F94BF1C99EF980F9230A8F49F85E9
:108F9000993379F48E85893341F48D858933F1F0E5
:108FA0008F5F8D87DE86DF86E7CFDF868F5F8E87D8
:108FB000E3CF9F5F9F87E0CF811112C081E1FE0167
:108FC0003396D70101900D928A95E1F7F701118A46
:108FD00081E007C080E005C080E003C080E001C000
:108FE00080E06496CDBFDEBFDF91CF911F910F91DE
:108FF000FF90EF90DF900895DF92EF92FF920F9332
:109000001F93CF93DF93CDB7DEB76497CDBFDEBF9D
:109010008C0184E1EFE9F3E2DE01119601900D92FB
:109020008A95E1F70115110509F449C0611571052B
:1090300009F447C080E389838AE38A834115510597
:1090400059F0DA01FE0134969E01285F3F4F9D9151
:109050009193E217F307D9F77B010F2EF0E3DF2E90
:10906000F02D46E0BE016F5F7F4FC8010F94BF1C1B
:1090700099EF980F9230A8F49F85993379F48E85F3
:10908000893341F48D858933F1F08F5F8D87DE86DA
:10909000DF86E7CFDF868F5F8E87E3CF9F5F9F8777
:1090A000E0CF811112C081E1FE013396D70101901A
:1090B0000D928A95E1F7F701118A81E007C080E0FF
:1090C00005C080E003C080E001C080E06496CDBFB1
:1090D000DEBFDF91CF911F910F91FF90EF90DF9056
:1090E00008950F931F93CF93DF93CDB7DEB76097AB
:1090F000CDBFDEBF009761F18C0180E389838AE3F5
:109100008A838BE0E3EBF3E2DE01139601900D928C
:109110008A95E1F7613049F441E0BE016F5F7F4F0E
:10912000C8010F94BF1C982F0EC041E060E0CE0133
:1091300003960F942F234AE0BE016F5F7F4FC80153
:109140000F94BF1C982F81E0992319F080E001C093
:1091500080E06096CDBFDEBFDF91CF911F910F9170
:109160000895CF93DF93CDB7DEB76097CDBFDEBF55
:109170009BE0E3EBF3E2DE01119601900D929A95EC
:10918000E1F7813041F441E061E0CE0101960F94B6
:109190002F23982F07C041E060E0CE0101960F9485
:1091A0002F23982F81E0911180E06096CDBFDEBF24
:1091B000DF91CF910895009721F041E061E00D9497
:1091C0002F2308951F93CF93DF93CDB7DEB7649716
:1091D000CDBFDEBF009701F1162FBC0180E389836C
:1091E0008AE38A83CE0103960F94C32A113041F497
:1091F00041E061E0CE0101960F942F23982F07C024
:1092000041E060E0CE0101960F942F23982F81E07A
:10921000992319F080E001C080E06496CDBFDEBFE5
:10922000DF91CF911F910895EF92FF920F931F93BB
:10923000CF93DF93CDB7DEB76497CDBFDEBF6115A7
:10924000710589F1009789F18B017C0180E38983A5
:109250008AE38A83CE0103960F94C32A43E0BE01BA
:109260006F5F7F4FC7010F94BF1C873069F460E0C8
:10927000C801A8DF982F8823D9F043E0BE016F5FB3
:109280007F4FC7010F94BF1C811111C0F7014285A8
:10929000538564857585C7010F945D2191E088230E
:1092A00039F090E005C090E003C090E001C090E08C
:1092B000892F6496CDBFDEBFDF91CF911F910F91B3
:1092C000FF90EF900895CF93DF93CDB7DEB760970F
:1092D000CDBFDEBF0097C1F020E329832AE32A83B4
:1092E0002AE0EEEBF3E2DE01139601900D922A954F
:1092F000E1F741E0BE016F5F7F4F0F94BF1C91E02B
:10930000882319F090E001C090E0892F6096CDBFCE
:10931000DEBFDF91CF9108953F924F925F926F929F
:109320007F928F929F92AF92BF92CF92DF92EF92F5
:10933000FF920F931F93CF93DF93CDB7DEB7619763
:10934000CDBFDEBF6115710509F470C0009709F447
:109350006FC04115510509F46DC03FEF320F383031
:1093600008F06AC0322E7A018C01FB01138A41E0B9
:109370000F94BF1C811162C0F8014285538564853A
:109380007585483EF3E05F076105710508F458C034
:10939000413B84E058076105710508F053C0C32CB8
:1093A000D12C5601E6E0AE0EB11C25010B2C000CB1
:1093B000660877084419550966097709C8010F94AA
:1093C0005D21811141C0A50160E070E0CE010396EE
:1093D0000F94BC2A9E012F5F3F4FA501BE016D5F18
:1093E0007F4FC8010F94111EC8010F945221FE0136
:1093F000EC0DFD1D12868E010D5F1F4F812C912CEF
:109400005401A601B801C7010F94A62A892BF1F0D7
:10941000FFEF8F1A9F0AAF0ABF0A0F5F1F4F481452
:1094200059046A047B0468F780E011C080E00FC033
:1094300080E00DC080E00BC080E009C080E007C084
:1094400081E005C080E003C080E001C081E061965A
:10945000CDBFDEBFDF91CF911F910F91FF90EF90B5
:10946000DF90CF90BF90AF909F908F907F906F9044
:109470005F904F903F9008954F925F926F927F92CE
:10948000AF92BF92CF92DF92EF92FF920F931F9312
:10949000CF93DF93CDB7DEB76897CDBFDEBF68014E
:1094A00014E1ECE6F3E2DE01159601900D921A95B7
:1094B000E1F7009709F491C0C114D10409F48FC0F9
:1094C000EFEFEE0DE83008F08CC0860129013A017B
:1094D0005B016C01283E83E03807410551050CF41F
:1094E00082C01F921F921F9281E08F9383EE90E2C1
:1094F0009F938F93CE0101969F938F930F94D92AB8
:109500008981898B8A818A8B8B818B8B80E38D8388
:109510008AE38E83CDBFDEBFA114B10459F0D5011B
:10952000FE0138969E01245F3F4F8D918193E21793
:10953000F307D9F70F2EF0E3FF2EF02D46E0BE0122
:109540006B5F7F4F80EE99E30F94BF1C99EF980FEC
:10955000923090F52E2DA801BE016B5F7F4F80EEFB
:1095600099E3DADE882379F060E0C6012BDE8823F8
:1095700051F04AE0BE016B5F7F4F80EE99E30F949C
:10958000BF1C8823F9F09B89993399F48A89893320
:1095900061F48989893321F410922F2D80E042C033
:1095A0008F5F898BFA8AFB8AC9CFFB8A8F5F8A8B90
:1095B000C5CF9F5F9B8BC2CF882321F010922F2DA8
:1095C00080E030C081E080932F2DBE01695F7F4F26
:1095D000C6010F94C32A81E025C080E023C080E04B
:1095E00021C080E01FC07F926F925F922F9383EE25
:1095F00090E29F938F93CE0101969F938F930F9448
:10960000D92A8981898B8A818A8B8B818B8B80E394
:109610008D838AE38E83CDBFDEBFA114B10409F030
:109620007ECF88CF6896CDBFDEBFDF91CF911F91EF
:109630000F91FF90EF90DF90CF90BF90AF907F9011
:109640006F905F904F90089580915F2F08950895D7
:10965000089581E080935F2F089510925F2F089501
:10966000CF92DF92EF92FF920F931F936623B9F090
:1096700081111DC0C12CD12C760100E010E62AEE2C
:1096800030E040E06CE170E280EB98E00F94390943
:109690006CE170E280EB98E00F94830908C08111BF
:1096A00006C06CE170E280EB98E00F9499091F917D
:1096B0000F91FF90EF90DF90CF900895CF93DF93BD
:1096C0001F921F92CDB7DEB78091602F9091612FCE
:1096D000A091622FB091632F072E75E1B695A795E3
:1096E000979587957A95D1F7702D61E0B9DF87ED71
:1096F0008A8341E050E0BE016E5F7F4F80EB98E0CF
:109700000F94540941E050E0BE016F5F7F4F80EB42
:1097100098E00F946B0989818823A4F78091602FCA
:109720009091612FA091622FB091632F072E75E168
:10973000B695A795979587957A95D1F7702D60E0A6
:109740008FDF0F900F90DF91CF91089580EB98E01D
:109750000F9402091092642F81E008951F93CF9314
:10976000DF93CDB7DEB72C97CDBFDEBF6115710596
:1097700020E28207910508F0A1C0DC01CB018093B3
:10978000602F9093612FA093622FB093632F8091ED
:10979000642F811193DF1092642F8091602F90913C
:1097A000612FA091622FB091632F072E75E1B695BE
:1097B000A795979587957A95D1F7702D61E050DF41
:1097C00082ED8C8741E050E0BE01645F7F4F80EB0B
:1097D00098E00F9454098091602F9091612FA0918F
:1097E000622FB091632FAC01BD01032E39E0769555
:1097F0006795579547953A95D1F7302D032E3AE066
:10980000440F551F661F771F3A95D1F7302D917081
:10981000AA27BB27842B952BA62BB72B89839A834A
:10982000AB83BC838B818D8341E050E0BE016B5FD5
:109830007F4F80EB98E00F9454098A818E8341E03A
:1098400050E0BE016A5F7F4F80EB98E00F945409AF
:1098500089818F8341E050E0BE01695F7F4F80EBDB
:1098600098E00F94540915E5188741E050E0BE01D7
:10987000685F7F4F80EB98E00F945409198741E0AF
:1098800050E0BE01675F7F4F80EB98E00F94540972
:109890001A8741E050E0BE01665F7F4F80EB98E0A1
:1098A0000F9454091B8741E050E0BE01655F7F4F74
:1098B00080EB98E00F94540981E001C080E02C9681
:1098C000CDBFDEBFDF91CF911F910895052E59E0E6
:1098D000660F771F881F991F5A95D1F7502D611574
:1098E000710520E28207910510F438CF089580E0D9
:1098F00008958091602F9091612FA091622FB09177
:10990000632F0097A105B10569F00197A109B1097D
:10991000072E75E1B695A795979587957A95D1F716
:10992000702D01C080E060E09BDE1092642F0895EE
:10993000CF93DF93CDB7DEB72897CDBFDEBF6115DC
:10994000710520E28207910508F078C0DC01CB01A7
:109950008093602F9093612FA093622FB093632F19
:109960008091642F8111AADE1092642F8091602F64
:109970009091612FA091622FB091632F072E75E116
:10998000B695A795979587957A95D1F7702D61E053
:1099900067DE82E8888741E050E0BE01685F7F4F64
:1099A00080EB98E00F9454098091602F9091612F83
:1099B000A091622FB091632FAC01BD01032E39E05D
:1099C00076956795579547953A95D1F7302D032EA3
:1099D0003AE0440F551F661F771F3A95D1F7302D97
:1099E0009170AA27BB27842B952BA62BB72B898395
:1099F0009A83AB83BC838B818D8341E050E0BE01B1
:109A00006B5F7F4F80EB98E00F9454098A818E83BF
:109A100041E050E0BE016A5F7F4F80EB98E00F9419
:109A2000540989818F8341E050E0BE01695F7F4F17
:109A300080EB98E00F94540981E001C080E0289603
:109A4000CDBFDEBFDF91CF910895CF93DF931F92FB
:109A5000CDB7DEB78091602F9091612FA091622FDA
:109A6000B091632FAC01BD01517066277727452B5C
:109A7000462B472B31F1198241E050E0BE016F5F68
:109A80007F4F80EB98E00F9454098091602F909164
:109A9000612FA091622FB091632F0196A11DB11D7E
:109AA0008093602F9093612FA093622FB093632FC8
:109AB000AC01BD01517066277727452B462B472BFC
:109AC000D1F60097A105B10569F00197A109B10987
:109AD000072E75E1B695A795979587957A95D1F755
:109AE000702D01C080E060E0BBDD81E08093642FD9
:109AF0000F90DF91CF9108950F931F93CF93DF9332
:109B00001F92CDB7DEB78091642F8823B1F01092F9
:109B1000642F8091602F9091612FA091622FB0915E
:109B2000632FBC01CD01052E59E096958795779559
:109B300067955A95D1F7502DC9DE41E050E0BE013E
:109B40006F5F7F4F80EB98E00F946B098091602FDF
:109B50009091612FA091622FB091632FAC01BD0154
:109B60004F5F5F4F6F4F7F4F4093602F5093612F38
:109B70006093622F7093632F8A019B0111702227DB
:109B80003327012B022B032BA1F4452B462B472B0C
:109B900051F0072E75E1B695A795979587957A951B
:109BA000D1F7702D01C080E060E05ADD81E0809344
:109BB000642F89810F90DF91CF911F910F910895AC
:109BC0000F931F93CF93DF931F92CDB7DEB7182F5C
:109BD0008091642F882349F06091602F7091612FEC
:109BE0008091622F9091632FA3DE198341E050E0B2
:109BF000BE016F5F7F4F80EB98E00F945409809116
:109C0000602F9091612FA091622FB091632FAC01D2
:109C1000BD014F5F5F4F6F4F7F4F4093602F509359
:109C2000612F6093622F7093632F8A019B011170E3
:109C300022273327012B022B032BA1F4452B462B84
:109C4000472B51F0072E75E1B695A7959795879507
:109C50007A95D1F7702D01C080E060E001DD81E0F0
:109C60008093642F81E00F90DF91CF911F910F912E
:109C70000895CF93DF931F921F92CDB7DEB78091E7
:109C8000642F882309F440C08091602F9091612F48
:109C9000A091622FB091632F072E75E1B695A7951D
:109CA000979587957A95D1F7702D61E0D9DC87ED8E
:109CB0008A8341E050E0BE016E5F7F4F80EB98E009
:109CC0000F94540941E050E0BE016F5F7F4F80EB7D
:109CD00098E00F946B098091602F9091612FA09173
:109CE000622FB091632F072E75E1B695A7959795D2
:109CF00087957A95D1F7702D60E0B2DC89818095E7
:109D0000881F8827881F01C080E00F900F90DF9187
:109D1000CF910895CF93DF93EC01803C28E0920728
:109D200029F468E083E00F94830810C0803C29E0A8
:109D3000920729F468E084E00F94830807C0803C10
:109D40009A4021F468E085E00F948308888180615F
:109D50008883DF91CF910895EF92FF920F931F9325
:109D6000CF937C01C42FB901A80100E010E62AEED0
:109D700030E00E94B658882344F0F7018081CC0F70
:109D8000CC0FCC70837FC82BC083CF911F910F91D4
:109D9000FF90EF90089580E0089591E0811101C057
:109DA00090E09093003A81E08093442008950F93CF
:109DB0001F930BEA10E52FE130E048EA5FE261E033
:109DC00082E00E943969811105C067ED7EE482E07E
:109DD0000E94896A1F910F910895CF93DF9310928B
:109DE0008B2F10928C2F0F94AF09811104C0109209
:109DF000A42FD0E012C081508093A42F2ADCD82F4A
:109E0000882359F0C0E060E08C2F0F94C509CF5F24
:109E10008091A42F8C17B8F7CADF8D2FDF91CF91D7
:109E20000895C5CF08950F931F9301E11FE42DE01E
:109E300030E048E450E260E081E80E943969811135
:109E400005C063E17FE481E80E94896A1F910F9158
:109E5000089580918C2F882341F082E00E94626AED
:109E600069E27FE482E00C94896A089580918C2FE6
:109E7000882341F081E80E94626A66E37FE481E81A
:109E80000C94896A08958091502090915120A0915E
:109E90005220B0915320892B8A2B8B2B59F0809123
:109EA000B42F882324F481E80E94626A03C082E010
:109EB0000E94626A8091AC2F9091AD2FA091AE2F3D
:109EC000B091AF2F80934C2090934D20A0934E20C3
:109ED000B0934F20A8CF0895E0E9FFE282E1DF01CF
:109EE0001D928A95E9F780EF80838AE08783089541
:109EF000DF92EF92FF920F931F93CF93DF93D82EB1
:109F0000C62FD72F122F032FF42EE52EE5DF81E089
:109F100080935420E0E9FFE2D282E382F482058359
:109F20001683D487C587DF91CF911F910F91FF9042
:109F3000EF90DF90089520E030E0A90160E074E246
:109F400085E0D6CF08950F931F932091B42F422719
:109F50006CF00091502010915120209152203091AE
:109F60005320061717072807390720F4E4DF8BDF93
:109F700080E001C081E01F910F91089520E030E062
:109F8000A90160E070E084E0B3CF08950F931F93C0
:109F9000262F30E00CEE1FE4AC0161E081E80E9466
:109FA0003969811102C0EADF6EDF1F910F910895B8
:109FB00020E030E0A90160E078E286E099CF0895E2
:109FC00020E030E0A90160E07AE382E091CF0895DB
:109FD00083DF109254200895CF93DF93811111C035
:109FE000EB01F6DFE8E4F0E280859185A285B38598
:109FF0008C1B9D0BA109B10980879187A287B3872C
:10A0000042DFDF91CF9108951F93CF93DF93D82F35
:10A0100084E1E0E7FFE2DF011D928A95E9F7DD23A5
:10A0200031F09091BF2FE8E7FFE218E005C0909172
:10A03000BB2FE4E7FFE214E08091B92F8F738C31DE
:10A0400011F08F3339F48CE180838AE0818385E0DD
:10A050008383145FC12F911708F4C92F8C2F90E0D0
:10A06000A0E0B0E040E8BC01CD016DDF882309F13C
:10A070008091B52F0F94CC09811102C020E001C05E
:10A0800020E8DD2361F0E0E7FFE2812F90E0029716
:10A0900098278927982780839183238306C0E0E748
:10A0A000FFE28FEF810F808322836C2F80E79FE296
:10A0B0006DDFDF91CF911F910895CF93C82F81114C
:10A0C0000FC08091B52F0F94CC09882349F020E070
:10A0D00030E0A90160E077E287E00ADFD4DE39C032
:10A0E000A6E8BFE2E8EAFFE2818913968C93139712
:10A0F000828912968C931297838911968C9311976B
:10A1000084898C93A4E8BFE2868911968C93119779
:10A1100087898C936091842F7091852FCB01A0E06B
:10A12000B0E0BC01CD01052E59E0660F771F881FF6
:10A13000991F5A95D1F7502DC11102C040E001C0BE
:10A1400040E801DF882329F0C0938A2F81E08093C3
:10A150008B2FCF9108950F931F93CF93DF9381118E
:10A1600032C16F31710569F48091A82F9091A92FA8
:10A17000A091AA2FB091AB2F85359345A244B3444B
:10A1800031F081E080938C2F64DE70DE1CC1E8EA40
:10A19000FFE295859F7095878091A42F891718F409
:10A1A000CADE71DE10C1E8EAFFE2408551856285B2
:10A1B00073854093502050935120609352207093A8
:10A1C0005320478550E04B35510508F0EEC0FA01A9
:10A1D0008827EF5BFE4F8F4F0D94D128C091BB2F86
:10A1E000C33108F0C2E18C2F90E0A0E0B0E040E87D
:10A1F000BC01CD01A8DE882309F4E5C06C2F80E9FD
:10A200009FE2C4DEE0C0C091BB2FC53208F0C4E2BB
:10A210008C2F90E0A0E0B0E040E8BC01CD0193DEDF
:10A22000882309F4D0C08091B82F837021F4D09195
:10A23000B92FDD2319F07FDE26DEC5C08091B52F52
:10A240000F94D3098111D0E800E210E2F801D18324
:10A250008091B52F0F94DA0920E1FC013196A0E33B
:10A26000B0E201900D922A95E1F7F80180898823E8
:10A2700009F4A4C0823209F4A3C0E1E3F0E281E072
:10A280009191992309F49DC0923209F49AC08F5F8D
:10A290008031B1F708C0E82FF0E0E05EFF4D908B11
:10A2A0008F5F8031C1F76C2F80E290E26FDE8BC050
:10A2B00080E0AADE88C081E0A7DE85C0892F0F94E8
:10A2C000B109823039F0833019F0811105C006C020
:10A2D0006FDE05C075DE03C051DE01C079DED3DD5F
:10A2E00072C040E868E070E080E090E02CDE8823F7
:10A2F00009F469C068E67FE28091B52F0F94B80930
:10A30000823041F0833019F0811107C009C050DE5E
:10A31000BADD59C055DEB7DD56C030DEB4DD53C0FE
:10A32000E8E6FFE280E090E0A2E0B0E0848395837D
:10A33000A683B78380819181A281B3815A2F4B2F4D
:10A3400060E070E0982789279827A0E0B0E0DC0162
:10A3500099278827842B952BA62BB72B8083918355
:10A36000A283B38368E0CF0111DE2DC08091BB2FA3
:10A3700081FF06C08095682F6170892F0F94C509F1
:10A3800027DE81DD20C08091BB2F811102C020DE3D
:10A3900001C0D1DD78DD17C01BDE75DD14C081E0A2
:10A3A0008CDE11C080E089DE0EC020E030E0A90123
:10A3B00060E070E285E09CDD66DD05C080E001C004
:10A3C00080E090E268CFDF91CF911F910F910895C7
:10A3D00010928B2F42C908958091093A8823F4F492
:10A3E00080768032D9F580910A3A8E3FC9F5809106
:10A3F0000F3A9091103A0197A9F580910B3A9091FC
:10A400000C3A892B89F5E9E0FAE384EA9FE2808738
:10A41000918781E090E082879387089580768032EB
:10A4200029F580910A3A8F3F19F580910F3A909162
:10A43000103A892BF9F480910B3A90910C3A892BC0
:10A44000D9F410928C2F10928B2F82E00E94F76922
:10A4500081E80E94F769ABDC81E0089580E008950F
:10A4600080E0089580E0089580E0089580E00895F8
:10A4700080E0089580E0089580E00895CF93C09132
:10A480008B2FCC23A9F110928B2F80918A2F8823B8
:10A4900089F02091842F3091852F4091862F509103
:10A4A000872F6091882F7091892F8091B52F0F94FD
:10A4B000E20910C02091842F3091852F4091862F82
:10A4C0005091872F6091882F7091892F8091B52F9F
:10A4D0000F94060A823041F0833021F0811106C0CA
:10A4E00077DD05C065DD03C06BDD01C047DDCBDC7A
:10A4F0008C2FCF910895EF92FF920F931F93CF93DC
:10A50000DF93982F80914420882309F448C010924B
:10A5100044202115310511F0890102C00DEC1EE423
:10A52000911102C082E001C081E8E9017A01AB012A
:10A53000970160E00E943969811104C091E0909315
:10A5400044202DC0CD2BD9F4809144208823E1F301
:10A550008091003A811122C0E8E4F0E28085918583
:10A56000A285B3858E199F09A109B10980879187BA
:10A57000A287B3879091003A81E0892710C0E8E470
:10A58000F0E240855185628573854E195F09610946
:10A590007109408751876287738701C080E0DF912E
:10A5A000CF911F910F91FF90EF900895E091CD2FE3
:10A5B000F091CE2F0190F081E02D228133812E0F7A
:10A5C0003F1FFC014081E40FF11DE217F307A0F4E7
:10A5D00081818430A1F0861306C014C0818184304B
:10A5E000A1F08617A9F08081E80FF11DE217F307AB
:10A5F000A8F380E090E0089580E090E0089580E086
:10A6000090E008958E2F9F2F089580E090E00895A8
:10A610008E2F9F2F089580910B3A8F770C9454685A
:10A6200008959091CF2F992381F1E091CD2FF09152
:10A63000CE2F0190F081E02D9481891740F5E093B1
:10A64000CB2FF093CC2F228133812E0F3F1FE217A7
:10A65000F307F8F49181943061F49281891309C071
:10A660009381961306C0E093CB2FF093CC2F81E01B
:10A6700008959081E90FF11DE217F30758F3E09375
:10A68000CB2FF093CC2F80E0089580E0089580E0F8
:10A69000089580E00895EF92FF921F93CF93DF9388
:10A6A000C82F60E0BEDF182F882381F1A091CD2F45
:10A6B000B091CE2FEC2FF0E0EE0FFF1F12968D9190
:10A6C0009C911397E80FF91FE080F180D70116964F
:10A6D000ED91FC9117971995682F8C2FA2DF182FF9
:10A6E0008823A1F0C091CB2FD091CC2F65E0CE0173
:10A6F0005DDFEC01892B21F08A810E94466AF6CF4A
:10A70000D7011296ED91FC9113971995812FDF9146
:10A71000CF911F91FF90EF9008951F93CF93DF93F8
:10A72000182F7FDF882341F1C091CB2FD091CC2F00
:10A7300065E0CE013BDFEC01892B49F04C815D8166
:10A740006B818A810E9461688111F2CF15C0A0914E
:10A75000CD2FB091CE2FE12FF0E0EE0FFF1F12961C
:10A760008D919C911397E80FF91F0190F081E02DD6
:10A770000190F081E02D1995DF91CF911F910895FF
:10A780000C94EC670895CF938091CF2F8823C1F06C
:10A79000E091CD2FF091CE2F0190F081E02D8481BA
:10A7A000882371F0C0E08C2F76DFCF5FE091CD2F52
:10A7B000F091CE2F0190F081E02D8481C81798F39D
:10A7C0001092CF2F81E090E08093D02F9093D12FE3
:10A7D000CF9108950E94B867D6CF0895CF93809106
:10A7E000CF2F882349F1A091CD2FB091CE2FED919D
:10A7F000FC91119784818823F9F0C0E0EC2FF0E000
:10A80000EE0FFF1F12968D919C911397E80FF91F81
:10A810000190F081E02D0084F185E02D309709F062
:10A820001995CF5FA091CD2FB091CE2FED91FC91D6
:10A8300011978481C81710F3CF9108950F931F9338
:10A84000CF93DF93E9E0FAE3128613861486158628
:10A8500016861786808188230CF060C220910F3AFB
:10A860003091103A2115310509F05DC24FC28F7148
:10A8700009F097C090910A3A963081F0983009F427
:10A8800085C091118EC02230310509F0FBC162E014
:10A8900070E080ED9FE20E945A684EC280910B3AB0
:10A8A00090910C3A292F33272230310589F023303B
:10A8B000310579F12130310509F0A6C1809162207E
:10A8C00090916320DC016C9170E00E945A684FC047
:10A8D000E0916220F09163202189821708F0D2C1B3
:10A8E0009927880F991F880F991FE0916420F09194
:10A8F0006520E80FF91F80819181FC0162817381DD
:10A900000E945A68E091113AF091123A82E08183F4
:10A910002EC099278130910599F058F08230910529
:10A9200009F406C2039709F078C13CE0E8ECF3E2D1
:10A930000AC064E070E088EC90E20E945A6817C098
:10A94000EEEBF0E239E0A2EAB0E220E0819190E0A3
:10A950008D939D932F5F2317C8F3632F660F6E5F50
:10A960006093A02070E080EA90E20E945A68E9E0DB
:10A97000FAE386819781228533858217930708F051
:10A98000DBC18093133A9093143AD6C1213031053C
:10A9900009F078C161E070E08FEC9FE20E945A6894
:10A9A000CBC18130E9F590910A3A9A30C9F521304E
:10A9B000310509F037C18091CF2F882309F432C1C6
:10A9C000C0910D3AD0910E3A0091CD2F1091CE2F1B
:10A9D000D801ED91FC918481C81708F023C160E093
:10A9E0008C2F1FDE882309F418C1CE019927880F08
:10A9F000991FD8011296ED91FC911397E80FF91F5A
:10AA00000190F081E02D86819781FC01199580935A
:10AA1000CA2F61E070E08AEC9FE20E945A688CC104
:10AA2000823009F0FAC080910A3A8111EFC02230D9
:10AA3000310509F027C180910D3A0E94E96890E044
:10AA40008093C82F9093C92F62E070E088EC9FE25A
:10AA50000E945A6871C18F7109F084C090910A3ABE
:10AA6000933009F4D5C018F49130A1F07BC0953033
:10AA700019F0993039F176C080910F3A9091103ADF
:10AA8000892B09F0FFC08BE093E58093153A9093F2
:10AA9000163A52C180910F3A9091103A892B09F0E1
:10AAA000F1C080910B3A90910C3A019709F0EAC0FD
:10AAB0008091D02F9091D12F8D7F8093D02F909324
:10AAC000D12F3AC180910F3A9091103A892B09F019
:10AAD000D9C00E945768882309F49FC020910B3A7F
:10AAE00030910C3A3327E0916220F0916320818904
:10AAF00090E08217930708F490C045DE80910B3AEE
:10AB000090910C3A8093CF2F882309F415C199278F
:10AB10008150904C880F991F880F991FE0916420F5
:10AB2000F0916520E80FF91FE093CD2FF093CE2F21
:10AB30000190F081E02D8481882309F4FDC0C0E0FC
:10AB400060E08C2FEADD882309F467C0CF5FE091D5
:10AB5000CD2FF091CE2F0190F081E02D8481C81788
:10AB600078F3EAC08130E9F490910A3A9B30C9F455
:10AB700080910F3A9091103A892B09F053C080913F
:10AB8000CF2F882309F44EC0E9E0FAE3C481D281D3
:10AB90008C2F81DD882309F440C06D2F8C2FBDDD03
:10ABA0003AC08230D1F580910A3A813019F0833071
:10ABB000A1F030C080910F3A9091103A892B09F0A2
:10ABC00061C080910B3A90910C3A892B09F05AC0E0
:10ABD00080910D3A0E9404691EC080910F3A9091B5
:10ABE000103A892B09F04EC080910B3A90910C3AA3
:10ABF000892B09F047C0C9E0DAE38C810E94F7692C
:10AC00008C810E94626A07C080E005C080E003C0BA
:10AC100080E001C080E0811190C08091093A8F717D
:10AC2000813081F58091CF2F882309F471C0009184
:10AC30000D3A10910E3AC091CD2FD091CE2FE881D0
:10AC4000F9818481081708F065C060E0802FE9DC95
:10AC50008823C1F0F801FF27CF01880F991FEA81EF
:10AC6000FB81E80FF91FC081D181EE81FF81199529
:10AC7000682F802FD6DC882329F0EC81FD8119957F
:10AC800081115BC08091093A8F71823009F044C014
:10AC90008091CF2F8823B1F1A091CD2FB091CE2FED
:10ACA000ED91FC9111978481882371F1C0E0EC2F24
:10ACB000F0E0EE0FFF1F12968D919C911397E80F15
:10ACC000F91F00811181D8011696ED91FC9117971B
:10ACD0001995682F8C2FA5DC882379F1D80114965B
:10ACE000ED91FC9115971995811127C0CF5FA09127
:10ACF000CD2FB091CE2FED91FC9111979481C91772
:10AD0000B0F21BC080E019C080E017C080E015C021
:10AD100080E013C080E011C080E00FC0982F9076D3
:10AD200009F07BCF98CE982F907609F076CF9FCD03
:10AD300033E0EAEBF0E207CE81E0DF91CF911F91A3
:10AD40000F9108958038910558F1672B21F4873CC5
:10AD5000910571F41CC08F3F910509F0F8F49C0136
:10AD6000220F331FF901EB56F94D8081918108952F
:10AD7000E7E9F7E221E030E041915191841795072E
:10AD800041F02F5F3F4F20383105B1F702C020E07E
:10AD900030E020583F4FC9019927089580E090E0A6
:10ADA00008958136910589F0E7EBF5E240E050E047
:10ADB0004F5F5F4F219131912115310591F0281797
:10ADC0003907B1F7892B19F40AC040E050E0440F6D
:10ADD000551FFA01EB52FC4D80819181089580E06E
:10ADE00090E0089543E050E060E880E096E00F9442
:10ADF000DB0843E050E064E080E296E00F94DB087B
:10AE000043E050E062E080E296E00F94DB0840E02F
:10AE100058E160E280EA96E00F94DB0841E050E000
:10AE200062E080EA96E00F94DB0843E050E060E1E6
:10AE300080E896E00F94DB0843E050E060E180E4B6
:10AE400096E00F94DB0841E050E061E080E496E09A
:10AE50000F94DB0841E050E062E080E496E00F945C
:10AE6000DB0841E050E060E280E696E00F94DB080A
:10AE700041E050E062E080E096E00F94DB0841E0C2
:10AE800050E062E080E896E00F94DB0843E050E099
:10AE900062E080E696E00F94DB0840E050E061E07D
:10AEA00080EA96E00F94DB0840E050E061E080E04B
:10AEB00096E00F94DB0840E050E068E080E096E028
:10AEC0000F94DB0841E050E060E480E096E00F94EE
:10AED000DB0840E058E161E080E896E00F94DB0891
:10AEE00040E050E061E080E096E00F94DB0840E055
:10AEF00050E060E280E096E00F94DB0840E050E034
:10AF000064E080E096E00F94DB0840E050E061E010
:10AF100080EA96E00F94DB0843E050E060E880E4CC
:10AF200096E00F94DB0843E050E060E280E496E0B6
:10AF30000F94DB0840E050E060E480E496E00F947A
:10AF4000DB0841E050E060E880E896E00F94DB0821
:10AF500041E050E060E280E896E00F94DB0840E0DA
:10AF600050E060E480E896E00F94DB0843E050E0B6
:10AF700068E080E496E00F94DB0840E050E064E095
:10AF800080E496E00F94DB0843E050E068E080E660
:10AF900096E00F94DB0840E050E064E080E696E045
:10AFA0000F94DB0843E050E068E080E896E00F94FF
:10AFB000DB0840E050E064E080E896E00F94DB08B6
:10AFC00043E050E068E080EA96E00F94DB0840E060
:10AFD00050E064E080EA96E00F94DB0840E058E13E
:10AFE00060E480EA96E00F94DB0840E058E160E11D
:10AFF00080E696E00F94DB0840E058E161E080E2F3
:10B0000096E00F94DB0843E050E060E880E496E0CF
:10B010000F94DB0843E050E060E280E496E00F9498
:10B02000DB0840E050E060E480E496E00F94DB0849
:10B0300043E050E060E880EA96E00D94DB08089574
:10B040001F920F920FB60F9211240BB60F928F938F
:10B050009F93EF93FF93E1E0FAE380819181019662
:10B0600080839183FF91EF919F918F910F900BBE01
:10B070000F900FBE0F901F9018951F920F920FB652
:10B080000F9211240BB60F92CF92DF92EF92FF92A4
:10B090000F931F932F933F934F935F936F937F93E0
:10B0A0008F939F93AF93BF93EF93FF93E1E0FAE306
:10B0B000808191812281338182179307F0F121E011
:10B0C00020930204E091073AF091083A3097A9F1F1
:10B0D0006091080470910904A0E0B0E0DC019927B8
:10B0E0008827AB0160E070E08C019D01042B152BDB
:10B0F000262B372BC901B801A1E0BAE312960D91B6
:10B100001C91139720E030E0980111270027149636
:10B11000CD90DC901597E12CF12C0C291D292E29BE
:10B120003F29061717072807390730F0C901B8016A
:10B130006F5F7F4F8F4F9F4F1995FF91EF91BF9199
:10B14000AF919F918F917F916F915F914F913F91BF
:10B150002F911F910F91FF90EF90DF90CF900F9064
:10B160000BBE0F900FBE0F901F901895CF92DF92DD
:10B17000EF92FF920F931F93CF93DF93EC016A013D
:10B180007B01DB01CA010197A109B109BC01CD0115
:10B19000600F711F821F931FA70196010F949328C0
:10B1A0002138310541055105F8F4213460F421328C
:10B1B00060F4213160F4293060F4253060F42330EC
:10B1C00060F490E80BC093E009C092E007C092E8F9
:10B1D00005C091E003C091E801C090E088818C77C0
:10B1E000892B888381E001C08FEFDF91CF911F9180
:10B1F0000F91FF90EF90DF90CF9008951F920F92E4
:10B200000FB60F9211240BB60F922F933F934F93CB
:10B210005F936F937F938F939F93AF93BF93EF93BE
:10B22000FF93E0911830F0911930309709F019959B
:10B23000FF91EF91BF91AF919F918F917F916F910E
:10B240005F914F913F912F910F900BBE0F900FBECA
:10B250000F901F9018951F920F920FB60F92112406
:10B260000BB60F922F933F934F935F936F937F9300
:10B270008F939F93AF93BF93EF93FF93E09116301B
:10B28000F0911730309709F01995FF91EF91BF9128
:10B29000AF919F918F917F916F915F914F913F916E
:10B2A0002F910F900BBE0F900FBE0F901F9018950F
:10B2B0001F920F920FB60F9211240BB60F922F937D
:10B2C0003F934F935F936F937F938F939F93AF932E
:10B2D000BF93EF93FF93E0911430F09115303097C6
:10B2E00009F01995FF91EF91BF91AF919F918F91C7
:10B2F0007F916F915F914F913F912F910F900BBE76
:10B300000F900FBE0F901F9018951F920F920FB6BF
:10B310000F9211240BB60F922F933F934F935F938D
:10B320006F937F938F939F93AF93BF93EF93FF930D
:10B33000E0911230F0911330309709F01995FF9198
:10B34000EF91BF91AF919F918F917F916F915F919D
:10B350004F913F912F910F900BBE0F900FBE0F900A
:10B360001F9018951F920F920FB60F9211240BB6D3
:10B370000F922F933F934F935F936F937F938F938E
:10B380009F93AF93BF93EF93FF93E0911030F091B1
:10B390001130309709F01995FF91EF91BF91AF915E
:10B3A0009F918F917F916F915F914F913F912F91DD
:10B3B0000F900BBE0F900FBE0F901F9018951F920D
:10B3C0000F920FB60F9211240BB60F922F933F934B
:10B3D0004F935F936F937F938F939F93AF93BF939D
:10B3E000EF93FF93E0910E30F0910F30309709F01A
:10B3F0001995FF91EF91BF91AF919F918F917F919F
:10B400006F915F914F913F912F910F900BBE0F90D5
:10B410000FBE0F901F9018951F920F920FB60F92AC
:10B4200011240BB60F922F933F934F935F936F931B
:10B430007F938F939F93AF93BF93EF93FF93E0918D
:10B440000C30F0910D30309709F01995FF91EF9184
:10B45000BF91AF919F918F917F916F915F914F912C
:10B460003F912F910F900BBE0F900FBE0F901F902A
:10B4700018951F920F920FB60F9211240BB60F92D0
:10B480002F933F934F935F936F937F938F939F93EC
:10B49000AF93BF93EF93FF93E0910A30F0910B309D
:10B4A000309709F01995FF91EF91BF91AF919F915E
:10B4B0008F917F916F915F914F913F912F910F905D
:10B4C0000BBE0F900FBE0F901F9018951F920F92FA
:10B4D0000FB60F9211240BB60F922F933F934F93F9
:10B4E0005F936F937F938F939F93AF93BF93EF93EC
:10B4F000FF93E0910830F0910930309709F01995E9
:10B50000FF91EF91BF91AF919F918F917F916F913B
:10B510005F914F913F912F910F900BBE0F900FBEF7
:10B520000F901F9018951F920F920FB60F92112433
:10B530000BB60F922F933F934F935F936F937F932D
:10B540008F939F93AF93BF93EF93FF93E091063058
:10B55000F0910730309709F01995FF91EF91BF9165
:10B56000AF919F918F917F916F915F914F913F919B
:10B570002F910F900BBE0F900FBE0F901F9018953C
:10B580001F920F920FB60F9211240BB60F922F93AA
:10B590003F934F935F936F937F938F939F93AF935B
:10B5A000BF93EF93FF93E0910430F0910530309713
:10B5B00009F01995FF91EF91BF91AF919F918F91F4
:10B5C0007F916F915F914F913F912F910F900BBEA3
:10B5D0000F900FBE0F901F9018951F920F920FB6ED
:10B5E0000F9211240BB60F922F933F934F935F93BB
:10B5F0006F937F938F939F93AF93BF93EF93FF933B
:10B60000E0910230F0910330309709F01995FF91E5
:10B61000EF91BF91AF919F918F917F916F915F91CA
:10B620004F913F912F910F900BBE0F900FBE0F9037
:10B630001F9018951F920F920FB60F9211240BB600
:10B640000F922F933F934F935F936F937F938F93BB
:10B650009F93AF93BF93EF93FF93E0910030F091EE
:10B660000130309709F01995FF91EF91BF91AF919B
:10B670009F918F917F916F915F914F913F912F910A
:10B680000F900BBE0F900FBE0F901F9018951F923A
:10B690000F920FB60F9211240BB60F922F933F9378
:10B6A0004F935F936F937F938F939F93AF93BF93CA
:10B6B000EF93FF93E091FE2FF091FF2F309709F069
:10B6C0001995FF91EF91BF91AF919F918F917F91CC
:10B6D0006F915F914F913F912F910F900BBE0F9003
:10B6E0000FBE0F901F9018951F920F920FB60F92DA
:10B6F00011240BB60F922F933F934F935F936F9349
:10B700007F938F939F93AF93BF93EF93FF93E091BA
:10B71000FC2FF091FD2F309709F01995FF91EF91D3
:10B72000BF91AF919F918F917F916F915F914F9159
:10B730003F912F910F900BBE0F900FBE0F901F9057
:10B7400018951F920F920FB60F9211240BB60F92FD
:10B750002F933F934F935F936F937F938F939F9319
:10B76000AF93BF93EF93FF93E091FA2FF091FB2FEC
:10B77000309709F01995FF91EF91BF91AF919F918B
:10B780008F917F916F915F914F913F912F910F908A
:10B790000BBE0F900FBE0F901F9018951F920F9227
:10B7A0000FB60F9211240BB60F922F933F934F9326
:10B7B0005F936F937F938F939F93AF93BF93EF9319
:10B7C000FF93E091F82FF091F92F309709F0199538
:10B7D000FF91EF91BF91AF919F918F917F916F9169
:10B7E0005F914F913F912F910F900BBE0F900FBE25
:10B7F0000F901F9018951F920F920FB60F92112461
:10B800000BB60F922F933F934F935F936F937F935A
:10B810008F939F93AF93BF93EF93FF93E091F62F96
:10B82000F091F72F309709F01995FF91EF91BF91A3
:10B83000AF919F918F917F916F915F914F913F91C8
:10B840002F910F900BBE0F900FBE0F901F90189569
:10B850001F920F920FB60F9211240BB60F922F93D7
:10B860003F934F935F936F937F938F939F93AF9388
:10B87000BF93EF93FF93E091F42FF091F52F309762
:10B8800009F01995FF91EF91BF91AF919F918F9121
:10B890007F916F915F914F913F912F910F900BBED0
:10B8A0000F900FBE0F901F9018951F920F920FB61A
:10B8B0000F9211240BB60F922F933F934F935F93E8
:10B8C0006F937F938F939F93AF93BF93EF93FF9368
:10B8D000E091F22FF091F32F309709F01995FF9135
:10B8E000EF91BF91AF919F918F917F916F915F91F8
:10B8F0004F913F912F910F900BBE0F900FBE0F9065
:10B900001F9018951F920F920FB60F9211240BB62D
:10B910000F922F933F934F935F936F937F938F93E8
:10B920009F93AF93BF93EF93FF93E091F02FF0912C
:10B93000F12F309709F01995FF91EF91BF91AF91D9
:10B940009F918F917F916F915F914F913F912F9137
:10B950000F900BBE0F900FBE0F901F9018951F9267
:10B960000F920FB60F9211240BB60F922F933F93A5
:10B970004F935F936F937F938F939F93AF93BF93F7
:10B98000EF93FF93E091EE2FF091EF2F309709F0B6
:10B990001995FF91EF91BF91AF919F918F917F91F9
:10B9A0006F915F914F913F912F910F900BBE0F9030
:10B9B0000FBE0F901F9018951F920F920FB60F9207
:10B9C00011240BB60F922F933F934F935F936F9376
:10B9D0007F938F939F93AF93BF93EF93FF93E091E8
:10B9E000EC2FF091ED2F309709F01995FF91EF9121
:10B9F000BF91AF919F918F917F916F915F914F9187
:10BA00003F912F910F900BBE0F900FBE0F901F9084
:10BA100018951F920F920FB60F9211240BB60F922A
:10BA20002F933F934F935F936F937F938F939F9346
:10BA3000AF93BF93EF93FF93E091EA2FF091EB2F39
:10BA4000309709F01995FF91EF91BF91AF919F91B8
:10BA50008F917F916F915F914F913F912F910F90B7
:10BA60000BBE0F900FBE0F901F9018951F920F9254
:10BA70000FB60F9211240BB60F922F933F934F9353
:10BA80005F936F937F938F939F93AF93BF93EF9346
:10BA9000FF93E091E82FF091E92F309709F0199585
:10BAA000FF91EF91BF91AF919F918F917F916F9196
:10BAB0005F914F913F912F910F900BBE0F900FBE52
:10BAC0000F901F9018951F920F920FB60F9211248E
:10BAD0000BB60F922F933F934F935F936F937F9388
:10BAE0008F939F93AF93BF93EF93FF93E091E62FD4
:10BAF000F091E72F309709F01995FF91EF91BF91E1
:10BB0000AF919F918F917F916F915F914F913F91F5
:10BB10002F910F900BBE0F900FBE0F901F90189596
:10BB20001F920F920FB60F9211240BB60F922F9304
:10BB30003F934F935F936F937F938F939F93AF93B5
:10BB4000BF93EF93FF93E091E42FF091E52F3097AF
:10BB500009F01995FF91EF91BF91AF919F918F914E
:10BB60007F916F915F914F913F912F910F900BBEFD
:10BB70000F900FBE0F901F9018951F920F920FB647
:10BB80000F9211240BB60F922F933F934F935F9315
:10BB90006F937F938F939F93AF93BF93EF93FF9395
:10BBA000E091E22FF091E32F309709F01995FF9182
:10BBB000EF91BF91AF919F918F917F916F915F9125
:10BBC0004F913F912F910F900BBE0F900FBE0F9092
:10BBD0001F9018951F920F920FB60F9211240BB65B
:10BBE0000F922F933F934F935F936F937F938F9316
:10BBF0009F93AF93BF93EF93FF93E091E02FF0916A
:10BC0000E12F309709F01995FF91EF91BF91AF9116
:10BC10009F918F917F916F915F914F913F912F9164
:10BC20000F900BBE0F900FBE0F901F9018951F9294
:10BC30000F920FB60F9211240BB60F922F933F93D2
:10BC40004F935F936F937F938F939F93AF93BF9324
:10BC5000EF93FF93E091DE2FF091DF2F309709F003
:10BC60001995FF91EF91BF91AF919F918F917F9126
:10BC70006F915F914F913F912F910F900BBE0F905D
:10BC80000FBE0F901F9018951F920F920FB60F9234
:10BC900011240BB60F922F933F934F935F936F93A3
:10BCA0007F938F939F93AF93BF93EF93FF93E09115
:10BCB000DC2FF091DD2F309709F01995FF91EF916E
:10BCC000BF91AF919F918F917F916F915F914F91B4
:10BCD0003F912F910F900BBE0F900FBE0F901F90B2
:10BCE00018951F920F920FB60F9211240BB60F9258
:10BCF0002F933F934F935F936F937F938F939F9374
:10BD0000AF93BF93EF93FF93E091DA2FF091DB2F86
:10BD1000309709F01995FF91EF91BF91AF919F91E5
:10BD20008F917F916F915F914F913F912F910F90E4
:10BD30000BBE0F900FBE0F901F9018951F920F9281
:10BD40000FB60F9211240BB60F922F933F934F9380
:10BD50005F936F937F938F939F93AF93BF93EF9373
:10BD6000FF93E091D82FF091D92F309709F01995D2
:10BD7000FF91EF91BF91AF919F918F917F916F91C3
:10BD80005F914F913F912F910F900BBE0F900FBE7F
:10BD90000F901F9018951F920F920FB60F921124BB
:10BDA0000BB60F922F933F934F935F936F937F93B5
:10BDB0008F939F93AF93BF93EF93FF93E091D62F11
:10BDC000F091D72F309709F01995FF91EF91BF911E
:10BDD000AF919F918F917F916F915F914F913F9123
:10BDE0002F910F900BBE0F900FBE0F901F901895C4
:10BDF0001F920F920FB60F9211240BB60F922F9332
:10BE00003F934F935F936F937F938F939F93AF93E2
:10BE1000BF93EF93FF93E091D42FF091D52F3097FC
:10BE200009F01995FF91EF91BF91AF919F918F917B
:10BE30007F916F915F914F913F912F910F900BBE2A
:10BE40000F900FBE0F901F9018951F920F920FB674
:10BE50000F9211240BB60F922F933F934F935F9342
:10BE60006F937F938F939F93AF93BF93EF93FF93C2
:10BE7000E091D22FF091D32F309709F01995FF91CF
:10BE8000EF91BF91AF919F918F917F916F915F9152
:10BE90004F913F912F910F900BBE0F900FBE0F90BF
:10BEA0001F901895CF93CFB7F894282F392F2115CD
:10BEB00088E0380749F461E083E00F94830864E088
:10BEC00083E00F9483084FC0203488E0380749F49A
:10BED00062E083E00F94830864E083E00F948308BA
:10BEE00042C0211589E0380749F461E084E00F94ED
:10BEF000830864E084E00F94830835C0203489E02F
:10BF0000380749F462E084E00F94830864E084E039
:10BF10000F94830828C021158AE0380749F461E0AE
:10BF200085E00F94830864E085E00F9483081BC0CC
:10BF300020348AE0380749F462E085E00F948308F2
:10BF400064E085E00F9483080EC021153B4049F45E
:10BF500061E086E00F94830864E086E00F94830834
:10BF600002C0CFBF01C0CFBFCF910895CF93CFB74D
:10BF7000F894282F392F211588E0380749F461E01B
:10BF800083E00F948F0864E083E00F948F084FC024
:10BF9000203488E0380749F462E083E00F948F088A
:10BFA00064E083E00F948F0842C0211589E03807D0
:10BFB00049F461E084E00F948F0864E084E00F941A
:10BFC0008F0835C0203489E0380749F462E084E006
:10BFD0000F948F0864E084E00F948F0828C0211527
:10BFE0008AE0380749F461E085E00F948F0864E047
:10BFF00085E00F948F081BC020348AE0380749F48D
:10C0000062E085E00F948F0864E085E00F948F086C
:10C010000EC021153B4049F461E086E00F948F0883
:10C0200064E086E00F948F0802C0CFBF01C0CFBF8D
:10C03000CF910895811528E0920729F46093183074
:10C04000709319300895803428E0920729F46093A2
:10C050000C3070930D300895811529E0920729F472
:10C0600060930430709305300895803429E092077E
:10C0700029F46093F82F7093F92F089581152AE021
:10C08000920729F46093F02F7093F12F0895803474
:10C090002AE0920729F46093E42F7093E52F089526
:10C0A00081159B4021F46093DC2F7093DD2F089560
:10C0B000FC01918195FFFDCF608380E090E00895C1
:10C0C0004F925F926F927F928F929F92AF92BF92A8
:10C0D000EF92FF920F931F93CF937C014A015B0174
:10C0E00028013901FC01848182FF16C0D901C801F1
:10C0F000689412F8B695A795979587951694D1F7F9
:10C10000B901A801032E36E17695679557954795B5
:10C110003A95D1F7302D15C0D901C801689413F8AC
:10C12000B695A795979587951694D1F7B901A8016B
:10C13000032E37E176956795579547953A95D1F750
:10C14000302D88159905AA05BB0508F4A6C08416EC
:10C150009506A606B70608F4A2C0F701848182FD01
:10C1600004C0880C991CAA1CBB1CC301B201A50108
:10C1700094010F9493282F3F31054105510508F490
:10C1800090C08FEF90E0A0E0B0E0C9EF05C02817A5
:10C1900039074A075B0758F0880F991FAA1FBB1F72
:10C1A000CD3F0CF48160CF5FC73089F74FC0CC23FF
:10C1B0000CF04CC0D501C401880F991FAA1FBB1FEA
:10C1C000880F991FAA1FBB1F880F991FAA1FBB1F8B
:10C1D000481A590A6A0A7B0ACE3FF4F48DEF9FEFA2
:10C1E0008C1B9109C7FD939504C0440C551C661C1B
:10C1F000771C8A95D2F7D501C401B695A795979576
:10C200008795BC01CD01640D751D861D971DA50187
:10C2100094010F94932837C083E08C0FA5019401FB
:10C2200004C0220F331F441F551F8A95D2F7DA012D
:10C23000C901B695A79597958795BC01CD01640D69
:10C24000751D861D971D0F9493281DC083E08C0FCC
:10C25000A501940104C0220F331F441F551F8A9566
:10C26000D2F7DA01C901B695A79597958795BC01D4
:10C27000CD01640D751D861D971D0F9493282150C7
:10C28000310941095109832F8F70C295C07FC82B96
:10C29000F701C783268381E018C080E016C080E0E4
:10C2A00014C0D501C401880F991FAA1FBB1F880F96
:10C2B000991FAA1FBB1F880F991FAA1FBB1F481ACF
:10C2C000590A6A0A7B0AC9EF89CFCF911F910F9152
:10C2D000FF90EF90BF90AF909F908F907F906F9066
:10C2E0005F904F9008950F931F93CF93DF93EC01CE
:10C2F0008B01009709F41EC1803C910529F460E18F
:10C3000080E00F94830816C1C11584E0D80729F492
:10C3100064E080E00F9483080DC1C038E1E0DE07DF
:10C3200029F462E080E00F94830804C1C115F1E0B4
:10C33000DF0729F461E080E00F948308FBC0C03878
:10C3400083E0D80729F461E081E00F948308F2C00C
:10C35000C039E3E0DE0729F461E082E00F9483084E
:10C36000E9C0C115F2E0DF0729F462E081E00F9433
:10C370008308E0C0C03482E0D80729F462E082E09C
:10C380000F948308D7C0C032E3E0DE0729F464E0ED
:10C3900082E00F948308CEC0C115F8E0DF0729F4CE
:10C3A00061E083E00F948308C5C0C11589E0D80718
:10C3B00029F461E084E00F948308BCC0C115EAE071
:10C3C000DE0729F461E085E00F948308B3C0C1154E
:10C3D000FBE0DF0729F461E086E00F948308AAC040
:10C3E000C03488E0D80729F462E083E00F94830822
:10C3F000A1C0C034E9E0DE0729F462E084E00F94D4
:10C40000830898C0C034FAE0DF0729F462E085E0D1
:10C410000F9483088FC0C03988E0D80729F464E0FE
:10C4200083E00F94830886C0C039E9E0DE0729F471
:10C4300064E084E00F9483087DC0C039FAE0DF0730
:10C4400029F464E085E00F94830874C0C0398BE060
:10C45000D80729F464E086E00F9483086BC0C03CE1
:10C46000E8E0DE0729F468E083E00F94830862C007
:10C47000C03CF9E0DF0729F468E084E00F9483080A
:10C4800059C0C03C8AE0D80729F468E085E00F94E1
:10C49000830850C0C03AE8E0DE0729F460E183E099
:10C4A0000F94830847C0C03AF9E0DF0729F460E140
:10C4B00084E00F9483083EC0C03A8AE0D80729F48C
:10C4C00060E185E00F94830835C0C03AEBE0DE07F9
:10C4D00029F460E186E00F9483082CC0C03BF8E0AB
:10C4E000DF0729F460E283E00F94830823C0C03B98
:10C4F00089E0D80729F460E284E00F9483081AC029
:10C50000C03BEAE0DE0729F460E285E00F9483088F
:10C5100011C0C038F4E0DF0729F460E483E00F9431
:10C52000830808C0C03A84E0D80721F460E485E0BD
:10C530000F9483088D818F738D83F8019581848199
:10C54000892B9681911198E0892B8D83F801408188
:10C5500051816281738100E010E62AEE30E0CE0165
:10C56000AFDD9C8198609C839C8190619C83DF916E
:10C57000CF911F910F910895CF92DF92EF92FF928A
:10C580000F931F93CF93DF93EC01D901C801B695A8
:10C59000A79597958795481759076A077B0778F4F9
:10C5A0006A017B01CC0CDD1CEE1CFF1CC901B8012B
:10C5B000A70196010F9493282150310902C020E071
:10C5C00030E0832F8F708F832E83DF91CF911F9167
:10C5D0000F91FF90EF90DF90CF900895EF92FF9230
:10C5E0000F931F93CF93DF93EC017B01009709F426
:10C5F000B9C1803C910529F460E180E00F94830883
:10C60000B1C18115944029F464E080E00F9483085F
:10C61000A9C1C03881E0D80729F462E080E00F9416
:10C620008308A0C1C115E1E0DE0729F461E080E0E4
:10C630000F94830897C1C038F3E0DF0729F461E065
:10C6400081E00F9483088EC1C03933E0D30729F409
:10C6500061E082E00F94830885C1C11582E0D807AC
:10C6600029F462E081E00F9483087CC1C034E2E0E9
:10C67000DE0729F462E082E00F94830873C1C032C0
:10C68000F3E0DF0729F464E082E00F9483086AC1D5
:10C69000C11538E0D30729F461E083E00F948308E3
:10C6A00061C1C11589E0D80729F461E084E00F94E5
:10C6B000830858C1C115EAE0DE0729F461E085E08E
:10C6C0000F9483084FC1C115FBE0DF0729F461E037
:10C6D00086E00F94830846C1C03438E0D30729F4BC
:10C6E00062E083E00F9483083DC1C03489E0D8073D
:10C6F00029F462E084E00F94830834C1C034EAE096
:10C70000DE0729F462E085E00F9483082BC1C0396D
:10C71000F8E0DF0729F464E083E00F94830822C186
:10C72000C03939E0D30729F464E084E00F9483082A
:10C7300019C1C0398AE0D80729F464E085E00F9474
:10C74000830810C1C039EBE0DE0729F464E086E01D
:10C750000F94830807C1C03CF8E0DF0729F468E0C4
:10C7600083E00F948308FEC0C03C39E0D30729F46E
:10C7700068E084E00F948308F5C0C03C8AE0D807E5
:10C7800029F468E085E00F948308ECC0C03AE8E043
:10C79000DE0769F460E183E00F948308E0EAF8E0E3
:10C7A00084818F7E8483F7012481225053C0C03A54
:10C7B000F9E0DF0729F460E184E00F948308D2C038
:10C7C000C03A3AE0D30729F460E185E00F9483088A
:10C7D000C9C0C03A8BE0D80729F460E186E00F9425
:10C7E0008308C0C0C03BE8E0DE0729F460E283E0D4
:10C7F0000F948308B7C0C03BF9E0DF0729F460E27B
:10C8000084E00F948308AEC0C03B3AE0D30729F41C
:10C8100060E285E00F948308A5C0C03884E0D807A3
:10C8200029F460E483E00F9483089CC0C03AE4E0FC
:10C83000DE0729F460E485E00F94830893C08C81BF
:10C840008F7E8C83FB0124812250CE01C03AF8E018
:10C85000DF0731F480914E0684FD8CC011E18BC05E
:10C86000803B38E0930779F0803AE9E09E0731F4A5
:10C8700030916E0634FD82C019E110C0803BF9E0B2
:10C880009F0789F001C015E1803A3AE0930731F43F
:10C8900080918E0684FD74C011E212C0803BEAE0F4
:10C8A0009E0759F001C01DE1803A9B4049F48091F8
:10C8B000AE0684FD04C019E203C015E201C01DE20A
:10C8C000E12FE695E695E69530E2E39FF00111242D
:10C8D000FA5F177081E090E0012E02C0880F991F67
:10C8E0000A94E2F78183223010F040E001C040E476
:10C8F000DF015096A10FB11D3FB7F8942C9127701E
:10C900002C939C91942B9C933FBF85838D81806C4D
:10C910008D83F70184818D7F813021F48D81826048
:10C920008D8303C08D818D7F8D83F7018581882361
:10C9300021F08D8184608D8303C08D818B7F8D83F9
:10C94000F701408151816281738100E010E62AEE97
:10C9500030E0CE0111DE8C8188608C838C81806117
:10C960008C8310C08C818F7E8C83F70124812250B0
:10C97000CE0176CF15E180EA98E080CF1DE18ECF21
:10C9800015E29ECFDF91CF911F910F91FF90EF9015
:10C9900008950F93E8ECF4E080818F7D808380819F
:10C9A0008F7D8083E8E1F1E302E0059310921A3174
:10C9B00010921B3100E2069300E40693E0E1F1E3FC
:10C9C00000E2069300E40693E9E0FAE31486158694
:10C9D0001686178612861386109203310F910895DA
:10C9E0000F9385E080930331E9E1F1E304E00593DF
:10C9F000E1E1F1E304E005930F9108950F9383E0E3
:10CA00008093033110921A3110921B31E8E1F1E367
:10CA100002E006930F910895E091153AF091163ACD
:10CA2000309709F0199508950F93CF93DF93809174
:10CA30000331833019F4F0DFACDF5EC08091FF304A
:10CA400090910031C091133AD091143AC81BD90B80
:10CA500071F52091013130910231820F931F809343
:10CA600001319093023120910F3A3091103A8217A0
:10CA7000930721F080911A30882341F084E080935D
:10CA80000331E0E1F1E302E0069336C0E091173AAA
:10CA9000F091183A309799F01995882381F0109207
:10CAA000FF3010920031C091133AD091143AC03443
:10CAB000D10528F010921A30C0E4D0E003C081E024
:10CAC00080931A30E4E0F1E3C68BD78B8091FF307E
:10CAD000909100312091113A3091123A280F391F6C
:10CAE000208F318FC80FD91FC093FF30D0930031F2
:10CAF000E8E1F1E302E00693DF91CF910F91089511
:10CB0000FC018181E82FE7708E2F90E0FC013197C6
:10CB1000E730F105D8F48827E456FE4F8F4F0D9487
:10CB2000D12880E190E0089580E290E0089580E4CB
:10CB300090E0089580E890E0089580E091E0089505
:10CB400080E092E008958FEF93E0089588E090E010
:10CB50000895282F2F7030E0220F331F082E000C6D
:10CB6000990B8827990F881F9927820F931F029787
:10CB70009C01220F331F220F331F220F331F820FFE
:10CB8000931F85569F4C08950F93CF938091CC04AB
:10CB900080FF63C081E08093CC04E0E1F1E300E832
:10CBA0000693E8E1F1E300E806938093CA04E0E12C
:10CBB000F1E300E1069380910331882329F083504B
:10CBC000823008F429DFE5DE809112319091133133
:10CBD000089709F044C088E0EFEBF0E3A9E0BAE37E
:10CBE00001900D928A95E1F7E8ECF4E08081806293
:10CBF00080838081806280830E941E54C82F8111AF
:10CC000003C0EEDEC1E02CC08091093A88236CF4A9
:10CC100010920131109202311092FF3010920031C7
:10CC200082E08093033100DF1BC080910F3A909126
:10CC3000103A892B11F4E2DE13C0109201311092E8
:10CC400002311092FF301092003181E08093033165
:10CC5000E0E1F1E302E0069303C0C0E001C0C1E0FF
:10CC60008C2FCF910F9108958F929F92AF92BF9288
:10CC7000DF92EF92FF920F931F93CF93DF93D82E03
:10CC800068DF8C01CD2DCF70D0E0CE01880F991FC9
:10CC9000CD2D0D2C000CDD0BCC27DD0FCC1FDD279F
:10CCA000C80FD91FCE01880F991F880F991F880FB1
:10CCB000991F9C01205F3E4C7901C90121DF4C0185
:10CCC000DD200CF07BC0FE01EE0FFF1FEE0FFF1FFB
:10CCD000EE0FFF1FEC5FFE4C22893389D8011596B9
:10CCE0008D919C911697820F931F15968D939C930F
:10CCF000169713962D913C9114978217930709F478
:10CD000047C0281B390B2115B4E03B0740F02FEF3B
:10CD100033E0C901B4010F946C28281B390BF801CA
:10CD2000808181FF0AC0C901B4010F946C2841E0E1
:10CD3000892B09F040E0842F01C080E0D8019C914C
:10CD400080FB91F99C93FE01EE0FFF1FEE0FFF1F7A
:10CD5000EE0FFF1FEC5FFE4C128A138A268737877F
:10CD600011962D913C91129715968D919C91169745
:10CD7000820F931FCC0FDD1FCC0FDD1FCC0FDD1FEB
:10CD8000CC5EDE4C88839983F70102E00693E4C011
:10CD9000D8018C9181FFCDC08D7F8C93CC0FDD1F8E
:10CDA000CC0FDD1FCC0FDD1FCC5FDE4C1A8A1B8A37
:10CDB0001E861F86F70102E00693CEC0FE01EE0F2D
:10CDC000FF1FEE0FFF1FEE0FFF1FEC5FFE4CA68450
:10CDD000B784D8018C9182FF1BC01196ED91FC9114
:10CDE000129715962D913C91169713968D919C91C3
:10CDF0001497B4010F946C28B0E4DB9EB0011124A9
:10CE00006552704DAC01CF01820F931F0F94B32A6E
:10CE1000F801258136812A0D3B1D258336838381C8
:10CE200094818217930768F485839683CC0FDD1F66
:10CE3000CC0FDD1FCC0FDD1FCC5FDE4C8A899B89B8
:10CE400078C0FE01EE0FFF1FEE0FFF1FEE0FFF1F5A
:10CE5000EC5FFE4C42895389A416B50609F069C0FF
:10CE60002817390709F465C0AC01421B530B9A011E
:10CE7000211554E0350748F02FEF33E0C901B40124
:10CE80000F946C28281B390B06C0C901B4010F94FC
:10CE90006C28281B390BFE01EE0FFF1FEE0FFF1F42
:10CEA000EE0FFF1FEC5FFE4C16861786281539051E
:10CEB00000F5D8018C9184608C93B0E4DB9EC001B6
:10CEC00011248552904DFE01EE0FFF1FEE0FFF1F44
:10CED000EE0FFF1FEC5EFE4C80839183CC0FDD1FB5
:10CEE000CC0FDD1FCC0FDD1FCC5FDE4C8A8A9B8A06
:10CEF0001CC0F8014181528185819681840F951F64
:10CF0000FE01EE0FFF1FEE0FFF1FEE0FFF1FEC5E87
:10CF1000FE4C80839183CC0FDD1FCC0FDD1FCC0F27
:10CF2000DD1FCC5FDE4C2A8B3B8BF70102E00693C2
:10CF300013C0D8018C9180FF0FC08E7F8C93179601
:10CF4000ED91FC911897309739F015966D917C9181
:10CF500016974D2D80E01995DF91CF911F910F917C
:10CF6000FF90EF90DF90BF90AF909F908F900895CB
:10CF7000CF93CFB7F894E1ECF4E080818E7F80838B
:10CF80001092C00410820F94D20810924431CFBF87
:10CF9000CF9108959FB7F89481E080934431EAECF3
:10CFA000F4E080E4808380E28083E1ECF4E080813F
:10CFB00081608083A9ECB4E08C9182608C93E8EC72
:10CFC000F4E08081806480838C9181608C93808187
:10CFD000806880839FBF0895CF93DF93C0E6D0E041
:10CFE000188280E30F949A08E0ECF4E0808180647A
:10CFF000808381E08883CFB7F894E4E0F1E315867D
:10D00000158A158E15A215A615AAEBE9F0E3808105
:10D010008E7F8083E4EAF0E380818E7F8083EDEA77
:10D02000F0E380818E7F8083E6EBF0E380818E7F6A
:10D0300080836AE170E082E00F9494268F3F19F0BC
:10D040008093FA0403C08FE18093FA046BE170E0EF
:10D0500082E00F9494268F3F19F08093FB0403C065
:10D060008FE18093FB04E0ECF4E0808182608083B8
:10D0700080818068808380818061808380E191E30A
:10D08000868397838081806280838FEF8093C5043D
:10D09000E8ECF4E0808181608083109244317ADF93
:10D0A000CFBFDF91CF9108958093C30408958091FD
:10D0B000C3040895E9E0FAE3808791876287738764
:10D0C0000895282F2F7030E0220F331F082E000CF8
:10D0D000990B8827990F881F9927820F931FFC01AE
:10D0E000EE0FFF1FEE0FFF1FEE0FFF1FEC5FFE4C5A
:10D0F0002585207C09F069C06370613011F018F457
:10D1000004C060EC03C060E801C060E44038510531
:10D11000E9F050F440325105A9F040345105A1F036
:10D1200040315105D9F40CC0411522E0520791F06D
:10D130004F3F23E0520781F04115514079F408C078
:10D1400021E00DC022E00BC023E009C024E007C0AD
:10D1500025E005C026E003C027E001C020E0FC0177
:10D16000EE0FFF1FEE0FFF1FEE0FFF1FEC5FFE4CD9
:10D17000158636E03487262B2587FC01EE0FFF1F2E
:10D18000EE0FFF1FEE0FFF1FEC5FFE4C2585207C8E
:10D19000203C69F4FC01EE0FFF1FEE0FFF1FEE0FA6
:10D1A000FF1FEC5FFE4C25852770273081F0880F2C
:10D1B000991F880F991F880F991FFC01EC5FFE4C87
:10D1C00085858062858781E0089580E0089581E00B
:10D1D0000895E82FEF70F0E0EE0FFF1F082E000C0F
:10D1E000990B8827990F881F9927E80FF91FEE0FD1
:10D1F000FF1FEE0FFF1FEE0FFF1FEC5FFE4C85853C
:10D2000082FB882780F90895282F2F7030E0A9012C
:10D21000440F551F282F082E000C330B2227330FE5
:10D22000221F3327240F351FF901EE0FFF1FEE0FCA
:10D23000FF1FEE0FFF1FEC5FFE4C958592FF17C09E
:10D24000220F331F220F331F220F331FF901EC5F10
:10D25000FE4C95859B7F95877CDCFC01808180FF5F
:10D2600006C08E7F80830780F085E02D199581E0D0
:10D2700008958F929F92AF92BF92CF92DF92EF92DA
:10D28000FF920F931F93CF93DF93982E862E6A0100
:10D2900079015FDC5C01292DC92DCF70D0E0CE0172
:10D2A000880F991FC92D092C000CDD0BCC27DD0F31
:10D2B000CC1FDD27C80FD91FFE01EE0FFF1FEE0F99
:10D2C000FF1FEE0FFF1FEC5FFE4C8585807C09F48D
:10D2D0007EC0FE01EE0FFF1FEE0FFF1FEE0FFF1FC0
:10D2E000EC5FFE4C8585807C803C61F0FE01EE0F9A
:10D2F000FF1FEE0FFF1FEE0FFF1FEC5FFE4C85853B
:10D3000082FD67C08FB7F894F501908190FF03C04C
:10D310008FBF80E05FC0F5019081916090838FBFE7
:10D32000C182D282E382F48215821682078310873B
:10D33000811006C091E0E114F10419F090E001C001
:10D3400091E0F501808190FB81F98B7F808322231E
:10D350005CF4CC0FDD1FCC0FDD1FCC0FDD1FCC5FCD
:10D36000DE4C1A8A1B8A2FC0FE01EE0FFF1FEE0F44
:10D37000FF1FEE0FFF1FEC5FFE4C8585807C803C1D
:10D38000B1F4CE01880F991F880F991F880F991F3C
:10D39000805F9E4CB5DBBC01C7010F946C28892BC4
:10D3A00031F0F50180818E7F808380E013C0CC0F47
:10D3B000DD1FCC0FDD1FCC0FDD1FCC5FDE4C1E86CA
:10D3C0001F861A8A1B8A892D4FDC81E003C080E00A
:10D3D00001C080E0DF91CF911F910F91FF90EF90FE
:10D3E000DF90CF90BF90AF909F908F900895FF9265
:10D3F0000F931F93CF93DF93182FC82FCF70D0E0D8
:10D40000CE01880F991FC12F012E000CDD0BCC27F8
:10D41000DD0FCC1FDD27C80FD91F812F9ADBDC0160
:10D42000FE01EE0FFF1FEE0FFF1FEE0FFF1FE05F6D
:10D43000FE4C02E005938C9180FF22C08E7F8C937E
:10D440001796ED91FC9118973097D1F011235CF469
:10D45000CC0FDD1FCC0FDD1FCC0FDD1FCC5FDE4CF2
:10D460006A897B890AC0CC0FDD1FCC0FDD1FCC0F72
:10D47000DD1FCC5FDE4C6E857F85412F81E01995E5
:10D48000DF91CF911F910F91FF900895CF93C82FF7
:10D49000AEDFEC2FEF70F0E0EE0FFF1F8C2FCC0F04
:10D4A000990B8827990F881F9927E80FF91FEE0F0E
:10D4B000FF1FEE0FFF1FEE0FFF1FEC5FFE4C1586E8
:10D4C000CF9108950F93E82FEF70F0E0EE0FFF1F5C
:10D4D000282F082E000C330B2227330F221F33274F
:10D4E000E20FF31FEE0FFF1FEE0FFF1FEE0FFF1FE8
:10D4F000DF01AC5FBE4C1D969C911D9794601D96FC
:10D500009C93E05FFE4C01E0069371DF81E00F9198
:10D5100008950F931F93CF93DF938B01C82FCF7084
:10D52000D0E0CC0FDD1F282F082E000C330B222754
:10D53000330F221F3327C20FD31F0BDBCC0FDD1F8E
:10D54000CC0FDD1FCC0FDD1FCC5FDE4C2D8522FF05
:10D550000AC0FC01208120FD0AC0216020830783CE
:10D56000108781E005C0F801199581E001C080E0D5
:10D57000DF91CF911F910F9108951F920F920FB6D7
:10D580000F9211240BB60F920F932F933F934F934B
:10D590005F936F937F938F939F93AF93BF93EF931B
:10D5A000FF938091CB04882344F480E88093CA04DD
:10D5B0000E94EE530E94244B87C08091CB0482FFCF
:10D5C00020C084E08093CA048091183186FF7CC01B
:10D5D0008091CC0481FD78C0D7DA811175C080912B
:10D5E0000331813011F40ADA6FC0843009F06CC065
:10D5F000E9E1F1E304E00593E1E1F1E304E00593FF
:10D6000063C08091CB0481FF5AC082E08093CA043A
:10D610008091103186FF58C08091CC0481FD54C0A8
:10D62000B3DA811151C080910331823041F484E03A
:10D6300080930331E0E1F1E302E0069345C08330DB
:10D6400009F042C0E9E1F1E304E00593E1E1F1E32F
:10D6500004E0059339C080E18093CA0481E0C7DE0D
:10D6600081E8C5DE0E94C3531092C304E4E0F1E3F5
:10D67000158696E0948783E48587158A948B858B3D
:10D680008FEB90E3808B918B84D91EC08091CB046B
:10D6900086FF08C080E48093CA04109244310E943F
:10D6A000274B12C08091CB0485FF0EC080E280938F
:10D6B000CA0481E0809344310E94284B05C08091C8
:10D6C000CB0484FFE3CFC7CFFF91EF91BF91AF9120
:10D6D0009F918F917F916F915F914F913F912F918A
:10D6E0000F910F900BBE0F900FBE0F901F901895CB
:10D6F0001F920F920FB60F9211240BB60F920F9339
:10D700001F932F933F934F935F936F937F938F93C9
:10D710009F93AF93BF93CF93DF93EF93FF9380914A
:10D72000CC0481FD03C030DA8111C2C082E0809355
:10D73000CC048091C5048195880FE0E1F1E3E81BFA
:10D74000F109208131812051314336952795369555
:10D75000279536952795822F869520FD02C090E06B
:10D7600001C090E8890FE82FEF70F0E0EE0FFF1F87
:10D77000282F082E000C330B2227330F221F3327AC
:10D78000E20FF31FDF01AA0FBB1FAA0FBB1FAA0FD7
:10D79000BB1FAC5FBE4C1C969C9195FF89C0EE0FE1
:10D7A000FF1FEE0FFF1FEE0FFF1FE05FFE4C00E2BA
:10D7B0000693811178C080910331843019F42CD9FB
:10D7C000E8D876C000911231109113318091133A4C
:10D7D0009091143AC091FF30D091003198012C0FF4
:10D7E0003D1F8217930718F48C010C1B1D0B8091B1
:10D7F000113A9091123AA8016FEB70E38C0F9D1FC4
:10D800000F94B32AC00FD11FC093FF30D0930031C3
:10D810000034110569F480910131909102318C0F2F
:10D820009D1F20910F3A3091103A8217930780F094
:10D83000E9E0FAE3C287D3870684F785E02D3097C5
:10D8400029F01995811102C0CBD832C0D7D830C089
:10D850008091133A9091143AC817D907F9F4E091DE
:10D86000173AF091183A309711F4BAD821C01995A7
:10D87000811102C0B5D81CC0209101313091023114
:10D880008091FF3090910031820F931F809301317E
:10D89000909302311092FF3010920031E0E1F1E3F9
:10D8A00002E0069305C0803811F4BED801C0DCD96F
:10D8B000FF91EF91DF91CF91BF91AF919F918F91A8
:10D8C0007F916F915F914F913F912F911F910F9198
:10D8D0000F900BBE0F900FBE0F901F901895909158
:10D8E000800024E0829FB00111246C7392709160DB
:10D8F000692B80E890E00F943526E0E8F0E0828123
:10D9000080FDFDCF0895609180006C73636080E8B6
:10D9100090E00F943526E0E8F0E0828180FDFDCFB5
:10D920000895CF92DF92EF92FF92CF93DF93EC01B5
:10D930006B01E12CF12C60E070E68AEE90E0A7012B
:10D9400096010F949328CA01B9012FEF3FEF40E0F1
:10D9500050E00F9493282115310529F481E08C8340
:10D9600021E030E02DC02230310528F482E08C83A4
:10D9700022E030E025C02430310528F483E08C8398
:10D9800024E030E01DC02830310528F484E08C8389
:10D9900028E030E015C02034310528F485E08C8380
:10D9A00020E430E00DC02F3F310509F028F486E077
:10D9B0008C8320E031E004C087E08C8320E034E0F9
:10D9C00040E050E060E070E68AEE90E00F9493282B
:10D9D000CA01B901A70196010F9493282D833E83B4
:10D9E0002436310518F41C821D821E82DF91CF91EE
:10D9F000FF90EF90DF90CF9008950F931F93CF93F8
:10DA0000DF93EC018901862F90E08730910508F0C3
:10DA10008BC0FC018827ED55FE4F8F4F0D94D12808
:10DA200080E098E088839983E0E4F6E0308181E04B
:10DA300090E02FEF240F02C0880F991F2A95E2F77C
:10DA4000832B808371C080E498E088839983E0E42D
:10DA5000F6E0308181E090E023E0240F02C0880FDF
:10DA6000991F2A95E2F7832B80835EC080E099E0BE
:10DA700088839983E0E6F6E0308181E090E02FEF43
:10DA8000240F02C0880F991F2A95E2F7832B808309
:10DA90004BC080E499E088839983E0E6F6E030812A
:10DAA00081E090E023E0240F02C0880F991F2A959F
:10DAB000E2F7832B808338C080E09AE088839983E3
:10DAC000E0E8F6E0308181E090E02FEF240F02C023
:10DAD000880F991F2A95E2F7832B808325C080E465
:10DAE0009AE088839983E0E8F6E0308181E090E075
:10DAF00023E0240F02C0880F991F2A95E2F7832B99
:10DB0000808312C080E09BE088839983E0EAF6E09E
:10DB1000308181E090E02FEF240F02C0880F991F21
:10DB20002A95E2F7832B80834A83423061F018F410
:10DB3000413031F010C0433049F0443051F00BC057
:10DB400080E18B8308C080E28B8305C080E48B83F7
:10DB500002C080E88B83888199810E94525FE881AE
:10DB6000F9818181887F836081831D821E821C826E
:10DB7000E881F9818081807F8083B801CE01D1DE88
:10DB8000DF91CF911F910F910895CF93DF93EC0117
:10DB90002D813E81A62FB0E00F94D92824E630E0F5
:10DBA00040E050E00F9493288A81E881F981E6FDF6
:10DBB00017C0823061F018F4813031F01BC083301F
:10DBC00049F0843051F016C020AF31AF13C022AFFE
:10DBD00033AF10C024AF35AF0DC026AF37AF0AC08A
:10DBE000813019F0823021F005C020AF31AF02C082
:10DBF00022AF33AF8D819E81E881F98186A397A3FF
:10DC00008B81E881F981E6FD04C09181892B8183B4
:10DC100004C091818073892B8183E881F98180819F
:10DC2000807F9C81892B8083DF91CF910895CF9352
:10DC3000DF93EC014115510509F443C0A6E7BCE3AD
:10DC400020E030E0922FF901E95DFE4EE491ED9382
:10DC50002F5F3F4F27303105A9F7FA01DE01C6E7F4
:10DC6000DCE380818B8381818C83F901EA58F34C5A
:10DC70008CE28083E2E0E90FF0E0EA58F34C608345
:10DC8000C4E0C90F9D5FE92FF0E0EA58F34C8DE73F
:10DC90008083D0E0FE01EA58F34C108221E0AE010F
:10DCA00066E77CE3CD010E94D0F60E94E426811154
:10DCB00008C021E0AE0166E77CE38BE093E30E94BD
:10DCC000D0F6DF91CF9108954F925F926F927F923D
:10DCD0008F929F92AF92BF92DF92EF92FF920F933B
:10DCE0001F93CF93DF931F92CDB7DEB77C01411511
:10DCF000510509F466C188E08983A6E7BCE320E00A
:10DD000030E0922FF901E95DFE4EE491ED932F5F33
:10DD10003F4F27303105A9F7FA01162FA6E7BCE3DC
:10DD2000808113968C931397818114968C9302E0D3
:10DD3000090FF901EA58F34C8CE28083623088F5D0
:10DD4000862F0E9424E68823B1F0812F0E94E9E506
:10DD50009F938F931F921F9385E998E29F938F93D0
:10DD6000E02FF0E0EA58F34CFF93EF930F94D92A99
:10DD7000CDBFDEBF08C1812F0E94A0A99F938F93C2
:10DD80001F921F9385E998E29F938F93E02FF0E015
:10DD9000EA58F34CFF93EF930F94D92ACDBFDEBF1F
:10DDA000F2C0663109F078C086E10E9449E52B0196
:10DDB0003C010E949CDE4B015C01672B682B692BA8
:10DDC000F1F4C301B20120E13EE040E050E00F94E5
:10DDD000B5285F934F933F932F931F9286E18F93C4
:10DDE0008CE998E29F938F93E02FF0E0EA58F34C90
:10DDF000FF93EF930F94D92ACDBFDEBFC4C0802F0D
:10DE00000E943BA9992334F5C301B20120E13EE011
:10DE100040E050E00F94B528CA01B9010E94E9FB27
:10DE2000BF92AF929F928F929F938F937F936F93A6
:10DE30001F9286E18F9384EA98E29F938F93E02F5D
:10DE4000F0E0EA58F34CFF93EF930F94D92ACDBF3B
:10DE5000DEBF99C0BF92AF929F928F92C301B20171
:10DE600020E13EE040E050E00F94B5285F934F93EF
:10DE70003F932F931F9286E18F9381EB98E29F93BC
:10DE80008F93E02FF0E0EA58F34CFF93EF930F9459
:10DE9000D92ACDBFDEBF77C0663071F5E02FF0E044
:10DEA000EA58F34C86E380836894DD24D2F8D90ED7
:10DEB0009D5FE92FF0E0EA58F34C8CE2808386E026
:10DEC0000E9449E58B019C018D2D90E04BE0BE0145
:10DED0006F5F7F4F8A58934C0E9442FCE981ED0DA1
:10DEE000AE2FB0E0AA58B34C8DE78C93EF5FF0E013
:10DEF000EA58F34C108247C0653071F5E02FF0E02E
:10DF0000EA58F34C85E380836894DD24D2F8D90E77
:10DF10009D5FE92FF0E0EA58F34C8CE2808385E0C6
:10DF20000E9449E58B019C018D2D90E04BE0BE01E4
:10DF30006F5F7F4F8A58934C0E948EFDE981ED0DF3
:10DF4000AE2FB0E0AA58B34C8DE78C93EF5FF0E0B2
:10DF5000EA58F34C108217C0862F0E9449E59F9320
:10DF60008F937F936F931F921F938CE998E29F93F7
:10DF70008F93802F90E08A58934C9F938F930F94A8
:10DF8000D92ACDBFDEBFE6E7FCE301900020E9F728
:10DF90003197E657FC43E983AF01552721E066E757
:10DFA0007CE3C7010E94D0F60E94E426811109C0DB
:10DFB000498150E021E066E77CE38BE093E30E9437
:10DFC000D0F60F90DF91CF911F910F91FF90EF90BE
:10DFD000DF90BF90AF909F908F907F906F905F90F9
:10DFE0004F900895AC016115710571F1E0E3F1E125
:10DFF000A6E7BCE32EE73CE394919D933196A217EC
:10E00000B307D1F7FB01CA01A6E7BCE32081139651
:10E010002C931397218114962C93149718961C9285
:10E02000189721E048E050E0BD010E94D0F60E9420
:10E03000E426811109C021E048E050E066E77CE376
:10E040008BE093E30C94D0F60895EF92FF920F9338
:10E050001F93CF93DF938C016115710509F47FC085
:10E060004115510509F47BC0EEE1F1E1A6E7BCE3FF
:10E07000CEE7DCE394919D933196AC17BD07D1F7C1
:10E08000FA017B01C6E7DCE380818B8381818C838D
:10E090001F922F938DEB98E29F938F938EE79CE3D3
:10E0A0009F938F930F94D92A09900020E9F7219725
:10E0B000C657DC43F70181810F900F900F900F90AE
:10E0C0000F900F90811115C080811F928F938DE664
:10E0D00091E29F938F93DD27CA58D34CDF93CF9360
:10E0E0000F94D92A0F900F900F900F900F900F90D0
:10E0F00016C01F928F93F70180811F928F938AE63B
:10E1000091E29F938F93DD27CA58D34CDF93CF932F
:10E110000F94D92AEDB7FEB73896EDBFFEBFE6E7FC
:10E12000FCE301900020E9F73197E657FC43EF014B
:10E13000DD2721E0AE0166E77CE3C8010E94D0F64E
:10E140000E94E42681110BC00B50134341F021E0E3
:10E15000AE0166E77CE38BE093E30E94D0F6DF91AB
:10E16000CF911F910F91FF90EF900895CF93DF9380
:10E17000EC014115510509F43FC0662361F0E0E36D
:10E18000F1E1A6E7BCE390E024912D939F5F3196E7
:10E190009730D1F70BC0E7E2F1E1A6E7BCE390E0EE
:10E1A00024912D939F5F31969730D1F7DA01CE01FC
:10E1B000E6E7FCE32C91238311962C9124832CE237
:10E1C00027833CE43087218720E322872DE72387BC
:10E1D000148621E04CE050E0BF010E94D0F60E947E
:10E1E000E426811109C021E04CE050E066E77CE3C1
:10E1F0008BE093E30E94D0F6DF91CF910895EF92E8
:10E20000FF920F931F93CF93DF9300D01F92CDB750
:10E21000DEB70097C9F166307105C0F1FC012081BD
:10E220002035B1F521812C32A9F524812C32A1F5BC
:10E230007A018C010B5F1F4FAB01455051099E01C4
:10E240002F5F3F4FB8018CE20E9419FC882349F1EF
:10E2500049815A814B5F5F4F49835A83463051054C
:10E26000E8F045509E012D5F3F4F60E0C8010E94DD
:10E27000A1FA8823B1F08B819C818C31910580F4C7
:10E28000F701808381E00DC080E00BC080E009C011
:10E2900080E007C080E005C080E003C080E001C0EE
:10E2A00080E02496CDBFDEBFDF91CF911F910F910B
:10E2B000FF90EF900895CF92DF92EF92FF920F932D
:10E2C0001F93CF93DF93CDB7DEB72C97CDBFDEBFC3
:10E2D000009709F4E4C06630710508F4E2C0FC015F
:10E2E0002081203509F0DFC021812C3209F0DDC00A
:10E2F00024812C3209F0DBC07B018C016C01F5E03C
:10E30000CF0ED11CAB01455051099E012F5F3F4FED
:10E31000B6018CE20E9419FC882309F4D7C0498118
:10E320005A814B5F5F4F49835A834630510508F449
:10E33000C0C045509E012D5F3F4F60E0C6010E9466
:10E34000A1FA882309F4C2C02B813C812C3131050C
:10E3500008F0B1C049815A81DA011196AE15BF05A6
:10E3600008F0ABC02C31310508F0A9C0F9018827AD
:10E37000E655FE4F8F4F0D94D128C8018A0F9B1F81
:10E38000FC0160816D3241F4FA013296EE15FF0511
:10E3900008F097C040E002C0FD0141E026313105A0
:10E3A00059F46E2D6E1B9E01275F3F4FC8018E0FE3
:10E3B0009F1F0E94ACD512C02630310541F46E2D4E
:10E3C0006A1BAE01475F5F4F0E9479D807C06E2D70
:10E3D0006A1BAE01475F5F4F0E9495D9882309F4FD
:10E3E00072C049855A856B857C858B810E9493AA72
:10E3F000882309F46BC049855A856B857C858B81A0
:10E400000E945CE581E062C04E2D4A1B9E012B5F9D
:10E410003F4F60E0C8018A0F9B1F0E942CFB88239E
:10E4200009F454C04D815E816F81788549875A8790
:10E430006B877C878B810E9493AA882349F049854A
:10E440005A856B857C858B810E945CE581E03EC0AE
:10E450002B813C81A9014C50510946305105B0F542
:10E4600049855A856B857C85452B462B472B71F555
:10E4700040E050E0BA01822F0E945CE581E026C0B6
:10E48000C7018A1B9B0B899700F56E2D6A1B422FD3
:10E49000C8018A0F9B1F0E94C7E581E017C080E07A
:10E4A00015C080E013C080E011C080E00FC080E0A4
:10E4B0000DC080E00BC080E009C080E007C080E0B4
:10E4C00005C080E003C080E001C080E02C96CDBF95
:10E4D000DEBFDF91CF911F910F91FF90EF90DF9002
:10E4E000CF9008950F931F93CF93DF931F921F92A6
:10E4F000CDB7DEB7009741F16630710538F1FC0108
:10E500002081203529F521812C3221F524812C32DE
:10E5100019F58C01AB0145505109BC016B5F7F4F70
:10E520009E012F5F3F4F8CE20E9419FC8823B9F0B7
:10E5300089819A810596069788F081E0F801958196
:10E54000963469F080E00BC080E009C080E007C02D
:10E5500080E005C080E003C080E001C080E00F9053
:10E560000F90DF91CF911F910F910895EF92FF923D
:10E570000F931F93CF93DF9300D000D0CDB7DEB7BA
:10E58000009709F453C06630710508F451C0FC01CE
:10E590002081203509F04EC021812C3209F04CC079
:10E5A00024812C3209F04AC07B018C01AB0145501B
:10E5B0005109BC016B5F7F4F9E012F5F3F4F8CE283
:10E5C0000E9419FC882309F442C089819A819C0128
:10E5D0002B5F3F4F29833A832630310588F1F801BC
:10E5E0002581263479F506968E159F0568F54E2D02
:10E5F000481B9E012D5F3F4F60E0800F911F0E94DE
:10E600002CFB882321F16B817C818D819E818B0184
:10E610009C010150110921093109073E13402105D0
:10E620003105A0F40E9424AA81E011C080E00FC04F
:10E6300080E00DC080E00BC080E009C080E007C032
:10E6400080E005C080E003C080E001C080E0269645
:10E65000CDBFDEBFDF91CF911F910F91FF90EF9063
:10E6600008950F931F93CF93DF93EC01611571050C
:10E6700009F444C0A6E7BCE320E030E0922FF901A2
:10E68000E95DFE4EE491ED932F5F3F4F273031055A
:10E69000A9F7FB01A6E7BCE3808113968C9313973F
:10E6A000818114968C931497F901EA58F34C8CE20B
:10E6B00080839E5FE92FF0E0EA58F34C86E49DE703
:10E6C000808391831282FD0101900020E9F7319748
:10E6D000E657FC438F01112721E0A801BD01CE01BF
:10E6E0000E94D0F60E94E426811108C021E0A80112
:10E6F00066E77CE38BE093E30E94D0F6DF91CF9155
:10E700001F910F910895FC01892B61F0653071050F
:10E7100058F08081803551F481E091819C3239F04C
:10E7200080E0089580E0089580E0089580E00895F5
:10E73000009799F06330710590F0FC01208120353D
:10E7400081F421812C3279F424812C3271F4858179
:10E750008354823060F080E0089580E0089580E086
:10E76000089580E0089580E0089580E0089581E0B4
:10E770000895009791F06330710588F0FC012081C5
:10E78000203579F421812C3271F424812C3269F402
:10E7900085818F3461F080E0089580E0089580E005
:10E7A000089580E0089580E0089580E0089581E074
:10E7B0000895009791F06330710588F0FC01208185
:10E7C000203579F421812C3271F424812C3269F4C2
:10E7D0008581873561F080E0089580E0089580E0CC
:10E7E000089580E0089580E0089580E0089581E034
:10E7F0000895CF92DF92EF92FF920F931F93CF93E2
:10E80000DF934115510509F4AAC0009709F4A9C086
:10E810006630710508F4A7C0FC012081203509F09D
:10E82000A4C021812C3209F0A2C024812C3209F02D
:10E83000A0C08581873509F09EC0EA0180E496E397
:10E840000E942012883009F498C080E496E30E9468
:10E850002012863009F493C00E94BFEF0E946E46DA
:10E8600061E086E496E30E94E2480E9468E60E9426
:10E87000721A813079F582E00E9449A96B017C010E
:10E88000DD24EE24FF24B701A60182E00E945CE5AE
:10E89000B701A60182E00E9431A90E94E4268111FD
:10E8A00019C084E1E1ECF8E2A1EDBDE301900D9225
:10E8B0008A95E1F7E1EDFDE301900020E9F731975A
:10E8C000AF01415D5D4320E061ED7DE38BE093E3CB
:10E8D0000E94D0F680E00E9417A99B01AC016894C9
:10E8E000EE24E2F808E312E2BE01685E7F4FCE013B
:10E8F00006960E943C4A8D8340E050E0BA01CE016A
:10E900000E94412B8D81882341F182E00E943BA926
:10E91000062F8BE00E943BA921E0611120E040EE30
:10E9200059E3BE016E5C7F4FCE01C4960E944F45F5
:10E93000CE010E94B0199E01285A3D4FAE01495A9E
:10E940005D4FBE016E5A7D4FCE018F5A9D4F0E9482
:10E95000C82968E0CE010E940D128D8111C080E0AF
:10E960000FC080E00DC080E00BC080E009C080E0F7
:10E9700007C080E005C080E003C080E001C080E007
:10E98000DF91CF911F910F91FF90EF90DF90CF908B
:10E990000895CF92DF92EF92FF920F93CF93DF9380
:10E9A0004115510509F4B0C0009709F4AFC06630B5
:10E9B000710508F4ADC0FC012081203509F0AAC022
:10E9C00021812C3209F0A8C024812C3209F0A6C084
:10E9D000EA018581833409F493C0843409F0A0C02E
:10E9E0000E94D9A90E9406E680E496E30E942012C4
:10E9F000883009F497C080E496E30E9420128630A4
:10EA000009F492C00E94BFEF0E946E4661E086E466
:10EA100096E30E94E2480E9468E60E94721A8130E2
:10EA200079F582E00E9449A96B017C01DD24EE2486
:10EA3000FF24B701A60182E00E945CE5B701A601B0
:10EA400082E00E9431A90E94E426811119C084E16C
:10EA5000E1ECF8E2A1EDBDE301900D928A95E1F7BA
:10EA6000E1EDFDE301900020E9F73197AF01415D51
:10EA70005D4320E061ED7DE38BE093E30E94D0F6FF
:10EA800080E00E9417A99B01AC01BE01685E7F4F28
:10EA9000CE0106960E9476468D8340E050E0BA0192
:10EAA000CE010E94412B8D81882341F182E00E949A
:10EAB0003BA9062F8BE00E943BA921E0611120E0D9
:10EAC00040EE59E3BE016E5C7F4FCE01C4960E94BA
:10EAD0004F45CE010E94B0199E01285A3D4FAE010C
:10EAE000495A5D4FBE016E5A7D4FCE018F5A9D4FE0
:10EAF0000E94C82968E0CE010E940D128D8115C0C8
:10EB00000E9406E681E011C080E00FC080E00DC0E9
:10EB100080E00BC080E009C080E007C080E005C055
:10EB200080E003C080E001C080E0DF91CF910F91D1
:10EB3000FF90EF90DF90CF900895BF92CF92DF9239
:10EB4000EF92FF920F931F93CF93DF931F92CDB756
:10EB5000DEB76115710509F464C0DB017C01E6E7ED
:10EB6000FCE38BE7808380E781838CE282839C9146
:10EB7000938311969C91948385839FE496838783E6
:10EB800080E00E9445B08B019C0148E0BE016F5FB0
:10EB90007F4F8EE79CE30E94F0FDE981E85FD12C76
:10EBA0000F2EFCE2BF2EF02DCC24C394CE0EF0E04D
:10EBB000EA58F34CB082D3948D2D0E9445B08B015E
:10EBC0009C018C2D90E048E0BE016F5F7F4F8A581A
:10EBD000934C0E94F0FDE981EC0D83E0D812E4CF64
:10EBE00081E08E0FF0E0EA58F34C9DE79083482FC8
:10EBF00050E0FA01EA58F34C1082898321E066E77D
:10EC00007CE3C7010E94D0F60E94E426811109C06E
:10EC1000498150E021E066E77CE38BE093E30E94CA
:10EC2000D0F60F90DF91CF911F910F91FF90EF9051
:10EC3000DF90CF90BF900895CF93DF93411551059A
:10EC4000A9F10097A9F165307105A0F1FC012081BF
:10EC5000203591F521812C3289F52281263481F5E8
:10EC6000EA0184818235E9F0833531F0843451F54D
:10EC70000E9403AA81E027C00E94BFEFBE016E5C24
:10EC80007F4FCE01C4960E94544380E496E30E94D5
:10EC9000901F81110E94E1EFCE010E947E268D819E
:10ECA00012C0CA01C4960E94F6DD0DC080E00BC000
:10ECB00080E009C080E007C080E005C080E003C0BC
:10ECC00080E001C080E0DF91CF910895FC01892BA5
:10ECD00079F06630710570F08081833569F4818147
:10ECE0008C3261F481E094819C3249F080E0089597
:10ECF00080E0089580E0089580E0089580E0089520
:10ED00000F93CF93DF93009709F476C066307105B7
:10ED100008F474C0FC016081633509F071C0618141
:10ED20006C3209F06FC064816C3209F06DC041151E
:10ED3000510509F46BC02115310509F469C08581BD
:10ED4000813309F067C0B901EA01F9011082CA01F3
:10ED50000E94771D882309F45FC0CE010E94581DD0
:10ED600081112BC0CE010E947E2661E0CE010E945F
:10ED7000AE2364E0CE010E940D1261E0CE010E943C
:10ED8000491D19820E94AD8FE2EBFCE3808190E087
:10ED9000DC01AE54B34C25853685880F991FFC01E4
:10EDA000EE54F34C418152811F960C9161E080E456
:10EDB00096E30E94DD2181E032C00E94E4268111A9
:10EDC0002DC083E1E5EDF8E2A6E7BCE301900D92EA
:10EDD0008A95E1F7E6E7FCE301900020E9F7319737
:10EDE000AF0146575C4321E066E77CE38BE093E3A9
:10EDF0000E94D0F681E013C080E011C080E00FC017
:10EE000080E00DC080E00BC080E009C080E007C05A
:10EE100080E005C080E003C081E001C081E0DF91B7
:10EE2000CF910F9108950F93CF93DF93009709F43B
:10EE3000DFC06630710508F4DDC0FC012081233598
:10EE400009F0DAC021812C3209F0D8C024812C329B
:10EE500009F0D6C04115510509F4D4C0EA018581F5
:10EE6000833309F46FC028F4803351F08233D9F131
:10EE7000CBC0833609F4A0C0823709F4ABC0C4C04C
:10EE8000CA010E942012843009F0C0C0CE010E9445
:10EE9000D51CCE010E947E260E94BFEF60E080E478
:10EEA00096E30E94AE2363E0CE010E940D12198208
:10EEB0000E949A8FE2EBFCE3808190E0DC01AE548B
:10EEC000B34C25853685880F991FFC01EE54F34C11
:10EED000418152811F960C9161E080E496E30E948B
:10EEE000DD2191E09CC0CA010E94581D882309F4CD
:10EEF0008FC081E0898360E0CE010E94C91260E08A
:10EF0000CE010E94BE120E94E426811183C080E1DE
:10EF1000E8EEF8E2A6E7BCE301900D928A95E1F7EE
:10EF2000E6E7FCE301900020E9F73197AF0146578F
:10EF30005C4321E066E77CE38BE093E30E94D0F63C
:10EF400091E06DC0CA010E94581D882309F464C075
:10EF500060E0CE010E94C91260E0CE010E94BE12A4
:10EF6000FE01EF5AFD4FDE01A95ABD4F8C918083FF
:10EF7000319611968C91808319820E94E42681112A
:10EF80004DC080E1E8EFF8E2A6E7BCE301900D9206
:10EF90008A95E1F7E6E7FCE301900020E9F7319775
:10EFA000AF0146575C4321E066E77CE38BE093E3E7
:10EFB0000E94D0F691E033C0CA010E94581D982FDC
:10EFC000882369F1CE010E944B2491E0811127C072
:10EFD00090E025C0CA010E94581D882329F0CE0167
:10EFE0000E94D523982F1BC00E9497B091E017C0B4
:10EFF00090E015C090E013C090E011C090E00FC009
:10F0000090E00DC090E00BC090E009C091E007C017
:10F0100091E005C091E003C091E001C091E0892F2B
:10F02000DF91CF910F910895FC01892B61F066303B
:10F03000710558F080818D3451F481E091819C32CA
:10F0400039F080E0089580E0089580E0089580E040
:10F050000895FC01892B61F06630710558F08081BC
:10F06000823551F481E091819C3239F080E008953D
:10F0700080E0089580E0089580E00895FC01892BE8
:10F0800061F06530710558F080818A3551F481E076
:10F0900091819C3239F080E0089580E0089580E00D
:10F0A000089580E00895CF92DF92EF92FF920F9340
:10F0B0001F93CF93DF93CDB7DEB72897CDBFDEBFC9
:10F0C000009709F457C06630710508F455C0FC017B
:10F0D00020812A3509F052C021812C3209F050C01C
:10F0E0007B018C016C01F2E0CF0ED11CAB014250D0
:10F0F00051099E012F5F3F4FB6018CE20E9419FC1F
:10F10000882309F446C049815A814E5F5F4F498385
:10F110005A8343305105B0F142509E012D5F3F4F5D
:10F1200060E0C6010E94A1FA882399F18B819C813D
:10F13000039750F589819A8101968E159F0530F5C8
:10F140004E2D481B9E012B5F3F4F60E0800F911FAB
:10F150000E942CFB8823E9F06D817E818F81988548
:10F16000623071058105910598F48B810E94F6C289
:10F1700081E00FC080E00DC080E00BC080E009C0DE
:10F1800080E007C080E005C080E003C080E001C0EF
:10F1900080E02896CDBFDEBFDF91CF911F910F9108
:10F1A000FF90EF90DF90CF9008952F923F924F9273
:10F1B0005F926F927F928F929F92AF92BF92CF9207
:10F1C000DF92EF92FF920F931F93CF93DF93CDB710
:10F1D000DEB76397CDBFDEBF8C01F62E81E08D8355
:10F1E0000115110509F423C38093CE2089E10E9403
:10F1F0003BA9672B682B692B09F025C30E942BE1E3
:10F20000B82E811103C0F11020C385C380E496E3BA
:10F210000E94CA1DB82E882309F47DC380E496E3BA
:10F220000E9420128F87F11004C08150823008F4B0
:10F2300000C32F85243031F480E496E30E94C22677
:10F2400033E03F870E9409E70E94F2E680E496E3FC
:10F250000E94901F81110E94E1EF80E496E30E94DA
:10F260007E2682E00E943BA9E62E8FEF8E0D8A302B
:10F2700008F0E1C2AE014A5F5F4FBE016B5F7F4F96
:10F280008E2D0E94051F8E810E9461C28E81847026
:10F290000E94D5C28D810E943FE30F2EF6E7CF2E4C
:10F2A000FCE3DF2EF02D8BE7D6018C938DE61196D3
:10F2B0008C9311978CE212968C93129787E7139692
:10F2C0008C9320E044E050E0B601C8010E94D0F6E3
:10F2D0001F92EF9288E099E29F938F93DF92CF92F3
:10F2E0000F94D92AF60101900020E9F73197AF0178
:10F2F00046575C4320E0B601C8010E94D0F6ECE717
:10F30000F7E487858F9386858F9385858F93848592
:10F310008F930F2EFCE0AF2EF9E2BF2EF02DBF929F
:10F32000AF92DF92CF920F94D92AF601019000207C
:10F33000E9F73197AF0146575C4320E0B601C801B9
:10F340000E94D0F68AE00E943BA99F938F937F93FF
:10F350006F93BF92AF92DF92CF920F94D92AF601AA
:10F3600001900020E9F73197AF0146575C4320E058
:10F37000B601C8010E94D0F68BE00E943BA99F9382
:10F380008F937F936F93BF92AF92DF92CF920F9440
:10F39000D92AF60101900020E9F73197AF014657CD
:10F3A0005C4320E0B601C8010E94D0F60F2EF6E9BA
:10F3B000CF2EF7E4DF2EF02DCDBFDEBF412C512C38
:10F3C000320145010F2EF6E7AF2EFCE3BF2EF02DE4
:10F3D0002BC0D6018C9111969C91119712962C916D
:10F3E000129713963C91B4E0CB0ED11C3F932F9310
:10F3F0009F938F939F928F92BF92AF920F94D92A2F
:10F40000F50101900020E9F73197AF0146575C43C1
:10F4100020E0B501C8010E94D0F6EFEF4E1A5E0A57
:10F420006E0A7E0ACDBFDEBF0E94C0F290E0A0E06F
:10F43000B0E0481659066A067B0658F28DE78093BD
:10F44000763C21E041E050E066E77CE3C8010E94A1
:10F45000D0F665E080E496E30E940D120E94BFEFB3
:10F4600080E496E30E94C8210E94A64B60E072E00F
:10F4700080E090E00E94984C1092193A10921A3A4B
:10F4800087EC9CE30E94B2930E94394E8111FCCF1D
:10F49000B82EF11004C00E94BD1C8823E1F389E05E
:10F4A0000E943BA96F3171058105910508F59B010B
:10F4B000AC01012E1CE0220F331F441F551F1A956B
:10F4C000D1F7102D2B873C874D875E87CA01B90184
:10F4D0000E94ABE60E9489F081E00E94D9F280E0B0
:10F4E00090E1A0E0B0E08F839887A987BA873FC0FA
:10F4F0009B01AC01012E19E0220F331F441F551F41
:10F500001A95D1F7102D2B873C874D875E87CA014E
:10F51000B9010E94ABE60E9489F00E9409F380E0E5
:10F5200092E0A0E0B0E08F839887A987BA871FC0D8
:10F53000412C512C32019F2CCB84DC84ED84FE8441
:10F540000E9446F38823E1F08D810E94D3EE67ECA0
:10F550007CE30E941594A82E0E9435F39FEF491A70
:10F56000590A690A790AA1100BC0F92C0FC02B8522
:10F570003C854D855E85232B242B252BC9F606C0A3
:10F580004C145D046E047F04D8F2F92C0E9430F311
:10F5900087EC9CE30E947994E82E0E94254D0E94FE
:10F5A00055EDEE2031F06F8580E496E30E940D1258
:10F5B000B2C180EF9EE30E94C1B5882351F0F110E3
:10F5C00008C06091EF3F70E080EF9EE30E94D99405
:10F5D00009C0E6E7FCE31082118262E070E0CF012F
:10F5E0000E94D99460E072E080E090E00E94AE4B0F
:10F5F0000E94394E8111FCCF8B859C85AD85BE85DF
:10F60000892B8A2B8B2B09F4F3C0C12CD12C7601CA
:10F610000F2EF6E72F2EFCE33F2EF02D4F8058845F
:10F6200069847A8491E0491A5108610871080E943E
:10F63000C8948093193A90931A3AAE014F5F5F4F86
:10F64000BC018D810E94D412882309F463C1C701D3
:10F65000B6012F81388549855A850F9493284B012F
:10F660005C01672B682B692BA1F5C701B6012F81BF
:10F67000388549855A850F949328288B398B4A8B76
:10F680005B8B89E00E943BA9AB89AF93BA89BF939A
:10F69000E989EF93F889FF939F938F937F936F93FB
:10F6A00021E139E23F932F933F922F920F94D92A71
:10F6B000F10101900020E9F73197AF0146575C4313
:10F6C00020E0B101C8010E94D0F61092CE20CDBF3B
:10F6D000DEBF2F81388549855A85211582E038079C
:10F6E0004105510509F4BAC02115304141055105C4
:10F6F00009F4DDC0D701C60187709927AA27BB2767
:10F70000892B8A2B8B2B09F043C08C818F938B81A3
:10F710008F938A818F9389818F93ABE3B9E2BF93F3
:10F72000AF933F922F920F94D92AF10101900020BC
:10F73000E9F73197AF0146575C4320E0B101C801BA
:10F740000E94D0F6C701B6012F81388549855A85B8
:10F750000F9493282F5F3F4F4F4F5F4F6F817885F6
:10F7600089859A850F945128CDBFDEBFA7019601E8
:10F77000285F3F4F4F4F5F4F62177307840795070E
:10F7800019F41092CE20C0C031E03093CE20BCC01E
:10F790001092CE2084149504A604B70479F4EDE702
:10F7A000D101EC9321E041E050E0B101C8010E9499
:10F7B000D0F60FC0ECE2D101EC9304C08091CE20D2
:10F7C000882339F020E041E050E0B101C8010E94F7
:10F7D000D0F6FFEFCF1ADF0AEF0AFF0A2B853C8530
:10F7E0004D855E85C216D306E406F50609F01FCFE7
:10F7F0000E94794C0E9455ED0E9445FF80EE99E3EE
:10F800000F940B216F8580E496E30E940D120E94F5
:10F8100080E780E496E30E94901F81110E94E1EF4F
:10F8200080E496E30E947E26BB24B39474C0B12C7E
:10F8300072C0B12C70C0B12C6EC080E496E30E94FF
:10F8400020128F87F6CCFF24F39480E496E30E9485
:10F85000CA1DB82E882309F45EC0EFCF8C818F9328
:10F860008B818F938A818F9389818F934BE359E2A8
:10F870005F934F933F922F920F94D92AF1010190F9
:10F880000020E9F73197AF0146575C4320E0B10112
:10F89000C8010E94D0F691E09093CE20CDBFDEBF8C
:10F8A000481459046A047B0409F084CF78CF8C8112
:10F8B0008F938B818F938A818F9389818F93EBE3D1
:10F8C000F9E2FF93EF933F922F920F94D92AF1011F
:10F8D00001900020E9F73197AF0146575C4320E0E3
:10F8E000B101C8010E94D0F631E03093CE20CDBFE7
:10F8F000DEBF481459046A047B0409F05BCF4FCF84
:10F90000ECE2D101EC935ACF84149504A604B70419
:10F91000B9F745CFB82E8B2D6396CDBFDEBFDF91F3
:10F92000CF911F910F91FF90EF90DF90CF90BF90FC
:10F93000AF909F908F907F906F905F904F903F908F
:10F940002F900895CF92DF92EF92FF921F93CF9363
:10F95000DF936115710509F474C04630510508F450
:10F9600072C0DB01EC91ED3409F06FC01196EC919F
:10F97000EC3209F06CC02115310509F46AC000971A
:10F9800009F469C069017A01EB012D81203341F44A
:10F9900040E060E00ADC11E0811160C010E05EC070
:10F9A000233541F5C6010E94D71D182F882309F47D
:10F9B00055C0C7010697029718F40E949A950CC08B
:10F9C0008E818C3219F00E949A9506C069EF6E0DF7
:10F9D000CE0107960E946595A601485E5F4FB6016D
:10F9E0006C5C7F4F80E00E94E83E11E0811136C0E0
:10F9F00010E034C00E94E426182F81112EC08D81A2
:10FA00001F928F938DE199E29F938F93C6E7DCE37A
:10FA1000DF93CF930F94D92A09900020E9F721971B
:10FA2000AE0146575C4321E066E77CE38BE093E35D
:10FA30000E94D0F60F900F900F900F900F900F90A4
:10FA40000DC010E00BC010E009C010E007C010E0CE
:10FA500005C010E003C010E001C010E0812FDF916D
:10FA6000CF911F91FF90EF90DF90CF900895FC0110
:10FA7000892BA9F068307105A0F08081813599F457
:10FA800081818C3291F484818C3289F486818C322C
:10FA900081F481E09581903369F080E0089580E001
:10FAA000089580E0089580E0089580E0089580E062
:10FAB000089580E00895EF92FF920F931F93CF93E4
:10FAC000DF9300D0CDB7DEB79CE29B8321153105D3
:10FAD000A9F161157105A1F1FA013197F39790F53C
:10FAE000823390F5803391F5C9017A018B010E9430
:10FAF0002012843069F59E012F5F3F4F41E050E0B6
:10FB0000BE016D5F7F4F80EE99E30F945D1F9E01F4
:10FB10002F5F3F4FA701B80180EE99E30F945D1F5F
:10FB200080EE99E30F940B210E9478F28BE19AE327
:10FB30000E94C78E0E944EF181E00BC080E009C098
:10FB400080E007C080E005C080E003C081E001C024
:10FB500080E02396CDBFDEBFDF91CF911F910F9143
:10FB6000FF90EF900895FC01892B61F063307105DF
:10FB700058F080818C3451F481E091819C3239F0CD
:10FB800080E0089580E0089580E0089580E0089581
:10FB9000452BB1F00097B1F0672BB1F0FC018581E6
:10FBA0008136A1F480E69BE30E94FA8E811110C099
:10FBB00060E070E080E69BE30E94058F81E008959D
:10FBC00080E0089580E0089580E0089580E0089541
:10FBD00080E00895CF93DF93452B11F1009711F149
:10FBE0006531710508F1FC0125812037F9F4278181
:10FBF000203319F410926E3B03C021E020936E3B3A
:10FC0000EC0180E69BE30E94FA8E811111C0BE01D7
:10FC1000675F7F4F80E69BE30E94058F81E009C00C
:10FC200080E007C080E005C080E003C080E001C044
:10FC300080E0DF91CF910895CF93DF93452B31F191
:10FC4000009731F16531710528F1FC0125812E36CF
:10FC500019F52781203319F410926E3B03C021E07F
:10FC600020936E3BEC0180E69BE30E94FA8E8111AB
:10FC700015C080916E3B882399F0BE01675F7F4F6E
:10FC800080E69BE30E94268F81E00BC080E009C0E4
:10FC900080E007C080E005C080E003C080E001C0D4
:10FCA00081E0DF91CF910895009799F0663071055A
:10FCB00090F0FC018581833681F480E69BE30E940D
:10FCC000FA8E882361F00E94A08D1092603B81E043
:10FCD000089580E0089580E0089580E0089581E02F
:10FCE0000895FC01892B49F06630710540F081E0F0
:10FCF0009581933729F080E0089580E0089580E0B1
:10FD00000895FC01892B49F06630710540F081E0CF
:10FD10009581953629F080E0089580E0089580E08F
:10FD20000895BF92CF92DF92EF92FF920F931F93AD
:10FD3000CF93DF9300D0CDB7DEB79CE29B838823BF
:10FD400059F000914E3B002311F010E009C00091E2
:10FD50001B3A10911C3A04C000914F3B1091503B4C
:10FD60000D3291E0190710F00CE211E001151105B8
:10FD700009F44CC0B82E9E012F5F3F4F41E050E088
:10FD8000BE016D5F7F4F80EE99E30F945D1F10926F
:10FD90001D3A10921E3A20E030E0C12CD12C0F2EDB
:10FDA000FBE1EF2EFAE3FF2EF02DF901E55EF54CB5
:10FDB00095819B839E012F5F3F4F41E050E0BE0144
:10FDC0006D5F7F4F80EE99E30F945D1F29813A812B
:10FDD000232B19F4EFEFCE1ADE0AF70122813381CB
:10FDE0002F5F3F4F2283338320173107F0F280EEDD
:10FDF00099E30F940B21B11004C010924F3B109265
:10FE0000503B81E0CD2819F080E001C080E02396CE
:10FE1000CDBFDEBFDF91CF911F910F91FF90EF908B
:10FE2000DF90CF90BF900895FC01892B49F0663098
:10FE3000710540F081E09581943629F080E00895C5
:10FE400080E0089580E00895E6E7FCE32BE7208357
:10FE50002CE621832CE22283662321F02FE62093D7
:10FE6000793C03C025E62093793CE6E7FCE32DE7E7
:10FE70002483158221E045E050E0BF010E94D0F6C6
:10FE80000E94E426811109C021E045E050E066E7C8
:10FE90007CE38BE093E30C94D0F60895EF92FF920D
:10FEA0000F931F93CF93DF936115710509F4F6C18A
:10FEB000009709F4F3C1FB012081222309F4EEC16C
:10FEC000EB018C010E94E426811125C088811F92DC
:10FED0008F9382E299E29F938F930F2EF1EDEF2E95
:10FEE000FDE3FF2EF02DFF92EF920F94D92AF70138
:10FEF00001900020E9F73197AF01415D5D4321E0BA
:10FF0000B7018BE093E30E94D0F60F900F900F9013
:10FF10000F900F900F90888190E08A30910508F043
:10FF2000B7C1FC018827EA53FE4F8F4F0D94D128AB
:10FF300089E998E30E945C8D0E9489F004E71CE344
:10FF40001EC062EF7BE389E998E30E947CF6F8012A
:10FF500080818130A1F40E94E42681110BC0409180
:10FF6000F23B5091F33B21E064EF7BE38BE093E3C2
:10FF70000E94D0F682EF9BE30E946DF607C00E94BC
:10FF8000A0F06838734181059105D8F289819FEF0F
:10FF9000980F983020F088818F5F88837FC1888395
:10FFA0007DC1E6E7FCE383E580838DE481838CE219
:10FFB000828380E38383148221E044E050E0BF0128
:10FFC00089E998E30E94D0F688818F5F88830E9438
:10FFD00089F0C4E7DCE31DC062EF7BE389E998E3C5
:10FFE0000E947CF688818130A1F40E94E426811170
:10FFF0000BC04091F23B5091F33B21E064EF7BE377
:020000021000EC
:100000008BE093E30E94D0F682EF9BE30E946DF6B3
:1000100045C10E94A0F06233710581059105E0F2AF
:100020003DC1E6E7FCE383E5808380E581838CE2E4
:1000300082838E8581110CC081E3838382E3848374
:1000400083E3858384E3868388818F5F88830AC006
:10005000E6E7FCE380E3838384838583868388816A
:100060008F5F888310927D3C21E047E050E066E797
:100070007CE389E998E30E94D0F60E9489F0C4E706
:10008000DCE31DC062EF7BE389E998E30E947CF624
:1000900088818130A1F40E94E42681110BC0409137
:1000A000F23B5091F33B21E064EF7BE38BE093E381
:1000B0000E94D0F682EF9BE30E946DF6EFC00E9493
:1000C000A0F06233710581059105E0F2E7C0E6E733
:1000D000FCE383E5808382E581838CE28283DE0119
:1000E0001296E9E7FCE325E83CE38D918193E21762
:1000F000F307D9F71092853C21E04FE050E066E726
:100100007CE389E998E30E94D0F688818F5F888339
:100110000E9489F0C4E7DCE31DC062EF7BE389E95C
:1001200098E30E947CF688818130A1F40E94E42645
:1001300081110BC04091F23B5091F33B21E064EF01
:100140007BE38BE093E30E94D0F682EF9BE30E9477
:100150006DF6A4C00E94A0F062337105810591057F
:10016000E0F29CC0E6E7FCE382E580838CE28183D9
:1001700081E38283138221E043E050E0BF0189E9FB
:1001800098E30E94D0F688818F5F888387C089E9D1
:1001900098E30E945C8D0E9489F004E71CE31EC076
:1001A00062EF7BE389E998E30E947CF6F8018081A5
:1001B0008130A1F40E94E42681110BC04091F23BF2
:1001C0005091F33B21E064EF7BE38BE093E30E94EB
:1001D000D0F682EF9BE30E946DF607C00E94A0F06C
:1001E0006233710581059105D8F288818F5F88831C
:1001F00055C0E6E7FCE383E480838CE28183DE0183
:100200001296E8E7FCE324E83CE38D918193E21742
:10021000F307D9F71092843C21E04EE050E066E706
:100220007CE389E998E30E94D0F688818F5F888318
:100230000E94CFEC33C00E947C8F882361F061E084
:10024000C80102DE0E94CFEC89E998E30E947E8D0E
:100250001882198223C00E94BBEC81319742F0F0D2
:1002600060E0C801F1DD0E94CFEC89E998E30E94CB
:100270007E8D1882198212C00E94BBEC883E93408A
:1002800068F00E94B18D0E94CFEC1882198206C0DE
:1002900089E998E30E947E8D18821982DF91CF91BF
:1002A0001F910F91FF90EF900895E6E7FCE32BE795
:1002B00020832CE621832CE22283605D63832DE77B
:1002C0002483158221E045E050E0BF010E94D0F672
:1002D0000E94E426811109C021E045E050E066E774
:1002E0007CE38BE093E30C94D0F60895DF92EF92D9
:1002F000FF920F931F93CF93DF93009709F481C16F
:10030000EC01888190E08931910508F075C1FC010C
:100310008827E053FE4F8F4F0D94D12882E194E35C
:100320000E945C8D88818F5F88836BC1E6E7FCE368
:1003300087E480838BE48183128221E042E050E0F5
:10034000BF0182E194E30E94D0F688818F5F8883A9
:100350008FE69BE30E946DF622968CE0FE011192DF
:100360008A95E9F74EC10E9489F0F12C01EF1BE359
:1003700029C06FE67BE382E194E30E947CF6F801FA
:1003800080818130F9F480916F3B9091703B0597AB
:1003900031F48091713B813311F4FF24F3940E9476
:1003A000E42681110BC040916F3B5091703B21E0DE
:1003B00061E77BE38BE093E30E94D0F68FE69BE35B
:1003C0000E946DF60E94A0F06233710581059105CF
:1003D00080F2FF2021F088818F5F888312C188E03E
:1003E00088830FC1E6E7FCE387E4808386E48183AA
:1003F000148221E042E050E0BF0182E194E30E94D8
:10040000D0F688818F5F8883FCC00E9489F0D12C50
:1004100001EF1BE30F2EFDE7EF2EFBE3FF2EF02D88
:100420002EC06FE67BE382E194E30E947CF6F80144
:100430008081813021F580916F3B9091703B0C97CA
:1004400059F4E1E7FBE3DE01129681918D93EE15FD
:10045000FF05D9F7DD24D3940E94E42681110BC057
:1004600040916F3B5091703B21E061E77BE38BE073
:1004700093E30E94D0F68FE69BE30E946DF60E9404
:10048000A0F0623371058105910558F2DD2021F05D
:1004900088818F5F8883B5C088E08883B2C0E6E733
:1004A000FCE383E5808382E581838CE28283DE0145
:1004B0001296E9E7FCE325E83CE38D918193E2178E
:1004C000F307D9F71092853C21E04FE050E066E752
:1004D0007CE382E194E30E94D0F688818F5F888379
:1004E00090C0E6E7FCE383E580838DE481838CE2C2
:1004F000828386E38383148221E044E050E0BF01DD
:1005000082E194E30E94D0F688818F5F888379C06E
:10051000E6E7FCE382E580838CE2818381E38283EA
:10052000138221E043E050E0BF0182E194E30E94A6
:10053000D0F688818F5F888364C08A81811108C06A
:100540004CEC50E267E582E194E30E94176E06C02E
:100550006CEC70E282E194E30E94F26F82E194E33A
:100560000E947E8D18824DC082E194E30E945C8DD2
:1005700088818F5F888345C00E94F1AEBC0182E113
:1005800094E30E94B58D88818F5F88833AC0E6E747
:10059000FCE382E580838CE2818381E382831382A2
:1005A00021E043E050E0BF0182E194E30E94D0F6F5
:1005B00088818F5F888325C082E194E30E947E8DCD
:1005C00018821FC0E6E7FCE382E580838CE281832A
:1005D00081E38283138221E043E050E0BF0182E1A6
:1005E00094E30E94D0F680E496E30E94581D8111A6
:1005F00010924136188205C082E194E30E947E8DFC
:100600001882DF91CF911F910F91FF90EF90DF90B3
:10061000089581E09091513B911101C080E00895CF
:10062000FC01892B61F06330710559F480818134BC
:1006300051F481E091819C3239F080E0089580E0AE
:10064000089580E0089580E00895FC01892B49F029
:100650006330710540F081E09281913329F080E0B0
:10066000089580E0089580E00895FC01892B49F009
:100670006330710540F081E092819E3429F080E082
:10068000089580E0089580E008958091513B8111A4
:100690000BC08CE0E3E5FBE3DF011D928A95E9F7EF
:1006A00081E08093513B089580E008958091513B13
:1006B000811105C084E18093513B81E0089580E081
:1006C0000895FC01892B49F080818F3441F481E049
:1006D00091819C3229F080E0089580E0089580E0C7
:1006E00008950097E9F06A307105E1F4FC01258175
:1006F0002136D1F426812C32C9F420852C32C1F464
:1007000021852133B9F487819FEC980F9730A0F4AD
:100710004115510599F08053FA01808381E00895D5
:1007200080E0089580E0089580E0089580E00895D5
:1007300080E0089580E0089580E0089581E00895C4
:10074000DC01E6E7FCE38BE780838FE681839CE2B4
:10075000928381E683839483605D65838DE78683DE
:100760001782109739F020E047E050E0BF01CD013B
:100770000E94D0F60E94E426811109C021E047E0E2
:1007800050E066E77CE38BE093E30C94D0F60895A9
:100790000E94E426882319F08BE093E302C082E1F3
:1007A00094E3E6E7FCE32BE7208323E721832CE2B5
:1007B000228324E623832DE724831582009731F0DA
:1007C00020E045E050E0BF010E94D0F60E94E42600
:1007D000811109C021E045E050E066E77CE38BE051
:1007E00093E30C94D0F608952F923F924F925F922C
:1007F0006F927F928F929F92AF92BF92CF92DF9231
:10080000EF92FF920F931F93CF93DF93CDB7DEB795
:100810006397CDBFDEBF89879A87062F892B09F49E
:1008200012C281E08093CE2089E10E943BA9672B10
:10083000682B692B09F011C20E942BE1182F81113E
:1008400003C001110BC27DC280E496E30E94CA1D61
:10085000182F882309F475C280E496E30E942012C1
:100860008B8B011104C08150823008F4EEC12B89BA
:10087000243031F480E496E30E94C22633E03B8BBF
:1008800082E10E943BA9672B682B692B21F081E054
:1008900097E09B8703C080E0A6E0AB870E942DC352
:1008A0008B850E943FE365E080E496E30E940D1291
:1008B0000E94BFEF0E94A64B60E072E080E090E0F3
:1008C0000E94984C1092193A10921A3A87EC9CE3C5
:1008D0000E94B2930E94394E8111FCCF182F011152
:1008E00004C00E94BD1C8823E1F389E00E943BA95B
:1008F0006F31710581059105E8F44B015C01072E0C
:100900007CE0880C991CAA1CBB1C7A95D1F7702D31
:10091000C501B4010E94ABE60E9489F081E00E940B
:10092000D9F280E090E1A0E0B0E08D839E83AF83B8
:10093000B88735C04B015C01072E79E0880C991C03
:10094000AA1CBB1C7A95D1F7702DC501B4010E9479
:10095000ABE60E9489F00E9409F380E092E0A0E0FB
:10096000B0E08D839E83AF83B88719C0C12CD12C92
:1009700076010E9446F38823C1F08B850E94D3EE56
:1009800067EC7CE30E941594782E0E9435F39FEF6C
:10099000C91AD90AE90AF90A711007C00BC08114F3
:1009A0009104A104B10411F705C0C814D904EA04E4
:1009B000FB04F8F20E9430F387EC9CE30E947994E8
:1009C000F82E0E94254D0E9455EDFF2031F06B89D5
:1009D00080E496E30E940D12B4C180EF9EE30E9472
:1009E000C1B5882351F0011108C06091EF3F70E05C
:1009F00080EF9EE30E94D99409C0E6E7FCE31082F1
:100A0000118262E070E0CF010E94D99460E072E050
:100A100080E090E00E94AE4B0E94394E8111FCCFE5
:100A200081149104A104B10409F4F8C0C12CD12CA3
:100A300076010F2EF6E72F2EFCE33F2EF02D8D8151
:100A40009E81AF81B8850197A109B1098C879D87E7
:100A5000AE87BF870CE20E94C8948093193A9093A6
:100A60001A3AAE014F5F5F4FBC018B850E94D412D2
:100A7000882309F465C1C701B6012D813E814F81EC
:100A800058850F9493282B013C01672B682B692B09
:100A9000A1F5C701B6012D813E814F8158850F9484
:100AA0009328122F388B498B5A8B89E00E943BA9DF
:100AB000AA89AF93B989BF93E889EF931F939F9356
:100AC0008F937F936F932BE239E23F932F933F9263
:100AD0002F920F94D92AF10101900020E9F7319764
:100AE000AF0146575C4320E0B10189859A850E9499
:100AF000D0F61092CE20CDBFDEBF8D819E81AF811A
:100B0000B8858115E2E09E07A105B10509F4DDC0B5
:100B100081159041A105B10509F4A9C0D701C6010D
:100B200087709927AA27BB27892B8A2B8B2B09F043
:100B300044C08C818F938B818F938A818F9389811D
:100B40008F932BE339E23F932F933F922F920F9491
:100B5000D92AF10101900020E9F73197AF014657FA
:100B60005C4320E0B10189859A850E94D0F6C701D7
:100B7000B6012D813E814F8158850F9493282F5FB8
:100B80003F4F4F4F5F4F6D817E818F8198850F94CE
:100B90005128CDBFDEBFA7019601285F3F4F4F4FC1
:100BA0005F4F621773078407950719F41092CE20E0
:100BB000BDC0B1E0B093CE20B9C01092CE208C85DC
:100BC0009D85AE85BF85481659066A067B0679F471
:100BD000EDE7D101EC9321E041E050E0B1018985DE
:100BE0009A850E94D0F60FC0D1010C9304C0809169
:100BF000CE20882341F020E041E050E0B10189851A
:100C00009A850E94D0F6BFEFCB1ADB0AEB0AFB0AEB
:100C1000C814D904EA04FB0409F01DCF0E94794CE2
:100C20000E9455ED0E9445FF80EE99E30F940B2141
:100C30006B8980E496E30E940D1280E496E30E94A3
:100C40007E2611E07EC010E07CC010E07AC080E417
:100C500096E30E9420128B8B0ACE01E080E496E39B
:100C60000E94CA1D182F882309F46BC0F0CF8C8115
:100C70008F938B818F938A818F9389818F93EBE3FD
:100C8000F9E2FF93EF933F922F920F94D92AF1014B
:100C900001900020E9F73197AF0146575C4320E00F
:100CA000B10189859A850E94D0F631E03093CE203B
:100CB000CDBFDEBF8C859D85AE85BF85841595052E
:100CC000A605B70509F090CF83CF8C818F938B81D8
:100CD0008F938A818F9389818F93ABE3B9E2BF931E
:100CE000AF933F922F920F94D92AF10101900020E7
:100CF000E9F73197AF0146575C4320E0B1018985A0
:100D00009A850E94D0F6F1E0F093CE20CDBFDEBFF1
:100D10008C859D85AE85BF85481659066A067B067B
:100D200009F062CF55CFD1010C9361CF8C859D85A1
:100D3000AE85BF85481659066A067B06A1F748CFDF
:100D4000182F812F6396CDBFDEBFDF91CF911F910A
:100D50000F91FF90EF90DF90CF90BF90AF909F905A
:100D60008F907F906F905F904F903F902F9008955D
:100D7000EF92FF920F931F93CF93DF93611571054D
:100D800009F44CC04630510508F44AC0009709F4F4
:100D900049C0DB01EC91E23509F046C01196EC91B7
:100DA000EC3209F043C02115310509F441C0790145
:100DB0008A01EB012D81263341F440E060E014DD2F
:100DC00091E0811138C090E036C0233599F5C70114
:100DD0000E94D71D982F882371F1C80106970297AA
:100DE00018F40E949A950CC08E818C3219F00E94E2
:100DF0009A9506C069EF600FCE0107960E9465952F
:100E0000A701485E5F4FB7016C5C7F4F81E00E9495
:100E1000E83E91E081110FC090E00DC090E00BC062
:100E200090E009C090E007C090E005C090E003C0EA
:100E300090E001C090E0892FDF91CF911F910F9139
:100E4000FF90EF900895CF93DF93009709F16530FD
:100E5000710500F141155105F9F0FC0120812035A3
:100E6000E9F421812C32E1F422812335D9F49B016C
:100E70002450310921313105B8F4EA016450049657
:100E80000E94BDAECE0148960E942DAF81E00DC0FC
:100E900080E00BC080E009C080E007C080E005C0B2
:100EA00080E003C080E001C080E0DF91CF91089531
:100EB000FC018581803389F4ACECB0E282818C93B3
:100EC000838111968C931197BD018BE093E30E946F
:100ED000F26F80E00E94DB2610C0ACECB0E28281B1
:100EE0008C93838111968C9381E00E94DB266CECBD
:100EF00070E28BE093E30E94F26F81E00895FC01C1
:100F0000892B79F06630710571F480818D3569F433
:100F100081818C3261F481E094819C3249F080E0DF
:100F2000089580E0089580E0089580E0089580E0CD
:100F30000895FC01892B61F06430710559F48081BA
:100F40008E3451F481E091819C3239F080E0089533
:100F500080E0089580E0089580E00895FF920F9367
:100F60001F93CF93DF93009709F445C06115710576
:100F700009F443C0FB018C01C6E7DCE38CE3DE012E
:100F80001D928A95E9F78BE788838EE689838CE248
:100F90008A8390819B8391819C838D8380E496E3F7
:100FA0000E94581DF82E80E496E30E94332B9F93F5
:100FB0008F937F936F931F92FF928CE998E29F9398
:100FC0008F938CE79CE39F938F930F94D92A09907A
:100FD0000020E9F72197AE0146575C4321E066E720
:100FE0007CE3C8010E94D0F68DB79EB70A968DBFEC
:100FF0009EBF81E003C080E001C080E0DF91CF911F
:101000001F910F91FF9008950F931F93CF93DF933C
:1010100000D0CDB7DEB7009739F12091513B2111B7
:1010200025C08C010E94581D882319F081E0F80129
:10103000818382E194E340D58BE489838CE28A83C7
:101040001B8221E042E050E0BE016F5F7F4F82E1F2
:1010500094E30E94D0F688E18093513B0E94F3EC28
:101060000E9455ED81E003C080E001C080E023963E
:10107000CDBFDEBFDF91CF911F910F910895FC018D
:10108000892B61F06430710559F48081883451F402
:1010900081E091819C3239F080E0089580E00895EC
:1010A00080E0089580E008952F923F924F925F92E2
:1010B0006F927F928F929F92AF92BF92CF92DF9268
:1010C000EF92FF920F931F93CF93DF93CDB7DEB7CD
:1010D0002E97CDBFDEBF009709F460C4611571057E
:1010E00009F45CC44115510509F458C421153105B2
:1010F00009F454C4DA01ED91FC91DF011697D797FA
:1011000008F04CC4E60FF71F3197E081ED3709F086
:1011100045C439017A018B0189879A87ECECF0E2AA
:10112000DB0113968C911397808314968C918183A5
:10113000FA01808091805401F2E0AF1AB1086B018E
:101140002FEFC21AD20AB501C601D9DE882321F0D9
:10115000B501C601ADDE22C4D80111969C9190352F
:1011600009F078C1B4E0AB16B10409F073C119827B
:101170000F2EF6E7EF2EFCE3FF2EF02D0F2EFCE3F3
:101180007F2EF02D0F2EFBE78F2EF02D0F2EF0E788
:101190009F2EF02D0F2EFCECAF2EF0E2BF2EF02D87
:1011A0000F2EFCE94F2EF8E25F2EF02D0F2EFCE7FC
:1011B0002F2EFCE33F2EF02DF701272D11922A95BB
:1011C000E9F7D7018C9211969C9211979CE21296A6
:1011D0009C931297F501208113962C9313972181EC
:1011E00014962C93149715969C93863109F072C02F
:1011F0000E940FD66B877C878D879E87672B682B15
:10120000692BC9F489810E943BA920E13EE040E0BE
:1012100050E00F94B5285F934F933F932F938981AC
:101220001F928F935F924F923F922F920F94D92AE1
:10123000CDBFDEBFE0C089810E943BA999233CF568
:1012400089810E943BA920E13EE040E050E00F94FC
:10125000B528CA01B9010E94E9FBAE85AF93BD85EF
:10126000BF93EC85EF93FB85FF939F938F937F93C1
:101270006F9389811F928F9384EA98E29F938F9353
:101280003F922F920F94D92ACDBFDEBFB4C089817F
:101290000E943BA9FE85FF932D852F93AC85AF93CC
:1012A000BB85BF9320E13EE040E050E00F94B528BD
:1012B0005F934F933F932F9389811F928F93E1EB1D
:1012C000F8E2FF93EF933F922F920F94D92ACDBF6C
:1012D000DEBF91C0823090F40E94A0A99F938F93AB
:1012E00089811F928F93A5E9B8E2BF93AF933F9294
:1012F0002F920F94D92ACDBFDEBF7DC08630A1F5D5
:101300001F928F93ADEBB8E2BF93AF933F922F92B2
:101310000F94D92AF70101900020E9F73197CF0106
:1013200086579C436C018A8389810E943BA98B016B
:101330009C01C60199274BE0BE016E5F7F4F8A5822
:10134000934C0E9442FCEA81CE0ECA82EC2DF0E062
:10135000EA58F34C8DE7808311820F900F900F9025
:101360000F900F900F9047C08530A1F51F928F937B
:10137000ADEBB8E2BF93AF933F922F920F94D92A6F
:10138000F70101900020E9F73197CF0186579C4380
:101390006C018A8389810E943BA98B019C01C60153
:1013A00099274BE0BE016E5F7F4F8A58934C0E9495
:1013B0008EFDEA81CE0ECA82EC2DF0E0EA58F34CA5
:1013C0008DE7808311820F900F900F900F900F90F8
:1013D0000F9011C00E943BA99F938F937F936F93AF
:1013E00089811F928F935F924F923F922F920F9419
:1013F000D92ACDBFDEBFF70101900020E9F7319770
:10140000AF0146575C4321E0B70189859A850E9468
:10141000D0F60E94E42681110EC0F7010190002051
:10142000E9F73197AF0146575C4320E0B7018BE005
:1014300093E30E94D0F689818F5F89838C3108F411
:10144000BBCE6CEC70E289859A850E94F26F0E9497
:1014500055EDA4C2B501C6010E948373813009F025
:10146000B0C0AE014D5F5F4FB501C6010E94FF7075
:101470008823C9F0F7016081718162507109C6014A
:101480000E945B71813039F46CEC70E289859A8539
:101490000E94F26F81C24CEC50E26B8189859A8583
:1014A0000E94646E79C2D7016D917C91625071097E
:1014B000AE014D5F5F4FC6010E9472728823C1F07A
:1014C000F7016081718162507109C6010E94B67294
:1014D000813039F46CEC70E289859A850E94F26F54
:1014E0005BC26CEC70E289859A850E94317354C2AC
:1014F000D7010D911C9102501109B801C6010E943B
:10150000D973882369F1CE0104960E94B5238130F6
:10151000D1F4F7016081718162507109A301C601A4
:101520000E94F973813039F46CEC70E289859A85F8
:101530000E94F26F31C24CEC50E267E589859A85D2
:101540000E94176E29C20E94F6D4282F4CEC50E25C
:10155000BE016C5F7F4F89859A850E9425701CC2F1
:10156000B801C6010E9498738823B1F0A301B801A5
:10157000C6010E94C974813039F46CEC70E289852F
:101580009A850E94F26F08C24CEC50E267E58985AB
:101590009A850E94176E00C2B801C6010E94B973F5
:1015A000882339F06CEC70E289859A850E949D75DC
:1015B000F3C14CEC50E267E589859A850E94176E6D
:1015C000EBC1B501C6010E946676813009F069C0A1
:1015D0001886A301B501C6010E9413778130D1F5A9
:1015E0006CEC70E289859A850E94F26FD80116969C
:1015F0008C91833619F0823709F0CEC180E38C8359
:101600008D83BE016C5F7F4F89859A850E949D7591
:10161000C3010E94581D882309F4BEC1E6E7FCE31C
:101620008DE080838AE081839E012A5F3F4F42E004
:1016300050E0BF0180EE99E30F945D1F80EE99E3C7
:101640000F940B2140E060EE79E386E79CE30E9473
:10165000BE44A2C1F70160817181625071099E018F
:10166000285F3F4FA301C6010E948076813089F434
:101670006885611107C06CEC70E289859A850E94CB
:10168000F26F8AC14CEC50E289859A850E94176EF0
:1016900083C14CEC50E267E589859A850E94176EFC
:1016A0007BC1B501C6010E9414788130C1F4930159
:1016B000A501B60189859A850E94A27C813039F402
:1016C0006CEC70E289859A850E94F26F65C14CECE2
:1016D00050E267E589859A850E94176E5DC1B50164
:1016E000C6010E9429788130B9F49301A501B601A1
:1016F00089859A853DDB813039F46CEC70E289850F
:101700009A850E94F26F48C14CEC50E267E58985EA
:101710009A850E94176E40C1B501C6010E94377DAF
:101720008130F1F4D80116968C918983A401495037
:101730005109B801685F7F4F93010E945B7D813042
:1017400039F46CEC70E289859A850E94F26F24C1AD
:101750004CEC50E267E589859A850E94176E1CC1A2
:10176000B501C6010E94B37D813009F09AC0A30182
:10177000B501C6010E94C87D813041F44CEC50E2B5
:1017800061E089859A850E94B67006C1F701608183
:10179000718162507109A301C6010E94EA7D813006
:1017A00041F44CEC50E261E089859A850E94B67064
:1017B000F3C0D7016D917C9162507109A301C601FC
:1017C0000E941C7E813041F44CEC50E261E089853E
:1017D0009A850E94B670E0C0F70160817181625005
:1017E0007109C6010E94547E813039F46CEC70E2BC
:1017F00089859A850E94F26FCFC0D7010D911C9107
:1018000002501109B801C6010E94717E8130F1F4C5
:101810000E9478F280E00E94917E813079F48BE121
:101820009AE3B5D28BE19AE3C4D20E944EF16CECFC
:1018300070E289859A850E94F26FAEC04CEC50E24E
:1018400067E589859A850E94176EA6C0B801C60112
:101850000E94817E813079F48BE19AE398D28BE10A
:101860009AE3A7D20E944EF16CEC70E289859A85CA
:101870000E94F26F91C0B801C6010E94147F8130AE
:1018800041F4FDD26CEC70E289859A850E94F26F7A
:1018900083C04CEC50E267E589859A850E94176EFB
:1018A0007BC0B501C6010E9410838130F1F5B501FE
:1018B000C6010E9425838130A9F40E9445838130AE
:1018C00049F46CEC70E289859A850E94F26F0E945F
:1018D000F3EC62C04CEC50E267E589859A850E9482
:1018E000176E5AC0B501C6010E9435838130A9F434
:1018F0000E945683813049F46CEC70E289859A85A8
:101900000E94F26F0E94F3EC47C04CEC50E267E596
:1019100089859A850E94176E3FC04CEC50E267E5BE
:1019200089859A850E94176E37C0B501C6010E944D
:1019300061838130D9F4AE014F5F5F4FB501C601BD
:101940000E947183813051F489810E94D6116CEC20
:1019500070E289859A850E94F26F1EC04CEC50E2BD
:1019600067E589859A850E94176E16C0B501C60184
:10197000E0DA813031F46CEC70E289859A85EEDA38
:101980000BC0B501C6017BDB813041F46CEC70E229
:1019900089859A850E94F26F0E9455ED2E96CDBFE3
:1019A000DEBFDF91CF911F910F91FF90EF90DF90FD
:1019B000CF90BF90AF909F908F907F906F905F90EF
:1019C0004F903F902F9008956115710559F0411582
:1019D000510541F02115310529F0DB01EC91EB3780
:1019E00009F462CB08950F931F93CF93DF93009771
:1019F00009F45DC06115710509F459C08B01EC0152
:101A00000E948FF7882309F452C0CE010E94A8F7E4
:101A10008D3049F018F48A3031F033C08B3791F0B3
:101A20008D37D9F02EC0F80180819181892B21F466
:101A3000EE57FF4F10823BC0F801EE57FF4F81E099
:101A4000808335C08BE7F801828381E090E080835A
:101A50009183EE57FF4F10822AC0F8018081918157
:101A60008C33910540F4E80FF91F2DE7228301968E
:101A7000F80180839183F801EE57FF4F81E0808366
:101A800016C0F801208131812038310511F410820F
:101A90001182F80120813181E20FF31F82832F5FD1
:101AA0003F4FF80120833183EE57FF4F1082DF91C3
:101AB000CF911F910F910895CF93DF930097D9F0A5
:101AC000EC010E94CFEC0E94BBEC8A3F9105D8F359
:101AD00064E2CE010E945CF764E2CE010E945CF7F2
:101AE00064E2CE010E945CF70E94CFEC0E94BBEC46
:101AF0008A3F9105D8F3DF91CF9108950F931F93FB
:101B0000CF93DF930097B9F08C01C0E0D0E06DE295
:101B1000C8010E945CF720E030E02F5F3F4F20318A
:101B200087E23807D1F72196C330D10581F76DE000
:101B3000C8010E945CF7DF91CF911F910F9108952A
:101B400082E0809366060E94CFEC0E94BBEC892B5A
:101B5000E1F382E080936506089582E08093660653
:101B6000089582E0809365060895CF93DF93EC019A
:101B7000892B09F45CC06115710509F458C0FB019B
:101B800001900020E9F73197E61BF70BE23008F4EB
:101B90004EC04E2FE53108F044E1E6E7FCE383E573
:101BA00080838EE481838CE282834423A9F0DB016D
:101BB000E9E7FCE34150242F30E02658334C9D9157
:101BC0009193E217F307D9F750E060E070E04C5FC3
:101BD0005F4F6F4F7F4F04C043E050E060E070E024
:101BE000CE01FA01EA58F34C1082E6E7FCE30190DB
:101BF0000020E9F73197AF0146575C4321E066E7E3
:101C00007CE30E94D0F60E94E426811110C0E6E732
